 Brackets

 Timestamp is 56ba56f6 (Wed Feb 10 00:15:34 2016)

 Preferred load address is 0000000180000000

 Start         Length     Name                   Class
 0001:00000000 00000010H .00cfg                  CODE
 0001:00000010 00000008H .CRT$XCA                CODE
 0001:00000018 00000008H .CRT$XCZ                CODE
 0001:00000020 00000008H .CRT$XIA                CODE
 0001:00000028 00000018H .CRT$XIC                CODE
 0001:00000040 00000008H .CRT$XIZ                CODE
 0001:00000048 00000008H .CRT$XPA                CODE
 0001:00000050 00000010H .CRT$XPX                CODE
 0001:00000060 00000008H .CRT$XPXA               CODE
 0001:00000068 00000008H .CRT$XPZ                CODE
 0001:00000070 00000008H .CRT$XTA                CODE
 0001:00000078 00000008H .CRT$XTZ                CODE
 0001:00000080 00007454H .rdata                  CODE
 0001:000074d8 000001f4H .rdata$r                CODE
 0001:000076d0 00000010H .rdata$zETW0            CODE
 0001:000076e0 00000077H .rdata$zETW1            CODE
 0001:00007757 0000002cH .rdata$zETW2            CODE
 0001:00007783 00000001H .rdata$zETW9            CODE
 0001:00007784 0000034cH .rdata$zzzdbg           CODE
 0001:00007ad0 00000008H .rtc$IAA                CODE
 0001:00007ad8 00000008H .rtc$IZZ                CODE
 0001:00007ae0 00000008H .rtc$TAA                CODE
 0001:00007ae8 00000008H .rtc$TZZ                CODE
 0001:00007af0 000001dbH .text                   CODE
 0001:00007cd0 0000c1e7H .text$mn                CODE
 0001:00013ec0 00000012H .text$mn$00             CODE
 0001:00013ee0 00000260H .text$x                 CODE
 0001:00014140 00000a54H .xdata                  CODE
 0001:00014b98 000000ecH .xdata$x                CODE
 0001:00014c90 000000a6H .edata                  CODE
 0002:00000000 000009a0H .data                   DATA
 0002:000009a0 000000a0H .data$r                 DATA
 0002:00000a40 00001278H .bss                    DATA
 0003:00000000 00000e58H .pdata                  DATA
 0004:00000000 00000240H .idata$5                DATA
 0004:00000240 0000003cH .idata$2                DATA
 0004:0000027c 00000014H .idata$3                DATA
 0004:00000290 00000240H .idata$4                DATA
 0004:000004d0 00000526H .idata$6                DATA
 0005:00000000 0000007cH .gfids$x                DATA
 0005:0000007c 00000038H .gfids$y                DATA
 0006:00000000 00000058H .rsrc$01                DATA
 0006:00000060 00000380H .rsrc$02                DATA

  Address         Publics by Value              Rva+Base               Lib:Object

 0000:00000000       __guard_iat_table          0000000000000000     <absolute>
 0000:00000000       __guard_iat_count          0000000000000000     <absolute>
 0000:00000000       __guard_longjmp_table      0000000000000000     <absolute>
 0000:00000000       __guard_longjmp_count      0000000000000000     <absolute>
 0000:00000000       __guard_fids_count         0000000000000000     <absolute>
 0000:00000000       ___safe_se_handler_table   0000000000000000     <absolute>
 0000:00000000       ___safe_se_handler_count   0000000000000000     <absolute>
 0000:00000000       __guard_fids_table         0000000000000000     <absolute>
 0000:00000100       __guard_flags              0000000000000100     <absolute>
 0000:00000000       __ImageBase                0000000180000000     <linker-defined>
 0001:00000000       __guard_check_icall_fptr   0000000180001000     LIBCMT:guard_support.obj
 0001:00000008       __guard_dispatch_icall_fptr 0000000180001008     LIBCMT:guard_support.obj
 0001:00000010       __xc_a                     0000000180001010     LIBCMT:initializers.obj
 0001:00000018       __xc_z                     0000000180001018     LIBCMT:initializers.obj
 0001:00000020       __xi_a                     0000000180001020     LIBCMT:initializers.obj
 0001:00000028       __acrt_multibyte_initializer 0000000180001028     libucrt:multibyte_initializer.obj
 0001:00000030       __acrt_stdio_initializer   0000000180001030     libucrt:stdio_initializer.obj
 0001:00000038       __acrt_tran_fma3_initializer 0000000180001038     libucrt:fma3_initializer.obj
 0001:00000040       __xi_z                     0000000180001040     LIBCMT:initializers.obj
 0001:00000048       __xp_a                     0000000180001048     LIBCMT:initializers.obj
 0001:00000050       __acrt_locale_terminator   0000000180001050     libucrt:locale_initializer.obj
 0001:00000058       __dcrt_console_output_terminator 0000000180001058     libucrt:console_output_initializer.obj
 0001:00000060       __acrt_stdio_terminator    0000000180001060     libucrt:stdio_initializer.obj
 0001:00000068       __xp_z                     0000000180001068     LIBCMT:initializers.obj
 0001:00000070       __xt_a                     0000000180001070     LIBCMT:initializers.obj
 0001:00000078       __xt_z                     0000000180001078     LIBCMT:initializers.obj
 0001:00000080       MainGuid                   0000000180001080     Brackets.obj
 0001:00000090       MenuGuid                   0000000180001090     Brackets.obj
 0001:000000a0       DialogGuid                 00000001800010a0     Brackets.obj
 0001:000000b0       ??_7?$DialogItemBinding@UFarDialogItem@@@@6B@ 00000001800010b0     Brackets.obj
 0001:000000c0       ??_7PluginCheckBoxBinding@@6B@ 00000001800010c0     Brackets.obj
 0001:000000d0       ??_7PluginRadioButtonBinding@@6B@ 00000001800010d0     Brackets.obj
 0001:000000e0       ??_7PluginEditFieldBinding@@6B@ 00000001800010e0     Brackets.obj
 0001:000000f0       ??_7PluginIntEditFieldBinding@@6B@ 00000001800010f0     Brackets.obj
 0001:00000100       ??_C@_15EFLNJKHH@?$AA?$CF?$AAu?$AA?$AA@ 0000000180001100     Brackets.obj
 0001:00000108       ??_7PluginUIntEditFieldBinding@@6B@ 0000000180001108     Brackets.obj
 0001:00000118       ??_7?$DialogBuilderBase@UFarDialogItem@@@@6B@ 0000000180001118     Brackets.obj
 0001:00000160       ??_7PluginDialogBuilder@@6B@ 0000000180001160     Brackets.obj
 0001:000001a8       ??_C@_11LOCGONAA@?$AA?$AA@ 00000001800011a8     Brackets.obj
 0001:000001b0       ??_C@_1BC@GJFAHMHB@?$AAB?$AAr?$AAa?$AAc?$AAk?$AAe?$AAt?$AAs?$AA?$AA@ 00000001800011b0     Brackets.obj
 0001:000001d0       ??_C@_1EE@CJLEEDHO@?$AAB?$AAr?$AAa?$AAc?$AAk?$AAe?$AAt?$AAs?$AA?5?$AAm?$AAa?$AAt?$AAc?$AAh?$AAi?$AAn?$AAg?$AA?5?$AAf?$AAo?$AAr?$AA?5?$AAF?$AAa?$AAr?$AA?5?$AAM?$AAa?$AAn?$AAa?$AAg?$AAe@ 00000001800011d0     Brackets.obj
 0001:00000218       ??_C@_1DE@BGKMIKPD@?$AAE?$AAu?$AAg?$AAe?$AAn?$AAe?$AA?5?$AAR?$AAo?$AAs?$AAh?$AAa?$AAl?$AA?5?$AA?$CG?$AA?5?$AAF?$AAa?$AAr?$AA?5?$AAG?$AAr?$AAo?$AAu?$AAp?$AA?$AA@ 0000000180001218     Brackets.obj
 0001:00000250       ??_C@_1BK@LFBLPBJM@?$AAI?$AAg?$AAn?$AAo?$AAr?$AAe?$AAQ?$AAu?$AAo?$AAt?$AAe?$AAs?$AA?$AA@ 0000000180001250     Brackets.obj
 0001:00000270       ??_C@_1BI@LPBIFPPH@?$AAI?$AAg?$AAn?$AAo?$AAr?$AAe?$AAA?$AAf?$AAt?$AAe?$AAr?$AA?$AA@ 0000000180001270     Brackets.obj
 0001:00000288       ??_C@_1BK@LJLNAEDP@?$AAB?$AAr?$AAa?$AAc?$AAk?$AAe?$AAt?$AAP?$AAr?$AAi?$AAo?$AAr?$AA?$AA@ 0000000180001288     Brackets.obj
 0001:000002a8       ??_C@_1BG@KDMBKMK@?$AAJ?$AAu?$AAm?$AAp?$AAT?$AAo?$AAP?$AAa?$AAi?$AAr?$AA?$AA@ 00000001800012a8     Brackets.obj
 0001:000002c0       ??_C@_19CNDHNALO@?$AAB?$AAe?$AAe?$AAp?$AA?$AA@ 00000001800012c0     Brackets.obj
 0001:000002d0       ??_C@_1BG@KHOAFHB@?$AA?8?$AA?8?$AA?$CC?$AA?$CC?$AA?$GA?$AA?8?$AA?$GA?$AA?$GA?5?$BO?5?$BN?$AA?$AA@ 00000001800012d0     Brackets.obj
 0001:000002e8       ??_C@_1BG@ICHMEPOB@?$AAQ?$AAu?$AAo?$AAt?$AAe?$AAs?$AAT?$AAy?$AAp?$AAe?$AA?$AA@ 00000001800012e8     Brackets.obj
 0001:00000300       ??_C@_1CC@FLEKOJBB@?$AA?$DM?$AA?$DO?$AA?$HL?$AA?$HN?$AA?$FL?$AA?$FN?$AA?$CI?$AA?$CJ?$AA?$CC?$AA?$CC?$AA?8?$AA?8?$AA?$CF?$AA?$CF?$AA?$KL?$AA?$LL?$AA?$AA@ 0000000180001300     Brackets.obj
 0001:00000328       ??_C@_1BE@CHAAIDDE@?$AAB?$AAr?$AAa?$AAc?$AAk?$AAe?$AAt?$AAs?$AA1?$AA?$AA@ 0000000180001328     Brackets.obj
 0001:00000340       ??_C@_1BK@EKFLELHE@?$AA?1?$AA?$CK?$AA?$CK?$AA?1?$AA?$DM?$AA?$DP?$AA?$DP?$AA?$DO?$AA?$DM?$AA?$CF?$AA?$CF?$AA?$DO?$AA?$AA@ 0000000180001340     Brackets.obj
 0001:00000360       ??_C@_1BE@DFLFCMNK@?$AAB?$AAr?$AAa?$AAc?$AAk?$AAe?$AAt?$AAs?$AA2?$AA?$AA@ 0000000180001360     Brackets.obj
 0001:00000378       ??_C@_19MGMPFFIA@?$AAF?$AAi?$AAn?$AAd?$AA?$AA@ 0000000180001378     Brackets.obj
 0001:00000388       ??_C@_1O@MDCABJAO@?$AAD?$AAi?$AAr?$AAe?$AAc?$AAt?$AA?$AA@ 0000000180001388     Brackets.obj
 0001:00000398       ??_C@_1BE@LCCGEFEM@?$AAS?$AAE?$AAA?$AAR?$AAC?$AAH?$AAF?$AAW?$AAD?$AA?$AA@ 0000000180001398     Brackets.obj
 0001:000003b0       ??_C@_1BG@LIFFHAGC@?$AAS?$AAE?$AAA?$AAR?$AAC?$AAH?$AAB?$AAA?$AAC?$AAK?$AA?$AA@ 00000001800013b0     Brackets.obj
 0001:000003c8       ??_C@_1BE@IFIBPANP@?$AAS?$AAE?$AAL?$AAE?$AAC?$AAT?$AAF?$AAW?$AAD?$AA?$AA@ 00000001800013c8     Brackets.obj
 0001:000003e0       ??_C@_1BG@FJDCNJBP@?$AAS?$AAE?$AAL?$AAE?$AAC?$AAT?$AAB?$AAA?$AAC?$AAK?$AA?$AA@ 00000001800013e0     Brackets.obj
 0001:000003f8       ??_C@_1O@BAHOLLMK@?$AAC?$AAO?$AAN?$AAF?$AAI?$AAG?$AA?$AA@ 00000001800013f8     Brackets.obj
 0001:00000410       __xmm@ffffffffffffffff0000000000000002 0000000180001410     Brackets.obj
 0001:00000420       __xmm@ffffffffffffffffffffffffffffffff 0000000180001420     Brackets.obj
 0001:00000430       _pRawDllMain               0000000180001430     LIBCMT:dll_dllmain.obj
 0001:00000430       _pDefaultRawDllMain        0000000180001430     LIBCMT:dll_dllmain.obj
 0001:00000440       ??_7exception@std@@6B@     0000000180001440     LIBCMT:throw_bad_alloc.obj
 0001:00000450       ??_C@_0BC@EOODALEL@Unknown?5exception?$AA@ 0000000180001450     LIBCMT:throw_bad_alloc.obj
 0001:00000470       ??_7bad_alloc@std@@6B@     0000000180001470     LIBCMT:throw_bad_alloc.obj
 0001:00000480       ??_C@_0P@GHFPNOJB@bad?5allocation?$AA@ 0000000180001480     LIBCMT:throw_bad_alloc.obj
 0001:00000498       ??_7bad_array_new_length@std@@6B@ 0000000180001498     LIBCMT:throw_bad_alloc.obj
 0001:000004a8       ??_C@_0BF@KINCDENJ@bad?5array?5new?5length?$AA@ 00000001800014a8     LIBCMT:throw_bad_alloc.obj
 0001:000004c8       ??_7type_info@@6B@         00000001800014c8     LIBCMT:std_type_info_static.obj
 0001:000004d0       _Microsoft_CRTProvider     00000001800014d0     libvcruntime:telemetry.obj
 0001:000004d8       ??_C@_00CNPNBAHC@?$AA@     00000001800014d8     libvcruntime:telemetry.obj
 0001:000004e0       ??_C@_0O@JEOPJOMI@Main?5Invoked?4?$AA@ 00000001800014e0     libvcruntime:telemetry.obj
 0001:000004f0       ??_C@_0P@NEAEIBDO@Main?5Returned?4?$AA@ 00000001800014f0     libvcruntime:telemetry.obj
 0001:00000560       ??_C@_1BC@DNHGCMLG@?$AAa?$AAd?$AAv?$AAa?$AAp?$AAi?$AA3?$AA2?$AA?$AA@ 0000000180001560     libvcruntime:winapi_downlevel.obj
 0001:00000578       ??_C@_1DM@KHCHBNEB@?$AAa?$AAp?$AAi?$AA?9?$AAm?$AAs?$AA?9?$AAw?$AAi?$AAn?$AA?9?$AAc?$AAo?$AAr?$AAe?$AA?9?$AAf?$AAi?$AAb?$AAe?$AAr?$AAs?$AA?9?$AAl?$AA1?$AA?9?$AA1?$AA?9?$AA1?$AA?$AA@ 0000000180001578     libvcruntime:winapi_downlevel.obj
 0001:000005b8       ??_C@_1DK@LPPGFMPP@?$AAa?$AAp?$AAi?$AA?9?$AAm?$AAs?$AA?9?$AAw?$AAi?$AAn?$AA?9?$AAc?$AAo?$AAr?$AAe?$AA?9?$AAs?$AAy?$AAn?$AAc?$AAh?$AA?9?$AAl?$AA1?$AA?9?$AA2?$AA?9?$AA0?$AA?$AA@ 00000001800015b8     libvcruntime:winapi_downlevel.obj
 0001:000005f8       ??_C@_1BC@GDMECMAK@?$AAk?$AAe?$AAr?$AAn?$AAe?$AAl?$AA3?$AA2?$AA?$AA@ 00000001800015f8     libvcruntime:winapi_downlevel.obj
 0001:00000610       ??_C@_0O@BAMBGLIE@EventRegister?$AA@ 0000000180001610     libvcruntime:winapi_downlevel.obj
 0001:00000628       ??_C@_0BE@BJEEGHGK@EventSetInformation?$AA@ 0000000180001628     libvcruntime:winapi_downlevel.obj
 0001:00000640       ??_C@_0BA@FAKLIPIC@EventUnregister?$AA@ 0000000180001640     libvcruntime:winapi_downlevel.obj
 0001:00000658       ??_C@_0BD@PKLHJPHD@EventWriteTransfer?$AA@ 0000000180001658     libvcruntime:winapi_downlevel.obj
 0001:00000678       ??_C@_08KNHFBNJ@FlsAlloc?$AA@ 0000000180001678     libvcruntime:winapi_downlevel.obj
 0001:00000690       ??_C@_07PEJMOBNF@FlsFree?$AA@ 0000000180001690     libvcruntime:winapi_downlevel.obj
 0001:000006a0       ??_C@_0M@GDNOONDI@FlsGetValue?$AA@ 00000001800016a0     libvcruntime:winapi_downlevel.obj
 0001:000006b8       ??_C@_0M@JCPCPOEF@FlsSetValue?$AA@ 00000001800016b8     libvcruntime:winapi_downlevel.obj
 0001:000006d0       ??_C@_0BM@HCFOFFN@InitializeCriticalSectionEx?$AA@ 00000001800016d0     libvcruntime:winapi_downlevel.obj
 0001:000006ec       ??_C@_01JOAMLHOP@?9?$AA@   00000001800016ec     libvcruntime:undname.obj
 0001:000006f0       ??_C@_01MIFGBAGJ@?$CL?$AA@ 00000001800016f0     libvcruntime:undname.obj
 0001:000006f4       ??_C@_01HNPIGOCE@?$CG?$AA@ 00000001800016f4     libvcruntime:undname.obj
 0001:000006f8       ??_C@_03MNHNFDLC@?9?$DO?$CK?$AA@ 00000001800016f8     libvcruntime:undname.obj
 0001:000006fc       ??_C@_01KMDKNFGN@?1?$AA@   00000001800016fc     libvcruntime:undname.obj
 0001:00000700       ??_C@_01FGNFDNOH@?$CF?$AA@ 0000000180001700     libvcruntime:undname.obj
 0001:00000704       ??_C@_01MNNFJEPP@?$DM?$AA@ 0000000180001704     libvcruntime:undname.obj
 0001:00000708       ??_C@_02EHCHHCKH@?$DM?$DN?$AA@ 0000000180001708     libvcruntime:undname.obj
 0001:0000070c       ??_C@_01PPODPGHN@?$DO?$AA@ 000000018000170c     libvcruntime:undname.obj
 0001:00000710       ??_C@_02EEKDKGMJ@?$DO?$DN?$AA@ 0000000180001710     libvcruntime:undname.obj
 0001:00000714       ??_C@_01IHBHIGKO@?0?$AA@   0000000180001714     libvcruntime:undname.obj
 0001:00000718       ??_C@_02HCKGKOFO@?$CI?$CJ?$AA@ 0000000180001718     libvcruntime:undname.obj
 0001:0000071c       ??_C@_01PJKLJHI@?$HO?$AA@  000000018000171c     libvcruntime:undname.obj
 0001:00000720       ??_C@_01JKBOJNNK@?$FO?$AA@ 0000000180001720     libvcruntime:undname.obj
 0001:00000724       ??_C@_01DNKMNLPK@?$HM?$AA@ 0000000180001724     libvcruntime:undname.obj
 0001:00000728       ??_C@_02PPKAJPJL@?$CG?$CG?$AA@ 0000000180001728     libvcruntime:undname.obj
 0001:0000072c       ??_C@_02NONPIBCD@?$HM?$HM?$AA@ 000000018000172c     libvcruntime:undname.obj
 0001:00000730       ??_C@_02FPIMKNGF@?$CK?$DN?$AA@ 0000000180001730     libvcruntime:undname.obj
 0001:00000734       ??_C@_02FOEOMHFC@?$CL?$DN?$AA@ 0000000180001734     libvcruntime:undname.obj
 0001:00000738       ??_C@_02FKMDLLOA@?9?$DN?$AA@ 0000000180001738     libvcruntime:undname.obj
 0001:0000073c       ??_C@_02FJEHGPIO@?1?$DN?$AA@ 000000018000173c     libvcruntime:undname.obj
 0001:00000740       ??_C@_02FENAOKFI@?$CF?$DN?$AA@ 0000000180001740     libvcruntime:undname.obj
 0001:00000744       ??_C@_03IKFCCPFF@?$DO?$DO?$DN?$AA@ 0000000180001744     libvcruntime:undname.obj
 0001:00000748       ??_C@_03CDNPDDLA@?$DM?$DM?$DN?$AA@ 0000000180001748     libvcruntime:undname.obj
 0001:0000074c       ??_C@_02FGJGFEAB@?$CG?$DN?$AA@ 000000018000174c     libvcruntime:undname.obj
 0001:00000750       ??_C@_02DHLNPPGH@?$HM?$DN?$AA@ 0000000180001750     libvcruntime:undname.obj
 0001:00000754       ??_C@_02MHEGNOJ@?$FO?$DN?$AA@ 0000000180001754     libvcruntime:undname.obj
 0001:00000758       ??_C@_09IFPLHPGF@?$GAvftable?8?$AA@ 0000000180001758     libvcruntime:undname.obj
 0001:00000768       ??_C@_09BLBHBJP@?$GAvbtable?8?$AA@ 0000000180001768     libvcruntime:undname.obj
 0001:00000778       ??_C@_07FEEIOKP@?$GAvcall?8?$AA@ 0000000180001778     libvcruntime:undname.obj
 0001:00000780       ??_C@_08LLFFHHDJ@?$GAtypeof?8?$AA@ 0000000180001780     libvcruntime:undname.obj
 0001:00000790       ??_C@_0BF@KDPPACIK@?$GAlocal?5static?5guard?8?$AA@ 0000000180001790     libvcruntime:undname.obj
 0001:000007a8       ??_C@_08OBABFOLI@?$GAstring?8?$AA@ 00000001800017a8     libvcruntime:undname.obj
 0001:000007b8       ??_C@_0BD@JDLKDPAB@?$GAvbase?5destructor?8?$AA@ 00000001800017b8     libvcruntime:undname.obj
 0001:000007d0       ??_C@_0BN@DEGPLNFK@?$GAvector?5deleting?5destructor?8?$AA@ 00000001800017d0     libvcruntime:undname.obj
 0001:000007f0       ??_C@_0BO@OBMKPJIG@?$GAdefault?5constructor?5closure?8?$AA@ 00000001800017f0     libvcruntime:undname.obj
 0001:00000810       ??_C@_0BN@IMDCHIKM@?$GAscalar?5deleting?5destructor?8?$AA@ 0000000180001810     libvcruntime:undname.obj
 0001:00000830       ??_C@_0BO@PFGOCPJJ@?$GAvector?5constructor?5iterator?8?$AA@ 0000000180001830     libvcruntime:undname.obj
 0001:00000850       ??_C@_0BN@LFPFMEDL@?$GAvector?5destructor?5iterator?8?$AA@ 0000000180001850     libvcruntime:undname.obj
 0001:00000870       ??_C@_0CE@IKBNEHA@?$GAvector?5vbase?5constructor?5iterat@ 0000000180001870     libvcruntime:undname.obj
 0001:00000898       ??_C@_0BL@NILFHHPC@?$GAvirtual?5displacement?5map?8?$AA@ 0000000180001898     libvcruntime:undname.obj
 0001:000008b8       ??_C@_0CB@JONCMFFK@?$GAeh?5vector?5constructor?5iterator?8@ 00000001800018b8     libvcruntime:undname.obj
 0001:000008e0       ??_C@_0CA@GCEOPDGL@?$GAeh?5vector?5destructor?5iterator?8?$AA@ 00000001800018e0     libvcruntime:undname.obj
 0001:00000900       ??_C@_0CH@OOJPLCPH@?$GAeh?5vector?5vbase?5constructor?5ite@ 0000000180001900     libvcruntime:undname.obj
 0001:00000928       ??_C@_0BL@LLKPOHJI@?$GAcopy?5constructor?5closure?8?$AA@ 0000000180001928     libvcruntime:undname.obj
 0001:00000948       ??_C@_0BA@KBCDOMBN@?$GAudt?5returning?8?$AA@ 0000000180001948     libvcruntime:undname.obj
 0001:00000958       ??_C@_03KLGMFNMG@?$GAEH?$AA@ 0000000180001958     libvcruntime:undname.obj
 0001:0000095c       ??_C@_05KHLCHHI@?$GARTTI?$AA@ 000000018000195c     libvcruntime:undname.obj
 0001:00000968       ??_C@_0BA@KKLDJDLB@?$GAlocal?5vftable?8?$AA@ 0000000180001968     libvcruntime:undname.obj
 0001:00000978       ??_C@_0CE@IIHCMGGL@?$GAlocal?5vftable?5constructor?5closu@ 0000000180001978     libvcruntime:undname.obj
 0001:0000099c       ??_C@_06FHBGPFGH@?5new?$FL?$FN?$AA@ 000000018000199c     libvcruntime:undname.obj
 0001:000009a8       ??_C@_09LBNFPBCA@?5delete?$FL?$FN?$AA@ 00000001800019a8     libvcruntime:undname.obj
 0001:000009b8       ??_C@_0P@HJKNJFNN@?$GAomni?5callsig?8?$AA@ 00000001800019b8     libvcruntime:undname.obj
 0001:000009c8       ??_C@_0BL@CNOONJFP@?$GAplacement?5delete?5closure?8?$AA@ 00000001800019c8     libvcruntime:undname.obj
 0001:000009e8       ??_C@_0BN@CKNJLHMB@?$GAplacement?5delete?$FL?$FN?5closure?8?$AA@ 00000001800019e8     libvcruntime:undname.obj
 0001:00000a08       ??_C@_0CG@CFDHKGGD@?$GAmanaged?5vector?5constructor?5iter@ 0000000180001a08     libvcruntime:undname.obj
 0001:00000a30       ??_C@_0CF@IMGKMJNO@?$GAmanaged?5vector?5destructor?5itera@ 0000000180001a30     libvcruntime:undname.obj
 0001:00000a58       ??_C@_0CG@HLDDJMAG@?$GAeh?5vector?5copy?5constructor?5iter@ 0000000180001a58     libvcruntime:undname.obj
 0001:00000a80       ??_C@_0CM@FCBBDIGB@?$GAeh?5vector?5vbase?5copy?5constructo@ 0000000180001a80     libvcruntime:undname.obj
 0001:00000ab0       ??_C@_0BL@CLIPGLGB@?$GAdynamic?5initializer?5for?5?8?$AA@ 0000000180001ab0     libvcruntime:undname.obj
 0001:00000ad0       ??_C@_0CB@PDBIFEP@?$GAdynamic?5atexit?5destructor?5for?5?8@ 0000000180001ad0     libvcruntime:undname.obj
 0001:00000af8       ??_C@_0CD@CGAJBKEJ@?$GAvector?5copy?5constructor?5iterato@ 0000000180001af8     libvcruntime:undname.obj
 0001:00000b20       ??_C@_0CJ@GJELGAMM@?$GAvector?5vbase?5copy?5constructor?5i@ 0000000180001b20     libvcruntime:undname.obj
 0001:00000b50       ??_C@_0CL@FGIJHLCE@?$GAmanaged?5vector?5copy?5constructor@ 0000000180001b50     libvcruntime:undname.obj
 0001:00000b80       ??_C@_0BM@PMGGMLDN@?$GAlocal?5static?5thread?5guard?8?$AA@ 0000000180001b80     libvcruntime:undname.obj
 0001:00000ba0       ??_C@_0N@BDNMDMOL@operator?5?$CC?$CC?5?$AA@ 0000000180001ba0     libvcruntime:undname.obj
 0001:00000ed8       ??_C@_0BC@DAFEJGAK@?5Type?5Descriptor?8?$AA@ 0000000180001ed8     libvcruntime:undname.obj
 0001:00000ef0       ??_C@_0BM@LDKODKLH@?5Base?5Class?5Descriptor?5at?5?$CI?$AA@ 0000000180001ef0     libvcruntime:undname.obj
 0001:00000f10       ??_C@_0BD@LGICGFMM@?5Base?5Class?5Array?8?$AA@ 0000000180001f10     libvcruntime:undname.obj
 0001:00000f28       ??_C@_0BN@MECKDCOJ@?5Class?5Hierarchy?5Descriptor?8?$AA@ 0000000180001f28     libvcruntime:undname.obj
 0001:00000f48       ??_C@_0BK@CFCOFLF@?5Complete?5Object?5Locator?8?$AA@ 0000000180001f48     libvcruntime:undname.obj
 0001:00000f68       ??_C@_08EHJDFFNH@__based?$CI?$AA@ 0000000180001f68     libvcruntime:undname.obj
 0001:00000f78       ??_C@_07KOLFKCDI@__cdecl?$AA@ 0000000180001f78     libvcruntime:undname.obj
 0001:00000f80       ??_C@_08GHMPAG@__pascal?$AA@ 0000000180001f80     libvcruntime:undname.obj
 0001:00000f90       ??_C@_09IFJBGAPI@__stdcall?$AA@ 0000000180001f90     libvcruntime:undname.obj
 0001:00000fa0       ??_C@_0L@NPHFGOKO@__thiscall?$AA@ 0000000180001fa0     libvcruntime:undname.obj
 0001:00000fb0       ??_C@_0L@JMKHOMEK@__fastcall?$AA@ 0000000180001fb0     libvcruntime:undname.obj
 0001:00000fc0       ??_C@_0N@BCKKPABJ@__vectorcall?$AA@ 0000000180001fc0     libvcruntime:undname.obj
 0001:00000fd0       ??_C@_09HIJEGCPM@__clrcall?$AA@ 0000000180001fd0     libvcruntime:undname.obj
 0001:00000fdc       ??_C@_06GHPCKEAG@__eabi?$AA@ 0000000180001fdc     libvcruntime:undname.obj
 0001:00000fe8       ??_C@_07JOMMBBKO@__ptr64?$AA@ 0000000180001fe8     libvcruntime:undname.obj
 0001:00000ff0       ??_C@_0L@PILCLIHE@__restrict?$AA@ 0000000180001ff0     libvcruntime:undname.obj
 0001:00001000       ??_C@_0M@GFIIJFMG@__unaligned?$AA@ 0000000180002000     libvcruntime:undname.obj
 0001:00001010       ??_C@_09DHDLOLLB@restrict?$CI?$AA@ 0000000180002010     libvcruntime:undname.obj
 0001:0000101c       ??_C@_04NIHEBCM@?5new?$AA@ 000000018000201c     libvcruntime:undname.obj
 0001:00001028       ??_C@_07FPCDHGMM@?5delete?$AA@ 0000000180002028     libvcruntime:undname.obj
 0001:00001030       ??_C@_01NEMOKFLO@?$DN?$AA@ 0000000180002030     libvcruntime:undname.obj
 0001:00001034       ??_C@_02GPIOPFAK@?$DO?$DO?$AA@ 0000000180002034     libvcruntime:undname.obj
 0001:00001038       ??_C@_02FODMEDOG@?$DM?$DM?$AA@ 0000000180002038     libvcruntime:undname.obj
 0001:0000103c       ??_C@_01DCLJPIOD@?$CB?$AA@ 000000018000203c     libvcruntime:undname.obj
 0001:00001040       ??_C@_02EGOFBIJA@?$DN?$DN?$AA@ 0000000180002040     libvcruntime:undname.obj
 0001:00001044       ??_C@_02FDNJECIE@?$CB?$DN?$AA@ 0000000180002044     libvcruntime:undname.obj
 0001:00001048       ??_C@_02GPECMEKF@?$FL?$FN?$AA@ 0000000180002048     libvcruntime:undname.obj
 0001:00001050       ??_C@_08LHJFAFGD@operator?$AA@ 0000000180002050     libvcruntime:undname.obj
 0001:0000105c       ??_C@_02HBOOOICD@?9?$DO?$AA@ 000000018000205c     libvcruntime:undname.obj
 0001:00001060       ??_C@_01NBENCBCI@?$CK?$AA@ 0000000180002060     libvcruntime:undname.obj
 0001:00001064       ??_C@_02ECNGHCIF@?$CL?$CL?$AA@ 0000000180002064     libvcruntime:undname.obj
 0001:00001068       ??_C@_02BAABKJLB@?9?9?$AA@ 0000000180002068     libvcruntime:undname.obj
 0001:00001070       __acrt_exception_action_table 0000000180002070     libucrt:exception_filter.obj
 0001:00001130       __acrt_signal_action_table_count 0000000180002130     libucrt:exception_filter.obj
 0001:00001138       __acrt_signal_action_first_fpe_index 0000000180002138     libucrt:exception_filter.obj
 0001:00001140       __acrt_signal_action_fpe_count 0000000180002140     libucrt:exception_filter.obj
 0001:00001148       ??_C@_1BI@BGOHAHKC@?$AAm?$AAs?$AAc?$AAo?$AAr?$AAe?$AAe?$AA?4?$AAd?$AAl?$AAl?$AA?$AA@ 0000000180002148     libucrt:exit.obj
 0001:00001160       ??_C@_0P@MIGLKIOC@CorExitProcess?$AA@ 0000000180002160     libucrt:exit.obj
 0001:00001300       ??_C@_1EG@CNNIPFIM@?$AAa?$AAp?$AAi?$AA?9?$AAm?$AAs?$AA?9?$AAw?$AAi?$AAn?$AA?9?$AAa?$AAp?$AAp?$AAm?$AAo?$AAd?$AAe?$AAl?$AA?9?$AAr?$AAu?$AAn?$AAt?$AAi?$AAm?$AAe?$AA?9?$AAl?$AA1?$AA?9?$AA1@ 0000000180002300     libucrt:winapi_thunks.obj
 0001:00001350       ??_C@_1EA@JGEFHKEI@?$AAa?$AAp?$AAi?$AA?9?$AAm?$AAs?$AA?9?$AAw?$AAi?$AAn?$AA?9?$AAc?$AAo?$AAr?$AAe?$AA?9?$AAd?$AAa?$AAt?$AAe?$AAt?$AAi?$AAm?$AAe?$AA?9?$AAl?$AA1?$AA?9?$AA1?$AA?9?$AA1?$AA?$AA@ 0000000180002350     libucrt:winapi_thunks.obj
 0001:00001390       ??_C@_1DI@GCIAAENM@?$AAa?$AAp?$AAi?$AA?9?$AAm?$AAs?$AA?9?$AAw?$AAi?$AAn?$AA?9?$AAc?$AAo?$AAr?$AAe?$AA?9?$AAf?$AAi?$AAl?$AAe?$AA?9?$AAl?$AA2?$AA?9?$AA1?$AA?9?$AA1?$AA?$AA@ 0000000180002390     libucrt:winapi_thunks.obj
 0001:000013d0       ??_C@_1EI@MPIAOHOC@?$AAa?$AAp?$AAi?$AA?9?$AAm?$AAs?$AA?9?$AAw?$AAi?$AAn?$AA?9?$AAc?$AAo?$AAr?$AAe?$AA?9?$AAl?$AAo?$AAc?$AAa?$AAl?$AAi?$AAz?$AAa?$AAt?$AAi?$AAo?$AAn?$AA?9?$AAl?$AA1?$AA?9@ 00000001800023d0     libucrt:winapi_thunks.obj
 0001:00001420       ??_C@_1FK@FPHCKFIE@?$AAa?$AAp?$AAi?$AA?9?$AAm?$AAs?$AA?9?$AAw?$AAi?$AAn?$AA?9?$AAc?$AAo?$AAr?$AAe?$AA?9?$AAl?$AAo?$AAc?$AAa?$AAl?$AAi?$AAz?$AAa?$AAt?$AAi?$AAo?$AAn?$AA?9?$AAo?$AAb?$AAs@ 0000000180002420     libucrt:winapi_thunks.obj
 0001:00001480       ??_C@_1EM@DILCGIIO@?$AAa?$AAp?$AAi?$AA?9?$AAm?$AAs?$AA?9?$AAw?$AAi?$AAn?$AA?9?$AAc?$AAo?$AAr?$AAe?$AA?9?$AAp?$AAr?$AAo?$AAc?$AAe?$AAs?$AAs?$AAt?$AAh?$AAr?$AAe?$AAa?$AAd?$AAs?$AA?9?$AAl@ 0000000180002480     libucrt:winapi_thunks.obj
 0001:000014d0       ??_C@_1DM@LNCGDDPN@?$AAa?$AAp?$AAi?$AA?9?$AAm?$AAs?$AA?9?$AAw?$AAi?$AAn?$AA?9?$AAc?$AAo?$AAr?$AAe?$AA?9?$AAs?$AAt?$AAr?$AAi?$AAn?$AAg?$AA?9?$AAl?$AA1?$AA?9?$AA1?$AA?9?$AA0?$AA?$AA@ 00000001800024d0     libucrt:winapi_thunks.obj
 0001:00001510       ??_C@_1DO@FPAPJEMD@?$AAa?$AAp?$AAi?$AA?9?$AAm?$AAs?$AA?9?$AAw?$AAi?$AAn?$AA?9?$AAc?$AAo?$AAr?$AAe?$AA?9?$AAs?$AAy?$AAs?$AAi?$AAn?$AAf?$AAo?$AA?9?$AAl?$AA1?$AA?9?$AA2?$AA?9?$AA1?$AA?$AA@ 0000000180002510     libucrt:winapi_thunks.obj
 0001:00001550       ??_C@_1DK@NDHNAHIO@?$AAa?$AAp?$AAi?$AA?9?$AAm?$AAs?$AA?9?$AAw?$AAi?$AAn?$AA?9?$AAc?$AAo?$AAr?$AAe?$AA?9?$AAw?$AAi?$AAn?$AAr?$AAt?$AA?9?$AAl?$AA1?$AA?9?$AA1?$AA?9?$AA0?$AA?$AA@ 0000000180002550     libucrt:winapi_thunks.obj
 0001:00001590       ??_C@_1DM@KGHDGBCM@?$AAa?$AAp?$AAi?$AA?9?$AAm?$AAs?$AA?9?$AAw?$AAi?$AAn?$AA?9?$AAc?$AAo?$AAr?$AAe?$AA?9?$AAx?$AAs?$AAt?$AAa?$AAt?$AAe?$AA?9?$AAl?$AA2?$AA?9?$AA1?$AA?9?$AA0?$AA?$AA@ 0000000180002590     libucrt:winapi_thunks.obj
 0001:000015d0       ??_C@_1EO@IJIOEFOH@?$AAa?$AAp?$AAi?$AA?9?$AAm?$AAs?$AA?9?$AAw?$AAi?$AAn?$AA?9?$AAr?$AAt?$AAc?$AAo?$AAr?$AAe?$AA?9?$AAn?$AAt?$AAu?$AAs?$AAe?$AAr?$AA?9?$AAw?$AAi?$AAn?$AAd?$AAo?$AAw?$AA?9@ 00000001800025d0     libucrt:winapi_thunks.obj
 0001:00001620       ??_C@_1FG@HHGEKANL@?$AAa?$AAp?$AAi?$AA?9?$AAm?$AAs?$AA?9?$AAw?$AAi?$AAn?$AA?9?$AAs?$AAe?$AAc?$AAu?$AAr?$AAi?$AAt?$AAy?$AA?9?$AAs?$AAy?$AAs?$AAt?$AAe?$AAm?$AAf?$AAu?$AAn?$AAc?$AAt?$AAi@ 0000000180002620     libucrt:winapi_thunks.obj
 0001:00001680       ??_C@_1FG@NCKKOLKO@?$AAe?$AAx?$AAt?$AA?9?$AAm?$AAs?$AA?9?$AAw?$AAi?$AAn?$AA?9?$AAk?$AAe?$AAr?$AAn?$AAe?$AAl?$AA3?$AA2?$AA?9?$AAp?$AAa?$AAc?$AAk?$AAa?$AAg?$AAe?$AA?9?$AAc?$AAu?$AAr?$AAr@ 0000000180002680     libucrt:winapi_thunks.obj
 0001:000016e0       ??_C@_1EG@DBIOJECG@?$AAe?$AAx?$AAt?$AA?9?$AAm?$AAs?$AA?9?$AAw?$AAi?$AAn?$AA?9?$AAn?$AAt?$AAu?$AAs?$AAe?$AAr?$AA?9?$AAd?$AAi?$AAa?$AAl?$AAo?$AAg?$AAb?$AAo?$AAx?$AA?9?$AAl?$AA1?$AA?9?$AA1@ 00000001800026e0     libucrt:winapi_thunks.obj
 0001:00001730       ??_C@_1EO@FIHMJCLF@?$AAe?$AAx?$AAt?$AA?9?$AAm?$AAs?$AA?9?$AAw?$AAi?$AAn?$AA?9?$AAn?$AAt?$AAu?$AAs?$AAe?$AAr?$AA?9?$AAw?$AAi?$AAn?$AAd?$AAo?$AAw?$AAs?$AAt?$AAa?$AAt?$AAi?$AAo?$AAn?$AA?9@ 0000000180002730     libucrt:winapi_thunks.obj
 0001:00001780       ??_C@_1O@BCCLBEOE@?$AAu?$AAs?$AAe?$AAr?$AA3?$AA2?$AA?$AA@ 0000000180002780     libucrt:winapi_thunks.obj
 0001:000017b8       ??_C@_0BE@JOGNEJCI@GetCurrentPackageId?$AA@ 00000001800027b8     libucrt:winapi_thunks.obj
 0001:000017e0       ??_C@_0O@KKBNKAPF@LCMapStringEx?$AA@ 00000001800027e0     libucrt:winapi_thunks.obj
 0001:000017f8       ??_C@_0BB@HBDEELFH@LocaleNameToLCID?$AA@ 00000001800027f8     libucrt:winapi_thunks.obj
 0001:00001830       ??_C@_1M@HPNHIDJI@?$AAj?$AAa?$AA?9?$AAJ?$AAP?$AA?$AA@ 0000000180002830     libucrt:mbctype.obj
 0001:00001840       ??_C@_1M@BIBDDEMK@?$AAz?$AAh?$AA?9?$AAC?$AAN?$AA?$AA@ 0000000180002840     libucrt:mbctype.obj
 0001:00001850       ??_C@_1M@JLOOOEGK@?$AAk?$AAo?$AA?9?$AAK?$AAR?$AA?$AA@ 0000000180002850     libucrt:mbctype.obj
 0001:00001860       ??_C@_1M@CLNBBOPM@?$AAz?$AAh?$AA?9?$AAT?$AAW?$AA?$AA@ 0000000180002860     libucrt:mbctype.obj
 0001:00001870       __lc_time_c                0000000180002870     libucrt:nlsdata.obj
 0001:00001b30       ??_C@_03KOEHGMDN@Sun?$AA@  0000000180002b30     libucrt:nlsdata.obj
 0001:00001b34       ??_C@_03PDAGKDH@Mon?$AA@   0000000180002b34     libucrt:nlsdata.obj
 0001:00001b38       ??_C@_03NAGEINEP@Tue?$AA@  0000000180002b38     libucrt:nlsdata.obj
 0001:00001b3c       ??_C@_03MHOMLAJA@Wed?$AA@  0000000180002b3c     libucrt:nlsdata.obj
 0001:00001b40       ??_C@_03IOFIKPDN@Thu?$AA@  0000000180002b40     libucrt:nlsdata.obj
 0001:00001b44       ??_C@_03IDIOELNC@Fri?$AA@  0000000180002b44     libucrt:nlsdata.obj
 0001:00001b48       ??_C@_03FEFJNEK@Sat?$AA@   0000000180002b48     libucrt:nlsdata.obj
 0001:00001b4c       ??_C@_06OOPIFAJ@Sunday?$AA@ 0000000180002b4c     libucrt:nlsdata.obj
 0001:00001b54       ??_C@_06JLEDEDGH@Monday?$AA@ 0000000180002b54     libucrt:nlsdata.obj
 0001:00001b60       ??_C@_07BAAGCFCM@Tuesday?$AA@ 0000000180002b60     libucrt:nlsdata.obj
 0001:00001b68       ??_C@_09DLIGFAKA@Wednesday?$AA@ 0000000180002b68     libucrt:nlsdata.obj
 0001:00001b78       ??_C@_08HACCIKIA@Thursday?$AA@ 0000000180002b78     libucrt:nlsdata.obj
 0001:00001b84       ??_C@_06JECMNKMI@Friday?$AA@ 0000000180002b84     libucrt:nlsdata.obj
 0001:00001b90       ??_C@_08INBOOONO@Saturday?$AA@ 0000000180002b90     libucrt:nlsdata.obj
 0001:00001b9c       ??_C@_03JIHJHPIE@Jan?$AA@  0000000180002b9c     libucrt:nlsdata.obj
 0001:00001ba0       ??_C@_03HJBDCHOM@Feb?$AA@  0000000180002ba0     libucrt:nlsdata.obj
 0001:00001ba4       ??_C@_03ODNJBKGA@Mar?$AA@  0000000180002ba4     libucrt:nlsdata.obj
 0001:00001ba8       ??_C@_03LEOLGMJP@Apr?$AA@  0000000180002ba8     libucrt:nlsdata.obj
 0001:00001bac       ??_C@_03CNMDKL@May?$AA@    0000000180002bac     libucrt:nlsdata.obj
 0001:00001bb0       ??_C@_03IDFGHECI@Jun?$AA@  0000000180002bb0     libucrt:nlsdata.obj
 0001:00001bb4       ??_C@_03LBGABGKK@Jul?$AA@  0000000180002bb4     libucrt:nlsdata.obj
 0001:00001bb8       ??_C@_03IFJFEIGA@Aug?$AA@  0000000180002bb8     libucrt:nlsdata.obj
 0001:00001bbc       ??_C@_03GGCAPAJC@Sep?$AA@  0000000180002bbc     libucrt:nlsdata.obj
 0001:00001bc0       ??_C@_03BMAOKBAD@Oct?$AA@  0000000180002bc0     libucrt:nlsdata.obj
 0001:00001bc4       ??_C@_03JPJOFNIA@Nov?$AA@  0000000180002bc4     libucrt:nlsdata.obj
 0001:00001bc8       ??_C@_03MKABNOCG@Dec?$AA@  0000000180002bc8     libucrt:nlsdata.obj
 0001:00001bd0       ??_C@_07CGJPFGJA@January?$AA@ 0000000180002bd0     libucrt:nlsdata.obj
 0001:00001bd8       ??_C@_08GNJGEPFN@February?$AA@ 0000000180002bd8     libucrt:nlsdata.obj
 0001:00001be4       ??_C@_05HPCKOFNC@March?$AA@ 0000000180002be4     libucrt:nlsdata.obj
 0001:00001bec       ??_C@_05DMJDNLEJ@April?$AA@ 0000000180002bec     libucrt:nlsdata.obj
 0001:00001bf4       ??_C@_04CNLMGBGM@June?$AA@ 0000000180002bf4     libucrt:nlsdata.obj
 0001:00001bfc       ??_C@_04MIEPOIFP@July?$AA@ 0000000180002bfc     libucrt:nlsdata.obj
 0001:00001c04       ??_C@_06LBBHFDDG@August?$AA@ 0000000180002c04     libucrt:nlsdata.obj
 0001:00001c10       ??_C@_09BHHEALKD@September?$AA@ 0000000180002c10     libucrt:nlsdata.obj
 0001:00001c20       ??_C@_07JJNFCEND@October?$AA@ 0000000180002c20     libucrt:nlsdata.obj
 0001:00001c28       ??_C@_08HCHEGEOA@November?$AA@ 0000000180002c28     libucrt:nlsdata.obj
 0001:00001c38       ??_C@_08EDHMEBNP@December?$AA@ 0000000180002c38     libucrt:nlsdata.obj
 0001:00001c44       ??_C@_02DEDBPAFC@AM?$AA@   0000000180002c44     libucrt:nlsdata.obj
 0001:00001c48       ??_C@_02CJNFDJBF@PM?$AA@   0000000180002c48     libucrt:nlsdata.obj
 0001:00001c50       ??_C@_08BPBNCDIB@MM?1dd?1yy?$AA@ 0000000180002c50     libucrt:nlsdata.obj
 0001:00001c60       ??_C@_0BE@CKGJFCPC@dddd?0?5MMMM?5dd?0?5yyyy?$AA@ 0000000180002c60     libucrt:nlsdata.obj
 0001:00001c78       ??_C@_08JCCMCCIL@HH?3mm?3ss?$AA@ 0000000180002c78     libucrt:nlsdata.obj
 0001:00001c88       ??_C@_17MBGCMIPB@?$AAS?$AAu?$AAn?$AA?$AA@ 0000000180002c88     libucrt:nlsdata.obj
 0001:00001c90       ??_C@_17KBOMKBF@?$AAM?$AAo?$AAn?$AA?$AA@ 0000000180002c90     libucrt:nlsdata.obj
 0001:00001c98       ??_C@_17BMKGEGOJ@?$AAT?$AAu?$AAe?$AA?$AA@ 0000000180002c98     libucrt:nlsdata.obj
 0001:00001ca0       ??_C@_17CJEDCEPE@?$AAW?$AAe?$AAd?$AA?$AA@ 0000000180002ca0     libucrt:nlsdata.obj
 0001:00001ca8       ??_C@_17PDPHAADD@?$AAT?$AAh?$AAu?$AA?$AA@ 0000000180002ca8     libucrt:nlsdata.obj
 0001:00001cb0       ??_C@_17HFOLPPLP@?$AAF?$AAr?$AAi?$AA?$AA@ 0000000180002cb0     libucrt:nlsdata.obj
 0001:00001cb8       ??_C@_17GGIBDPIH@?$AAS?$AAa?$AAt?$AA?$AA@ 0000000180002cb8     libucrt:nlsdata.obj
 0001:00001cc0       ??_C@_1O@IHNHDHPB@?$AAS?$AAu?$AAn?$AAd?$AAa?$AAy?$AA?$AA@ 0000000180002cc0     libucrt:nlsdata.obj
 0001:00001cd0       ??_C@_1O@MMNBFLIA@?$AAM?$AAo?$AAn?$AAd?$AAa?$AAy?$AA?$AA@ 0000000180002cd0     libucrt:nlsdata.obj
 0001:00001ce0       ??_C@_1BA@ENFBFFEK@?$AAT?$AAu?$AAe?$AAs?$AAd?$AAa?$AAy?$AA?$AA@ 0000000180002ce0     libucrt:nlsdata.obj
 0001:00001cf0       ??_C@_1BE@EBOGMDOH@?$AAW?$AAe?$AAd?$AAn?$AAe?$AAs?$AAd?$AAa?$AAy?$AA?$AA@ 0000000180002cf0     libucrt:nlsdata.obj
 0001:00001d08       ??_C@_1BC@HHMNLIHE@?$AAT?$AAh?$AAu?$AAr?$AAs?$AAd?$AAa?$AAy?$AA?$AA@ 0000000180002d08     libucrt:nlsdata.obj
 0001:00001d20       ??_C@_1O@PDICJHAG@?$AAF?$AAr?$AAi?$AAd?$AAa?$AAy?$AA?$AA@ 0000000180002d20     libucrt:nlsdata.obj
 0001:00001d30       ??_C@_1BC@ENMNNPAJ@?$AAS?$AAa?$AAt?$AAu?$AAr?$AAd?$AAa?$AAy?$AA?$AA@ 0000000180002d30     libucrt:nlsdata.obj
 0001:00001d48       ??_C@_17DKNBKCHM@?$AAJ?$AAa?$AAn?$AA?$AA@ 0000000180002d48     libucrt:nlsdata.obj
 0001:00001d50       ??_C@_17LMDJEKJN@?$AAF?$AAe?$AAb?$AA?$AA@ 0000000180002d50     libucrt:nlsdata.obj
 0001:00001d58       ??_C@_17CKNLEDEC@?$AAM?$AAa?$AAr?$AA?$AA@ 0000000180002d58     libucrt:nlsdata.obj
 0001:00001d60       ??_C@_17LFPOIHDD@?$AAA?$AAp?$AAr?$AA?$AA@ 0000000180002d60     libucrt:nlsdata.obj
 0001:00001d68       ??_C@_17PNNKMEED@?$AAM?$AAa?$AAy?$AA?$AA@ 0000000180002d68     libucrt:nlsdata.obj
 0001:00001d70       ??_C@_17KCJGOCPB@?$AAJ?$AAu?$AAn?$AA?$AA@ 0000000180002d70     libucrt:nlsdata.obj
 0001:00001d78       ??_C@_17IJPCKHK@?$AAJ?$AAu?$AAl?$AA?$AA@ 0000000180002d78     libucrt:nlsdata.obj
 0001:00001d80       ??_C@_17ICPELBCN@?$AAA?$AAu?$AAg?$AA?$AA@ 0000000180002d80     libucrt:nlsdata.obj
 0001:00001d88       ??_C@_17HCHCOKMG@?$AAS?$AAe?$AAp?$AA?$AA@ 0000000180002d88     libucrt:nlsdata.obj
 0001:00001d90       ??_C@_17FNLKOI@?$AAO?$AAc?$AAt?$AA?$AA@ 0000000180002d90     libucrt:nlsdata.obj
 0001:00001d98       ??_C@_17BBDMLCIG@?$AAN?$AAo?$AAv?$AA?$AA@ 0000000180002d98     libucrt:nlsdata.obj
 0001:00001da0       ??_C@_17EGKACKIF@?$AAD?$AAe?$AAc?$AA?$AA@ 0000000180002da0     libucrt:nlsdata.obj
 0001:00001da8       ??_C@_1BA@EFMEIEBA@?$AAJ?$AAa?$AAn?$AAu?$AAa?$AAr?$AAy?$AA?$AA@ 0000000180002da8     libucrt:nlsdata.obj
 0001:00001db8       ??_C@_1BC@JGDDFFAM@?$AAF?$AAe?$AAb?$AAr?$AAu?$AAa?$AAr?$AAy?$AA?$AA@ 0000000180002db8     libucrt:nlsdata.obj
 0001:00001dd0       ??_C@_1M@IKEENEDF@?$AAM?$AAa?$AAr?$AAc?$AAh?$AA?$AA@ 0000000180002dd0     libucrt:nlsdata.obj
 0001:00001de0       ??_C@_1M@GJNLMHFD@?$AAA?$AAp?$AAr?$AAi?$AAl?$AA?$AA@ 0000000180002de0     libucrt:nlsdata.obj
 0001:00001df0       ??_C@_19EPFLPGAP@?$AAJ?$AAu?$AAn?$AAe?$AA?$AA@ 0000000180002df0     libucrt:nlsdata.obj
 0001:00001e00       ??_C@_19BIFMLPCD@?$AAJ?$AAu?$AAl?$AAy?$AA?$AA@ 0000000180002e00     libucrt:nlsdata.obj
 0001:00001e10       ??_C@_1O@PAHLKOAC@?$AAA?$AAu?$AAg?$AAu?$AAs?$AAt?$AA?$AA@ 0000000180002e10     libucrt:nlsdata.obj
 0001:00001e20       ??_C@_1BE@DKAAMBJL@?$AAS?$AAe?$AAp?$AAt?$AAe?$AAm?$AAb?$AAe?$AAr?$AA?$AA@ 0000000180002e20     libucrt:nlsdata.obj
 0001:00001e38       ??_C@_1BA@EPANDLNG@?$AAO?$AAc?$AAt?$AAo?$AAb?$AAe?$AAr?$AA?$AA@ 0000000180002e38     libucrt:nlsdata.obj
 0001:00001e48       ??_C@_1BC@BGLIFPF@?$AAN?$AAo?$AAv?$AAe?$AAm?$AAb?$AAe?$AAr?$AA?$AA@ 0000000180002e48     libucrt:nlsdata.obj
 0001:00001e60       ??_C@_1BC@FEMKIFH@?$AAD?$AAe?$AAc?$AAe?$AAm?$AAb?$AAe?$AAr?$AA?$AA@ 0000000180002e60     libucrt:nlsdata.obj
 0001:00001e74       ??_C@_15ODEHAHHF@?$AAA?$AAM?$AA?$AA@ 0000000180002e74     libucrt:nlsdata.obj
 0001:00001e7c       ??_C@_15CLMNNGEL@?$AAP?$AAM?$AA?$AA@ 0000000180002e7c     libucrt:nlsdata.obj
 0001:00001e88       ??_C@_1BC@IEBCMHCM@?$AAM?$AAM?$AA?1?$AAd?$AAd?$AA?1?$AAy?$AAy?$AA?$AA@ 0000000180002e88     libucrt:nlsdata.obj
 0001:00001ea0       ??_C@_1CI@KNAKOEBC@?$AAd?$AAd?$AAd?$AAd?$AA?0?$AA?5?$AAM?$AAM?$AAM?$AAM?$AA?5?$AAd?$AAd?$AA?0?$AA?5?$AAy?$AAy?$AAy?$AAy?$AA?$AA@ 0000000180002ea0     libucrt:nlsdata.obj
 0001:00001ec8       ??_C@_1BC@GDGBMEMK@?$AAH?$AAH?$AA?3?$AAm?$AAm?$AA?3?$AAs?$AAs?$AA?$AA@ 0000000180002ec8     libucrt:nlsdata.obj
 0001:00001ee0       ??_C@_1M@BMHNFIME@?$AAe?$AAn?$AA?9?$AAU?$AAS?$AA?$AA@ 0000000180002ee0     libucrt:nlsdata.obj
 0001:00002060       __newctype                 0000000180003060     libucrt:ctype.obj
 0001:00002360       __newclmap                 0000000180003360     libucrt:ctype.obj
 0001:000024e0       __newcumap                 00000001800034e0     libucrt:ctype.obj
 0001:000034a0       ??_C@_15EMKDOKLE@?$AAa?$AAr?$AA?$AA@ 00000001800044a0     libucrt:lcidtoname_downlevel.obj
 0001:000034a8       ??_C@_15KNPADPLH@?$AAb?$AAg?$AA?$AA@ 00000001800044a8     libucrt:lcidtoname_downlevel.obj
 0001:000034b0       ??_C@_15EDMHLDMO@?$AAc?$AAa?$AA?$AA@ 00000001800044b0     libucrt:lcidtoname_downlevel.obj
 0001:000034b8       ??_C@_1O@BPEAJADD@?$AAz?$AAh?$AA?9?$AAC?$AAH?$AAS?$AA?$AA@ 00000001800044b8     libucrt:lcidtoname_downlevel.obj
 0001:000034c8       ??_C@_15LJNHCMNK@?$AAc?$AAs?$AA?$AA@ 00000001800044c8     libucrt:lcidtoname_downlevel.obj
 0001:000034d0       ??_C@_15FOMCIDHG@?$AAd?$AAa?$AA?$AA@ 00000001800044d0     libucrt:lcidtoname_downlevel.obj
 0001:000034d8       ??_C@_15NBKABECB@?$AAd?$AAe?$AA?$AA@ 00000001800044d8     libucrt:lcidtoname_downlevel.obj
 0001:000034e0       ??_C@_15GHPEIIAO@?$AAe?$AAl?$AA?$AA@ 00000001800044e0     libucrt:lcidtoname_downlevel.obj
 0001:000034e8       ??_C@_15MNPNEAIF@?$AAe?$AAn?$AA?$AA@ 00000001800044e8     libucrt:lcidtoname_downlevel.obj
 0001:000034f0       ??_C@_15GPIOMPMH@?$AAe?$AAs?$AA?$AA@ 00000001800044f0     libucrt:lcidtoname_downlevel.obj
 0001:000034f8       ??_C@_15NGLOAKJC@?$AAf?$AAi?$AA?$AA@ 00000001800044f8     libucrt:lcidtoname_downlevel.obj
 0001:00003500       ??_C@_15FBKGNKAM@?$AAf?$AAr?$AA?$AA@ 0000000180004500     libucrt:lcidtoname_downlevel.obj
 0001:00003508       ??_C@_15KGGCNEFK@?$AAh?$AAe?$AA?$AA@ 0000000180004508     libucrt:lcidtoname_downlevel.obj
 0001:00003510       ??_C@_15PGHLIDMF@?$AAh?$AAu?$AA?$AA@ 0000000180004510     libucrt:lcidtoname_downlevel.obj
 0001:00003518       ??_C@_15BIEMAPLM@?$AAi?$AAs?$AA?$AA@ 0000000180004518     libucrt:lcidtoname_downlevel.obj
 0001:00003520       ??_C@_15IFJLDHAF@?$AAi?$AAt?$AA?$AA@ 0000000180004520     libucrt:lcidtoname_downlevel.obj
 0001:00003528       ??_C@_15GEMIOCAG@?$AAj?$AAa?$AA?$AA@ 0000000180004528     libucrt:lcidtoname_downlevel.obj
 0001:00003530       ??_C@_15EPELEGJA@?$AAk?$AAo?$AA?$AA@ 0000000180004530     libucrt:lcidtoname_downlevel.obj
 0001:00003538       ??_C@_15NDDHIMN@?$AAn?$AAl?$AA?$AA@ 0000000180004538     libucrt:lcidtoname_downlevel.obj
 0001:00003540       ??_C@_15BPIGNHCD@?$AAn?$AAo?$AA?$AA@ 0000000180004540     libucrt:lcidtoname_downlevel.obj
 0001:00003548       ??_C@_15DEOPBLCG@?$AAp?$AAl?$AA?$AA@ 0000000180004548     libucrt:lcidtoname_downlevel.obj
 0001:00003550       ??_C@_15KBECGEFG@?$AAp?$AAt?$AA?$AA@ 0000000180004550     libucrt:lcidtoname_downlevel.obj
 0001:00003558       ??_C@_15GLJCBFMD@?$AAr?$AAo?$AA?$AA@ 0000000180004558     libucrt:lcidtoname_downlevel.obj
 0001:00003560       ??_C@_15FEDGKCDI@?$AAr?$AAu?$AA?$AA@ 0000000180004560     libucrt:lcidtoname_downlevel.obj
 0001:00003568       ??_C@_15GLKMLLHM@?$AAh?$AAr?$AA?$AA@ 0000000180004568     libucrt:lcidtoname_downlevel.obj
 0001:00003570       ??_C@_15CPKMFBDB@?$AAs?$AAk?$AA?$AA@ 0000000180004570     libucrt:lcidtoname_downlevel.obj
 0001:00003578       ??_C@_15BAAIOGMK@?$AAs?$AAq?$AA?$AA@ 0000000180004578     libucrt:lcidtoname_downlevel.obj
 0001:00003580       ??_C@_15INNPNOHD@?$AAs?$AAv?$AA?$AA@ 0000000180004580     libucrt:lcidtoname_downlevel.obj
 0001:00003588       ??_C@_15CABMMOGH@?$AAt?$AAh?$AA?$AA@ 0000000180004588     libucrt:lcidtoname_downlevel.obj
 0001:00003590       ??_C@_15BPLIHJJM@?$AAt?$AAr?$AA?$AA@ 0000000180004590     libucrt:lcidtoname_downlevel.obj
 0001:00003598       ??_C@_15NEOEKKDJ@?$AAu?$AAr?$AA?$AA@ 0000000180004598     libucrt:lcidtoname_downlevel.obj
 0001:000035a0       ??_C@_15NFICGAJK@?$AAi?$AAd?$AA?$AA@ 00000001800045a0     libucrt:lcidtoname_downlevel.obj
 0001:000035a8       ??_C@_15PJPFLCCM@?$AAu?$AAk?$AA?$AA@ 00000001800045a8     libucrt:lcidtoname_downlevel.obj
 0001:000035b0       ??_C@_15HPJPHDM@?$AAb?$AAe?$AA?$AA@ 00000001800045b0     libucrt:lcidtoname_downlevel.obj
 0001:000035b8       ??_C@_15LCHLGJII@?$AAs?$AAl?$AA?$AA@ 00000001800045b8     libucrt:lcidtoname_downlevel.obj
 0001:000035c0       ??_C@_15PCFJPHHO@?$AAe?$AAt?$AA?$AA@ 00000001800045c0     libucrt:lcidtoname_downlevel.obj
 0001:000035c8       ??_C@_15HPFPGODN@?$AAl?$AAv?$AA?$AA@ 00000001800045c8     libucrt:lcidtoname_downlevel.obj
 0001:000035d0       ??_C@_15NFFGKGLG@?$AAl?$AAt?$AA?$AA@ 00000001800045d0     libucrt:lcidtoname_downlevel.obj
 0001:000035d8       ??_C@_15BDAKCCHN@?$AAf?$AAa?$AA?$AA@ 00000001800045d8     libucrt:lcidtoname_downlevel.obj
 0001:000035e0       ??_C@_15NFGIAIAJ@?$AAv?$AAi?$AA?$AA@ 00000001800045e0     libucrt:lcidtoname_downlevel.obj
 0001:000035e8       ??_C@_15LMKNDMHN@?$AAh?$AAy?$AA?$AA@ 00000001800045e8     libucrt:lcidtoname_downlevel.obj
 0001:000035f0       ??_C@_15IJBHMCFL@?$AAa?$AAz?$AA?$AA@ 00000001800045f0     libucrt:lcidtoname_downlevel.obj
 0001:000035f8       ??_C@_15EKOFJABL@?$AAe?$AAu?$AA?$AA@ 00000001800045f8     libucrt:lcidtoname_downlevel.obj
 0001:00003600       ??_C@_15BGHADCNK@?$AAm?$AAk?$AA?$AA@ 0000000180004600     libucrt:lcidtoname_downlevel.obj
 0001:00003608       ??_C@_15JDNICKHM@?$AAa?$AAf?$AA?$AA@ 0000000180004608     libucrt:lcidtoname_downlevel.obj
 0001:00003610       ??_C@_15KPJEDBKD@?$AAk?$AAa?$AA?$AA@ 0000000180004610     libucrt:lcidtoname_downlevel.obj
 0001:00003618       ??_C@_15PDNFFFEO@?$AAf?$AAo?$AA?$AA@ 0000000180004618     libucrt:lcidtoname_downlevel.obj
 0001:00003620       ??_C@_15OMLEGLOC@?$AAh?$AAi?$AA?$AA@ 0000000180004620     libucrt:lcidtoname_downlevel.obj
 0001:00003628       ??_C@_15IDNNENKK@?$AAm?$AAs?$AA?$AA@ 0000000180004628     libucrt:lcidtoname_downlevel.obj
 0001:00003630       ??_C@_15MACJNBMH@?$AAk?$AAk?$AA?$AA@ 0000000180004630     libucrt:lcidtoname_downlevel.obj
 0001:00003638       ??_C@_15DKDJEOND@?$AAk?$AAy?$AA?$AA@ 0000000180004638     libucrt:lcidtoname_downlevel.obj
 0001:00003640       ??_C@_15DFGDLJBG@?$AAs?$AAw?$AA?$AA@ 0000000180004640     libucrt:lcidtoname_downlevel.obj
 0001:00003648       ??_C@_15BBFAICNG@?$AAu?$AAz?$AA?$AA@ 0000000180004648     libucrt:lcidtoname_downlevel.obj
 0001:00003650       ??_C@_15DKNDCGEA@?$AAt?$AAt?$AA?$AA@ 0000000180004650     libucrt:lcidtoname_downlevel.obj
 0001:00003658       ??_C@_15MGIFMDPL@?$AAp?$AAa?$AA?$AA@ 0000000180004658     libucrt:lcidtoname_downlevel.obj
 0001:00003660       ??_C@_15HCNDBBA@?$AAg?$AAu?$AA?$AA@ 0000000180004660     libucrt:lcidtoname_downlevel.obj
 0001:00003668       ??_C@_15FNBEIBON@?$AAt?$AAa?$AA?$AA@ 0000000180004668     libucrt:lcidtoname_downlevel.obj
 0001:00003670       ??_C@_15NCHGBGLK@?$AAt?$AAe?$AA?$AA@ 0000000180004670     libucrt:lcidtoname_downlevel.obj
 0001:00003678       ??_C@_15PHPHCBPF@?$AAk?$AAn?$AA?$AA@ 0000000180004678     libucrt:lcidtoname_downlevel.obj
 0001:00003680       ??_C@_15DLGBCKMP@?$AAm?$AAr?$AA?$AA@ 0000000180004680     libucrt:lcidtoname_downlevel.obj
 0001:00003688       ??_C@_15EABBLBFF@?$AAs?$AAa?$AA?$AA@ 0000000180004688     libucrt:lcidtoname_downlevel.obj
 0001:00003690       ??_C@_15CBKOMCOI@?$AAm?$AAn?$AA?$AA@ 0000000180004690     libucrt:lcidtoname_downlevel.obj
 0001:00003698       ??_C@_15CKDMCJAF@?$AAg?$AAl?$AA?$AA@ 0000000180004698     libucrt:lcidtoname_downlevel.obj
 0001:000036a0       ??_C@_17CNJFBPG@?$AAk?$AAo?$AAk?$AA?$AA@ 00000001800046a0     libucrt:lcidtoname_downlevel.obj
 0001:000036a8       ??_C@_17FFBJICPL@?$AAs?$AAy?$AAr?$AA?$AA@ 00000001800046a8     libucrt:lcidtoname_downlevel.obj
 0001:000036b0       ??_C@_17KPNDCPAF@?$AAd?$AAi?$AAv?$AA?$AA@ 00000001800046b0     libucrt:lcidtoname_downlevel.obj
 0001:000036b8       ??_C@_1M@OKAHONE@?$AAa?$AAr?$AA?9?$AAS?$AAA?$AA?$AA@ 00000001800046b8     libucrt:lcidtoname_downlevel.obj
 0001:000036c8       ??_C@_1M@FFFIGIGK@?$AAb?$AAg?$AA?9?$AAB?$AAG?$AA?$AA@ 00000001800046c8     libucrt:lcidtoname_downlevel.obj
 0001:000036d8       ??_C@_1M@BJNKEDC@?$AAc?$AAa?$AA?9?$AAE?$AAS?$AA?$AA@ 00000001800046d8     libucrt:lcidtoname_downlevel.obj
 0001:000036e8       ??_C@_1M@IJJHFJHA@?$AAc?$AAs?$AA?9?$AAC?$AAZ?$AA?$AA@ 00000001800046e8     libucrt:lcidtoname_downlevel.obj
 0001:000036f8       ??_C@_1M@CLPEOBGI@?$AAd?$AAa?$AA?9?$AAD?$AAK?$AA?$AA@ 00000001800046f8     libucrt:lcidtoname_downlevel.obj
 0001:00003708       ??_C@_1M@MCMADGCB@?$AAd?$AAe?$AA?9?$AAD?$AAE?$AA?$AA@ 0000000180004708     libucrt:lcidtoname_downlevel.obj
 0001:00003718       ??_C@_1M@OOCKEMAM@?$AAe?$AAl?$AA?9?$AAG?$AAR?$AA?$AA@ 0000000180004718     libucrt:lcidtoname_downlevel.obj
 0001:00003728       ??_C@_1M@DDNJFGID@?$AAf?$AAi?$AA?9?$AAF?$AAI?$AA?$AA@ 0000000180004728     libucrt:lcidtoname_downlevel.obj
 0001:00003738       ??_C@_1M@GLIPPMAC@?$AAf?$AAr?$AA?9?$AAF?$AAR?$AA?$AA@ 0000000180004738     libucrt:lcidtoname_downlevel.obj
 0001:00003748       ??_C@_1M@GFMCHPE@?$AAh?$AAe?$AA?9?$AAI?$AAL?$AA?$AA@ 0000000180004748     libucrt:lcidtoname_downlevel.obj
 0001:00003758       ??_C@_1M@MHLPGNKM@?$AAh?$AAu?$AA?9?$AAH?$AAU?$AA?$AA@ 0000000180004758     libucrt:lcidtoname_downlevel.obj
 0001:00003768       ??_C@_1M@LPDDNNPN@?$AAi?$AAs?$AA?9?$AAI?$AAS?$AA?$AA@ 0000000180004768     libucrt:lcidtoname_downlevel.obj
 0001:00003778       ??_C@_1M@MADIPODN@?$AAi?$AAt?$AA?9?$AAI?$AAT?$AA?$AA@ 0000000180004778     libucrt:lcidtoname_downlevel.obj
 0001:00003788       ??_C@_1M@IHBJJGG@?$AAn?$AAl?$AA?9?$AAN?$AAL?$AA?$AA@ 0000000180004788     libucrt:lcidtoname_downlevel.obj
 0001:00003798       ??_C@_1M@EANAGDL@?$AAn?$AAb?$AA?9?$AAN?$AAO?$AA?$AA@ 0000000180004798     libucrt:lcidtoname_downlevel.obj
 0001:000037a8       ??_C@_1M@NEIEMEGP@?$AAp?$AAl?$AA?9?$AAP?$AAL?$AA?$AA@ 00000001800047a8     libucrt:lcidtoname_downlevel.obj
 0001:000037b8       ??_C@_1M@BOCFIGEP@?$AAp?$AAt?$AA?9?$AAB?$AAR?$AA?$AA@ 00000001800047b8     libucrt:lcidtoname_downlevel.obj
 0001:000037c8       ??_C@_1M@IMPFOPBG@?$AAr?$AAo?$AA?9?$AAR?$AAO?$AA?$AA@ 00000001800047c8     libucrt:lcidtoname_downlevel.obj
 0001:000037d8       ??_C@_1M@IDNNEJMM@?$AAr?$AAu?$AA?9?$AAR?$AAU?$AA?$AA@ 00000001800047d8     libucrt:lcidtoname_downlevel.obj
 0001:000037e8       ??_C@_1M@LILEEOGM@?$AAh?$AAr?$AA?9?$AAH?$AAR?$AA?$AA@ 00000001800047e8     libucrt:lcidtoname_downlevel.obj
 0001:000037f8       ??_C@_1M@FKIFEHPB@?$AAs?$AAk?$AA?9?$AAS?$AAK?$AA?$AA@ 00000001800047f8     libucrt:lcidtoname_downlevel.obj
 0001:00003808       ??_C@_1M@LJMAMNPJ@?$AAs?$AAq?$AA?9?$AAA?$AAL?$AA?$AA@ 0000000180004808     libucrt:lcidtoname_downlevel.obj
 0001:00003818       ??_C@_1M@GIAKDKJK@?$AAs?$AAv?$AA?9?$AAS?$AAE?$AA?$AA@ 0000000180004818     libucrt:lcidtoname_downlevel.obj
 0001:00003828       ??_C@_1M@MKJKIKCL@?$AAt?$AAh?$AA?9?$AAT?$AAH?$AA?$AA@ 0000000180004828     libucrt:lcidtoname_downlevel.obj
 0001:00003838       ??_C@_1M@MFLCCMPB@?$AAt?$AAr?$AA?9?$AAT?$AAR?$AA?$AA@ 0000000180004838     libucrt:lcidtoname_downlevel.obj
 0001:00003848       ??_C@_1M@OIJHDKJN@?$AAu?$AAr?$AA?9?$AAP?$AAK?$AA?$AA@ 0000000180004848     libucrt:lcidtoname_downlevel.obj
 0001:00003858       ??_C@_1M@LHIPCIEK@?$AAi?$AAd?$AA?9?$AAI?$AAD?$AA?$AA@ 0000000180004858     libucrt:lcidtoname_downlevel.obj
 0001:00003868       ??_C@_1M@MFMOBGI@?$AAu?$AAk?$AA?9?$AAU?$AAA?$AA?$AA@ 0000000180004868     libucrt:lcidtoname_downlevel.obj
 0001:00003878       ??_C@_1M@OBGLJIPL@?$AAb?$AAe?$AA?9?$AAB?$AAY?$AA?$AA@ 0000000180004878     libucrt:lcidtoname_downlevel.obj
 0001:00003888       ??_C@_1M@BCFAJEAD@?$AAs?$AAl?$AA?9?$AAS?$AAI?$AA?$AA@ 0000000180004888     libucrt:lcidtoname_downlevel.obj
 0001:00003898       ??_C@_1M@FKFFEDDN@?$AAe?$AAt?$AA?9?$AAE?$AAE?$AA?$AA@ 0000000180004898     libucrt:lcidtoname_downlevel.obj
 0001:000038a8       ??_C@_1M@KGKKAACI@?$AAl?$AAv?$AA?9?$AAL?$AAV?$AA?$AA@ 00000001800048a8     libucrt:lcidtoname_downlevel.obj
 0001:000038b8       ??_C@_1M@IFGBIJO@?$AAl?$AAt?$AA?9?$AAL?$AAT?$AA?$AA@ 00000001800048b8     libucrt:lcidtoname_downlevel.obj
 0001:000038c8       ??_C@_1M@FGEAHEDM@?$AAf?$AAa?$AA?9?$AAI?$AAR?$AA?$AA@ 00000001800048c8     libucrt:lcidtoname_downlevel.obj
 0001:000038d8       ??_C@_1M@KBMAIBFN@?$AAv?$AAi?$AA?9?$AAV?$AAN?$AA?$AA@ 00000001800048d8     libucrt:lcidtoname_downlevel.obj
 0001:000038e8       ??_C@_1M@GPCBKDJK@?$AAh?$AAy?$AA?9?$AAA?$AAM?$AA?$AA@ 00000001800048e8     libucrt:lcidtoname_downlevel.obj
 0001:000038f8       ??_C@_1BG@BECMDDJB@?$AAa?$AAz?$AA?9?$AAA?$AAZ?$AA?9?$AAL?$AAa?$AAt?$AAn?$AA?$AA@ 00000001800048f8     libucrt:lcidtoname_downlevel.obj
 0001:00003910       ??_C@_1M@MAOFCAEA@?$AAe?$AAu?$AA?9?$AAE?$AAS?$AA?$AA@ 0000000180004910     libucrt:lcidtoname_downlevel.obj
 0001:00003920       ??_C@_1M@IGHABKPI@?$AAm?$AAk?$AA?9?$AAM?$AAK?$AA?$AA@ 0000000180004920     libucrt:lcidtoname_downlevel.obj
 0001:00003930       ??_C@_1M@IAIGNEJG@?$AAt?$AAn?$AA?9?$AAZ?$AAA?$AA?$AA@ 0000000180004930     libucrt:lcidtoname_downlevel.obj
 0001:00003940       ??_C@_1M@IIJCOJFA@?$AAx?$AAh?$AA?9?$AAZ?$AAA?$AA?$AA@ 0000000180004940     libucrt:lcidtoname_downlevel.obj
 0001:00003950       ??_C@_1M@LGPJHNJH@?$AAz?$AAu?$AA?9?$AAZ?$AAA?$AA?$AA@ 0000000180004950     libucrt:lcidtoname_downlevel.obj
 0001:00003960       ??_C@_1M@HOKAOIO@?$AAa?$AAf?$AA?9?$AAZ?$AAA?$AA?$AA@ 0000000180004960     libucrt:lcidtoname_downlevel.obj
 0001:00003970       ??_C@_1M@DPCLHLIE@?$AAk?$AAa?$AA?9?$AAG?$AAE?$AA?$AA@ 0000000180004970     libucrt:lcidtoname_downlevel.obj
 0001:00003980       ??_C@_1M@BLKMHJBI@?$AAf?$AAo?$AA?9?$AAF?$AAO?$AA?$AA@ 0000000180004980     libucrt:lcidtoname_downlevel.obj
 0001:00003990       ??_C@_1M@LGGJAPPB@?$AAh?$AAi?$AA?9?$AAI?$AAN?$AA?$AA@ 0000000180004990     libucrt:lcidtoname_downlevel.obj
 0001:000039a0       ??_C@_1M@FIKPIHFE@?$AAm?$AAt?$AA?9?$AAM?$AAT?$AA?$AA@ 00000001800049a0     libucrt:lcidtoname_downlevel.obj
 0001:000039b0       ??_C@_1M@HEGGPBFA@?$AAs?$AAe?$AA?9?$AAN?$AAO?$AA?$AA@ 00000001800049b0     libucrt:lcidtoname_downlevel.obj
 0001:000039c0       ??_C@_1M@EIBJEEPA@?$AAm?$AAs?$AA?9?$AAM?$AAY?$AA?$AA@ 00000001800049c0     libucrt:lcidtoname_downlevel.obj
 0001:000039d0       ??_C@_1M@FHLBGMPP@?$AAk?$AAk?$AA?9?$AAK?$AAZ?$AA?$AA@ 00000001800049d0     libucrt:lcidtoname_downlevel.obj
 0001:000039e0       ??_C@_1M@NGJJLCGI@?$AAk?$AAy?$AA?9?$AAK?$AAG?$AA?$AA@ 00000001800049e0     libucrt:lcidtoname_downlevel.obj
 0001:000039f0       ??_C@_1M@GIENNBFC@?$AAs?$AAw?$AA?9?$AAK?$AAE?$AA?$AA@ 00000001800049f0     libucrt:lcidtoname_downlevel.obj
 0001:00003a00       ??_C@_1BG@NDGMJIMJ@?$AAu?$AAz?$AA?9?$AAU?$AAZ?$AA?9?$AAL?$AAa?$AAt?$AAn?$AA?$AA@ 0000000180004a00     libucrt:lcidtoname_downlevel.obj
 0001:00003a18       ??_C@_1M@IDCCIHBC@?$AAt?$AAt?$AA?9?$AAR?$AAU?$AA?$AA@ 0000000180004a18     libucrt:lcidtoname_downlevel.obj
 0001:00003a28       ??_C@_1M@LOICPMOJ@?$AAb?$AAn?$AA?9?$AAI?$AAN?$AA?$AA@ 0000000180004a28     libucrt:lcidtoname_downlevel.obj
 0001:00003a38       ??_C@_1M@KPKKNEAH@?$AAp?$AAa?$AA?9?$AAI?$AAN?$AA?$AA@ 0000000180004a38     libucrt:lcidtoname_downlevel.obj
 0001:00003a48       ??_C@_1M@PJGPPBOG@?$AAg?$AAu?$AA?9?$AAI?$AAN?$AA?$AA@ 0000000180004a48     libucrt:lcidtoname_downlevel.obj
 0001:00003a58       ??_C@_1M@KMKMOPHI@?$AAt?$AAa?$AA?9?$AAI?$AAN?$AA?$AA@ 0000000180004a58     libucrt:lcidtoname_downlevel.obj
 0001:00003a68       ??_C@_1M@KFEHEPAC@?$AAt?$AAe?$AA?9?$AAI?$AAN?$AA?$AA@ 0000000180004a68     libucrt:lcidtoname_downlevel.obj
 0001:00003a78       ??_C@_1M@CDCLMGHI@?$AAk?$AAn?$AA?9?$AAI?$AAN?$AA?$AA@ 0000000180004a78     libucrt:lcidtoname_downlevel.obj
 0001:00003a88       ??_C@_1M@MIODLDKF@?$AAm?$AAl?$AA?9?$AAI?$AAN?$AA?$AA@ 0000000180004a88     libucrt:lcidtoname_downlevel.obj
 0001:00003a98       ??_C@_1M@PBIEACPO@?$AAm?$AAr?$AA?9?$AAI?$AAN?$AA?$AA@ 0000000180004a98     libucrt:lcidtoname_downlevel.obj
 0001:00003aa8       ??_C@_1M@NIDEAGPH@?$AAs?$AAa?$AA?9?$AAI?$AAN?$AA?$AA@ 0000000180004aa8     libucrt:lcidtoname_downlevel.obj
 0001:00003ab8       ??_C@_1M@FHIHCBIO@?$AAm?$AAn?$AA?9?$AAM?$AAN?$AA?$AA@ 0000000180004ab8     libucrt:lcidtoname_downlevel.obj
 0001:00003ac8       ??_C@_1M@JAIJPENP@?$AAc?$AAy?$AA?9?$AAG?$AAB?$AA?$AA@ 0000000180004ac8     libucrt:lcidtoname_downlevel.obj
 0001:00003ad8       ??_C@_1M@PHGFBEPN@?$AAg?$AAl?$AA?9?$AAE?$AAS?$AA?$AA@ 0000000180004ad8     libucrt:lcidtoname_downlevel.obj
 0001:00003ae8       ??_C@_1O@KPIPDNCP@?$AAk?$AAo?$AAk?$AA?9?$AAI?$AAN?$AA?$AA@ 0000000180004ae8     libucrt:lcidtoname_downlevel.obj
 0001:00003af8       ??_C@_1O@KNHJLDJA@?$AAs?$AAy?$AAr?$AA?9?$AAS?$AAY?$AA?$AA@ 0000000180004af8     libucrt:lcidtoname_downlevel.obj
 0001:00003b08       ??_C@_1O@MKEKBLAH@?$AAd?$AAi?$AAv?$AA?9?$AAM?$AAV?$AA?$AA@ 0000000180004b08     libucrt:lcidtoname_downlevel.obj
 0001:00003b18       ??_C@_1O@OHDCKDDF@?$AAq?$AAu?$AAz?$AA?9?$AAB?$AAO?$AA?$AA@ 0000000180004b18     libucrt:lcidtoname_downlevel.obj
 0001:00003b28       ??_C@_1M@LEPJNLFD@?$AAn?$AAs?$AA?9?$AAZ?$AAA?$AA?$AA@ 0000000180004b28     libucrt:lcidtoname_downlevel.obj
 0001:00003b38       ??_C@_1M@OMLEIIJB@?$AAm?$AAi?$AA?9?$AAN?$AAZ?$AA?$AA@ 0000000180004b38     libucrt:lcidtoname_downlevel.obj
 0001:00003b48       ??_C@_1M@PMPEAILG@?$AAa?$AAr?$AA?9?$AAI?$AAQ?$AA?$AA@ 0000000180004b48     libucrt:lcidtoname_downlevel.obj
 0001:00003b58       ??_C@_1M@CNKPNOEE@?$AAd?$AAe?$AA?9?$AAC?$AAH?$AA?$AA@ 0000000180004b58     libucrt:lcidtoname_downlevel.obj
 0001:00003b68       ??_C@_1M@LKMGMLKO@?$AAe?$AAn?$AA?9?$AAG?$AAB?$AA?$AA@ 0000000180004b68     libucrt:lcidtoname_downlevel.obj
 0001:00003b78       ??_C@_1M@PGKJFFGL@?$AAe?$AAs?$AA?9?$AAM?$AAX?$AA?$AA@ 0000000180004b78     libucrt:lcidtoname_downlevel.obj
 0001:00003b88       ??_C@_1M@DNNANBDC@?$AAf?$AAr?$AA?9?$AAB?$AAE?$AA?$AA@ 0000000180004b88     libucrt:lcidtoname_downlevel.obj
 0001:00003b98       ??_C@_1M@HLGMDFHM@?$AAi?$AAt?$AA?9?$AAC?$AAH?$AA?$AA@ 0000000180004b98     libucrt:lcidtoname_downlevel.obj
 0001:00003ba8       ??_C@_1M@CLLBGJH@?$AAn?$AAl?$AA?9?$AAB?$AAE?$AA?$AA@ 0000000180004ba8     libucrt:lcidtoname_downlevel.obj
 0001:00003bb8       ??_C@_1M@BODBOGLF@?$AAn?$AAn?$AA?9?$AAN?$AAO?$AA?$AA@ 0000000180004bb8     libucrt:lcidtoname_downlevel.obj
 0001:00003bc8       ??_C@_1M@HFFAHKAD@?$AAp?$AAt?$AA?9?$AAP?$AAT?$AA?$AA@ 0000000180004bc8     libucrt:lcidtoname_downlevel.obj
 0001:00003bd8       ??_C@_1BG@LNOAKHIE@?$AAs?$AAr?$AA?9?$AAS?$AAP?$AA?9?$AAL?$AAa?$AAt?$AAn?$AA?$AA@ 0000000180004bd8     libucrt:lcidtoname_downlevel.obj
 0001:00003bf0       ??_C@_1M@HBMHBGAK@?$AAs?$AAv?$AA?9?$AAF?$AAI?$AA?$AA@ 0000000180004bf0     libucrt:lcidtoname_downlevel.obj
 0001:00003c00       ??_C@_1BG@DGCJGJBE@?$AAa?$AAz?$AA?9?$AAA?$AAZ?$AA?9?$AAC?$AAy?$AAr?$AAl?$AA?$AA@ 0000000180004c00     libucrt:lcidtoname_downlevel.obj
 0001:00003c18       ??_C@_1M@KEJDAAHB@?$AAs?$AAe?$AA?9?$AAS?$AAE?$AA?$AA@ 0000000180004c18     libucrt:lcidtoname_downlevel.obj
 0001:00003c28       ??_C@_1M@HEIBJJAD@?$AAm?$AAs?$AA?9?$AAB?$AAN?$AA?$AA@ 0000000180004c28     libucrt:lcidtoname_downlevel.obj
 0001:00003c38       ??_C@_1BG@PBGJMCEM@?$AAu?$AAz?$AA?9?$AAU?$AAZ?$AA?9?$AAC?$AAy?$AAr?$AAl?$AA?$AA@ 0000000180004c38     libucrt:lcidtoname_downlevel.obj
 0001:00003c50       ??_C@_1O@LAOBCMDF@?$AAq?$AAu?$AAz?$AA?9?$AAE?$AAC?$AA?$AA@ 0000000180004c50     libucrt:lcidtoname_downlevel.obj
 0001:00003c60       ??_C@_1M@POEEMAIO@?$AAa?$AAr?$AA?9?$AAE?$AAG?$AA?$AA@ 0000000180004c60     libucrt:lcidtoname_downlevel.obj
 0001:00003c70       ??_C@_1M@EFAKDEDL@?$AAz?$AAh?$AA?9?$AAH?$AAK?$AA?$AA@ 0000000180004c70     libucrt:lcidtoname_downlevel.obj
 0001:00003c80       ??_C@_1M@HKKIJHGI@?$AAd?$AAe?$AA?9?$AAA?$AAT?$AA?$AA@ 0000000180004c80     libucrt:lcidtoname_downlevel.obj
 0001:00003c90       ??_C@_1M@KBFBEHJF@?$AAe?$AAn?$AA?9?$AAA?$AAU?$AA?$AA@ 0000000180004c90     libucrt:lcidtoname_downlevel.obj
 0001:00003ca0       ??_C@_1M@MNPLFAAH@?$AAe?$AAs?$AA?9?$AAE?$AAS?$AA?$AA@ 0000000180004ca0     libucrt:lcidtoname_downlevel.obj
 0001:00003cb0       ??_C@_1M@HJOOJFMA@?$AAf?$AAr?$AA?9?$AAC?$AAA?$AA?$AA@ 0000000180004cb0     libucrt:lcidtoname_downlevel.obj
 0001:00003cc0       ??_C@_1BG@JPOFPNAB@?$AAs?$AAr?$AA?9?$AAS?$AAP?$AA?9?$AAC?$AAy?$AAr?$AAl?$AA?$AA@ 0000000180004cc0     libucrt:lcidtoname_downlevel.obj
 0001:00003cd8       ??_C@_1M@LNFOCMOB@?$AAs?$AAe?$AA?9?$AAF?$AAI?$AA?$AA@ 0000000180004cd8     libucrt:lcidtoname_downlevel.obj
 0001:00003ce8       ??_C@_1O@MGJBOAMB@?$AAq?$AAu?$AAz?$AA?9?$AAP?$AAE?$AA?$AA@ 0000000180004ce8     libucrt:lcidtoname_downlevel.obj
 0001:00003cf8       ??_C@_1M@GJINLBOK@?$AAa?$AAr?$AA?9?$AAL?$AAY?$AA?$AA@ 0000000180004cf8     libucrt:lcidtoname_downlevel.obj
 0001:00003d08       ??_C@_1M@GGMNHJNL@?$AAz?$AAh?$AA?9?$AAS?$AAG?$AA?$AA@ 0000000180004d08     libucrt:lcidtoname_downlevel.obj
 0001:00003d18       ??_C@_1M@HOIKODND@?$AAd?$AAe?$AA?9?$AAL?$AAU?$AA?$AA@ 0000000180004d18     libucrt:lcidtoname_downlevel.obj
 0001:00003d28       ??_C@_1M@DDOCCGFG@?$AAe?$AAn?$AA?9?$AAC?$AAA?$AA?$AA@ 0000000180004d28     libucrt:lcidtoname_downlevel.obj
 0001:00003d38       ??_C@_1M@BNOEMJLF@?$AAe?$AAs?$AA?9?$AAG?$AAT?$AA?$AA@ 0000000180004d38     libucrt:lcidtoname_downlevel.obj
 0001:00003d48       ??_C@_1M@EOGNKEK@?$AAf?$AAr?$AA?9?$AAC?$AAH?$AA?$AA@ 0000000180004d48     libucrt:lcidtoname_downlevel.obj
 0001:00003d58       ??_C@_1M@FLIDJFHL@?$AAh?$AAr?$AA?9?$AAB?$AAA?$AA?$AA@ 0000000180004d58     libucrt:lcidtoname_downlevel.obj
 0001:00003d68       ??_C@_1O@FMCELNAJ@?$AAs?$AAm?$AAj?$AA?9?$AAN?$AAO?$AA?$AA@ 0000000180004d68     libucrt:lcidtoname_downlevel.obj
 0001:00003d78       ??_C@_1M@JHGLJMGJ@?$AAa?$AAr?$AA?9?$AAD?$AAZ?$AA?$AA@ 0000000180004d78     libucrt:lcidtoname_downlevel.obj
 0001:00003d88       ??_C@_1M@JKKFDCNP@?$AAz?$AAh?$AA?9?$AAM?$AAO?$AA?$AA@ 0000000180004d88     libucrt:lcidtoname_downlevel.obj
 0001:00003d98       ??_C@_1M@GEEFALPE@?$AAd?$AAe?$AA?9?$AAL?$AAI?$AA?$AA@ 0000000180004d98     libucrt:lcidtoname_downlevel.obj
 0001:00003da8       ??_C@_1M@IGEOFBG@?$AAe?$AAn?$AA?9?$AAN?$AAZ?$AA?$AA@ 0000000180004da8     libucrt:lcidtoname_downlevel.obj
 0001:00003db8       ??_C@_1M@KDBONEHP@?$AAe?$AAs?$AA?9?$AAC?$AAR?$AA?$AA@ 0000000180004db8     libucrt:lcidtoname_downlevel.obj
 0001:00003dc8       ??_C@_1M@FHMDOHNN@?$AAf?$AAr?$AA?9?$AAL?$AAU?$AA?$AA@ 0000000180004dc8     libucrt:lcidtoname_downlevel.obj
 0001:00003dd8       ??_C@_1BG@NFKKMAFG@?$AAb?$AAs?$AA?9?$AAB?$AAA?$AA?9?$AAL?$AAa?$AAt?$AAn?$AA?$AA@ 0000000180004dd8     libucrt:lcidtoname_downlevel.obj
 0001:00003df0       ??_C@_1O@IMNBEMCI@?$AAs?$AAm?$AAj?$AA?9?$AAS?$AAE?$AA?$AA@ 0000000180004df0     libucrt:lcidtoname_downlevel.obj
 0001:00003e00       ??_C@_1M@DHHMBNDP@?$AAa?$AAr?$AA?9?$AAM?$AAA?$AA?$AA@ 0000000180004e00     libucrt:lcidtoname_downlevel.obj
 0001:00003e10       ??_C@_1M@BNBLJCGH@?$AAe?$AAn?$AA?9?$AAI?$AAE?$AA?$AA@ 0000000180004e10     libucrt:lcidtoname_downlevel.obj
 0001:00003e20       ??_C@_1M@GEPAFMDL@?$AAe?$AAs?$AA?9?$AAP?$AAA?$AA?$AA@ 0000000180004e20     libucrt:lcidtoname_downlevel.obj
 0001:00003e30       ??_C@_1M@OJONDMDL@?$AAf?$AAr?$AA?9?$AAM?$AAC?$AA?$AA@ 0000000180004e30     libucrt:lcidtoname_downlevel.obj
 0001:00003e40       ??_C@_1BG@OBCNFJB@?$AAs?$AAr?$AA?9?$AAB?$AAA?$AA?9?$AAL?$AAa?$AAt?$AAn?$AA?$AA@ 0000000180004e40     libucrt:lcidtoname_downlevel.obj
 0001:00003e58       ??_C@_1O@KEMEEGPO@?$AAs?$AAm?$AAa?$AA?9?$AAN?$AAO?$AA?$AA@ 0000000180004e58     libucrt:lcidtoname_downlevel.obj
 0001:00003e68       ??_C@_1M@ELMGFODK@?$AAa?$AAr?$AA?9?$AAT?$AAN?$AA?$AA@ 0000000180004e68     libucrt:lcidtoname_downlevel.obj
 0001:00003e78       ??_C@_1M@BHDLHFAF@?$AAe?$AAn?$AA?9?$AAZ?$AAA?$AA?$AA@ 0000000180004e78     libucrt:lcidtoname_downlevel.obj
 0001:00003e88       ??_C@_1M@BMGIGLIF@?$AAe?$AAs?$AA?9?$AAD?$AAO?$AA?$AA@ 0000000180004e88     libucrt:lcidtoname_downlevel.obj
 0001:00003e98       ??_C@_1BG@CMBHIPBE@?$AAs?$AAr?$AA?9?$AAB?$AAA?$AA?9?$AAC?$AAy?$AAr?$AAl?$AA?$AA@ 0000000180004e98     libucrt:lcidtoname_downlevel.obj
 0001:00003eb0       ??_C@_1O@HEDBLHNP@?$AAs?$AAm?$AAa?$AA?9?$AAS?$AAE?$AA?$AA@ 0000000180004eb0     libucrt:lcidtoname_downlevel.obj
 0001:00003ec0       ??_C@_1M@DAGCADIM@?$AAa?$AAr?$AA?9?$AAO?$AAM?$AA?$AA@ 0000000180004ec0     libucrt:lcidtoname_downlevel.obj
 0001:00003ed0       ??_C@_1M@FODLMICG@?$AAe?$AAn?$AA?9?$AAJ?$AAM?$AA?$AA@ 0000000180004ed0     libucrt:lcidtoname_downlevel.obj
 0001:00003ee0       ??_C@_1M@DNMLCIHB@?$AAe?$AAs?$AA?9?$AAV?$AAE?$AA?$AA@ 0000000180004ee0     libucrt:lcidtoname_downlevel.obj
 0001:00003ef0       ??_C@_1O@EOKHMKJK@?$AAs?$AAm?$AAs?$AA?9?$AAF?$AAI?$AA?$AA@ 0000000180004ef0     libucrt:lcidtoname_downlevel.obj
 0001:00003f00       ??_C@_1M@CAFJMKOF@?$AAa?$AAr?$AA?9?$AAY?$AAE?$AA?$AA@ 0000000180004f00     libucrt:lcidtoname_downlevel.obj
 0001:00003f10       ??_C@_1M@CBFHIJLI@?$AAe?$AAn?$AA?9?$AAC?$AAB?$AA?$AA@ 0000000180004f10     libucrt:lcidtoname_downlevel.obj
 0001:00003f20       ??_C@_1M@BGNFLDN@?$AAe?$AAs?$AA?9?$AAC?$AAO?$AA?$AA@ 0000000180004f20     libucrt:lcidtoname_downlevel.obj
 0001:00003f30       ??_C@_1O@JMPHMAMC@?$AAs?$AAm?$AAn?$AA?9?$AAF?$AAI?$AA?$AA@ 0000000180004f30     libucrt:lcidtoname_downlevel.obj
 0001:00003f40       ??_C@_1M@JLANABKE@?$AAa?$AAr?$AA?9?$AAS?$AAY?$AA?$AA@ 0000000180004f40     libucrt:lcidtoname_downlevel.obj
 0001:00003f50       ??_C@_1M@HPKGCFGN@?$AAe?$AAn?$AA?9?$AAB?$AAZ?$AA?$AA@ 0000000180004f50     libucrt:lcidtoname_downlevel.obj
 0001:00003f60       ??_C@_1M@OLJCMLGM@?$AAe?$AAs?$AA?9?$AAP?$AAE?$AA?$AA@ 0000000180004f60     libucrt:lcidtoname_downlevel.obj
 0001:00003f70       ??_C@_1M@MKKGFKLE@?$AAa?$AAr?$AA?9?$AAJ?$AAO?$AA?$AA@ 0000000180004f70     libucrt:lcidtoname_downlevel.obj
 0001:00003f80       ??_C@_1M@EKPGLDNI@?$AAe?$AAn?$AA?9?$AAT?$AAT?$AA?$AA@ 0000000180004f80     libucrt:lcidtoname_downlevel.obj
 0001:00003f90       ??_C@_1M@OONGHFHE@?$AAe?$AAs?$AA?9?$AAA?$AAR?$AA?$AA@ 0000000180004f90     libucrt:lcidtoname_downlevel.obj
 0001:00003fa0       ??_C@_1M@OOJFGBHE@?$AAa?$AAr?$AA?9?$AAL?$AAB?$AA?$AA@ 0000000180004fa0     libucrt:lcidtoname_downlevel.obj
 0001:00003fb0       ??_C@_1M@GCEJHNEG@?$AAe?$AAn?$AA?9?$AAZ?$AAW?$AA?$AA@ 0000000180004fb0     libucrt:lcidtoname_downlevel.obj
 0001:00003fc0       ??_C@_1M@JNOCAHJI@?$AAe?$AAs?$AA?9?$AAE?$AAC?$AA?$AA@ 0000000180004fc0     libucrt:lcidtoname_downlevel.obj
 0001:00003fd0       ??_C@_1M@JEFHPGGB@?$AAa?$AAr?$AA?9?$AAK?$AAW?$AA?$AA@ 0000000180004fd0     libucrt:lcidtoname_downlevel.obj
 0001:00003fe0       ??_C@_1M@MLKIBJOJ@?$AAe?$AAn?$AA?9?$AAP?$AAH?$AA?$AA@ 0000000180004fe0     libucrt:lcidtoname_downlevel.obj
 0001:00003ff0       ??_C@_1M@BDNIPEND@?$AAe?$AAs?$AA?9?$AAC?$AAL?$AA?$AA@ 0000000180004ff0     libucrt:lcidtoname_downlevel.obj
 0001:00004000       ??_C@_1M@MPNMEKBD@?$AAa?$AAr?$AA?9?$AAA?$AAE?$AA?$AA@ 0000000180005000     libucrt:lcidtoname_downlevel.obj
 0001:00004010       ??_C@_1M@KBJALCPI@?$AAe?$AAs?$AA?9?$AAU?$AAY?$AA?$AA@ 0000000180005010     libucrt:lcidtoname_downlevel.obj
 0001:00004020       ??_C@_1M@LLCCOAGA@?$AAa?$AAr?$AA?9?$AAB?$AAH?$AA?$AA@ 0000000180005020     libucrt:lcidtoname_downlevel.obj
 0001:00004030       ??_C@_1M@PBFNCDEL@?$AAe?$AAs?$AA?9?$AAP?$AAY?$AA?$AA@ 0000000180005030     libucrt:lcidtoname_downlevel.obj
 0001:00004040       ??_C@_1M@EDGINPNP@?$AAa?$AAr?$AA?9?$AAQ?$AAA?$AA?$AA@ 0000000180005040     libucrt:lcidtoname_downlevel.obj
 0001:00004050       ??_C@_1M@MKDBIIJI@?$AAe?$AAs?$AA?9?$AAB?$AAO?$AA?$AA@ 0000000180005050     libucrt:lcidtoname_downlevel.obj
 0001:00004060       ??_C@_1M@CPKKEBLD@?$AAe?$AAs?$AA?9?$AAS?$AAV?$AA?$AA@ 0000000180005060     libucrt:lcidtoname_downlevel.obj
 0001:00004070       ??_C@_1M@NDBGMMJL@?$AAe?$AAs?$AA?9?$AAH?$AAN?$AA?$AA@ 0000000180005070     libucrt:lcidtoname_downlevel.obj
 0001:00004080       ??_C@_1M@JIJIBHDP@?$AAe?$AAs?$AA?9?$AAN?$AAI?$AA?$AA@ 0000000180005080     libucrt:lcidtoname_downlevel.obj
 0001:00004090       ??_C@_1M@CGFMKEEK@?$AAe?$AAs?$AA?9?$AAP?$AAR?$AA?$AA@ 0000000180005090     libucrt:lcidtoname_downlevel.obj
 0001:000040a0       ??_C@_1O@ICJHKIIK@?$AAz?$AAh?$AA?9?$AAC?$AAH?$AAT?$AA?$AA@ 00000001800050a0     libucrt:lcidtoname_downlevel.obj
 0001:000040b0       ??_C@_15CLNEJCE@?$AAs?$AAr?$AA?$AA@ 00000001800050b0     libucrt:lcidtoname_downlevel.obj
 0001:00004f00       ??_C@_1M@KAHEKEIG@?$AAa?$AAf?$AA?9?$AAz?$AAa?$AA?$AA@ 0000000180005f00     libucrt:lcidtoname_downlevel.obj
 0001:00004f10       ??_C@_1M@GIECOABL@?$AAa?$AAr?$AA?9?$AAa?$AAe?$AA?$AA@ 0000000180005f10     libucrt:lcidtoname_downlevel.obj
 0001:00004f20       ??_C@_1M@BMLMEKGI@?$AAa?$AAr?$AA?9?$AAb?$AAh?$AA?$AA@ 0000000180005f20     libucrt:lcidtoname_downlevel.obj
 0001:00004f30       ??_C@_1M@DAPFDGGB@?$AAa?$AAr?$AA?9?$AAd?$AAz?$AA?$AA@ 0000000180005f30     libucrt:lcidtoname_downlevel.obj
 0001:00004f40       ??_C@_1M@FJNKGKIG@?$AAa?$AAr?$AA?9?$AAe?$AAg?$AA?$AA@ 0000000180005f40     libucrt:lcidtoname_downlevel.obj
 0001:00004f50       ??_C@_1M@FLGKKCLO@?$AAa?$AAr?$AA?9?$AAi?$AAq?$AA?$AA@ 0000000180005f50     libucrt:lcidtoname_downlevel.obj
 0001:00004f60       ??_C@_1M@GNDIPALM@?$AAa?$AAr?$AA?9?$AAj?$AAo?$AA?$AA@ 0000000180005f60     libucrt:lcidtoname_downlevel.obj
 0001:00004f70       ??_C@_1M@DDMJFMGJ@?$AAa?$AAr?$AA?9?$AAk?$AAw?$AA?$AA@ 0000000180005f70     libucrt:lcidtoname_downlevel.obj
 0001:00004f80       ??_C@_1M@EJALMLHM@?$AAa?$AAr?$AA?9?$AAl?$AAb?$AA?$AA@ 0000000180005f80     libucrt:lcidtoname_downlevel.obj
 0001:00004f90       ??_C@_1M@MOBDBLOC@?$AAa?$AAr?$AA?9?$AAl?$AAy?$AA?$AA@ 0000000180005f90     libucrt:lcidtoname_downlevel.obj
 0001:00004fa0       ??_C@_1M@JAOCLHDH@?$AAa?$AAr?$AA?9?$AAm?$AAa?$AA?$AA@ 0000000180005fa0     libucrt:lcidtoname_downlevel.obj
 0001:00004fb0       ??_C@_1M@JHPMKJIE@?$AAa?$AAr?$AA?9?$AAo?$AAm?$AA?$AA@ 0000000180005fb0     libucrt:lcidtoname_downlevel.obj
 0001:00004fc0       ??_C@_1M@OEPGHFNH@?$AAa?$AAr?$AA?9?$AAq?$AAa?$AA?$AA@ 0000000180005fc0     libucrt:lcidtoname_downlevel.obj
 0001:00004fd0       ??_C@_1M@KJDONENM@?$AAa?$AAr?$AA?9?$AAs?$AAa?$AA?$AA@ 0000000180005fd0     libucrt:lcidtoname_downlevel.obj
 0001:00004fe0       ??_C@_1M@DMJDKLKM@?$AAa?$AAr?$AA?9?$AAs?$AAy?$AA?$AA@ 0000000180005fe0     libucrt:lcidtoname_downlevel.obj
 0001:00004ff0       ??_C@_1M@OMFIPEDC@?$AAa?$AAr?$AA?9?$AAt?$AAn?$AA?$AA@ 0000000180005ff0     libucrt:lcidtoname_downlevel.obj
 0001:00005000       ??_C@_1M@IHMHGAON@?$AAa?$AAr?$AA?9?$AAy?$AAe?$AA?$AA@ 0000000180006000     libucrt:lcidtoname_downlevel.obj
 0001:00005010       ??_C@_1BG@KDCPGJGB@?$AAa?$AAz?$AA?9?$AAa?$AAz?$AA?9?$AAc?$AAy?$AAr?$AAl?$AA?$AA@ 0000000180006010     libucrt:lcidtoname_downlevel.obj
 0001:00005028       ??_C@_1BG@IBCKDDOE@?$AAa?$AAz?$AA?9?$AAa?$AAz?$AA?9?$AAl?$AAa?$AAt?$AAn?$AA?$AA@ 0000000180006028     libucrt:lcidtoname_downlevel.obj
 0001:00005040       ??_C@_1M@EGPFDCPD@?$AAb?$AAe?$AA?9?$AAb?$AAy?$AA?$AA@ 0000000180006040     libucrt:lcidtoname_downlevel.obj
 0001:00005050       ??_C@_1M@PCMGMCGC@?$AAb?$AAg?$AA?9?$AAb?$AAg?$AA?$AA@ 0000000180006050     libucrt:lcidtoname_downlevel.obj
 0001:00005060       ??_C@_1M@BJBMFGOB@?$AAb?$AAn?$AA?9?$AAi?$AAn?$AA?$AA@ 0000000180006060     libucrt:lcidtoname_downlevel.obj
 0001:00005070       ??_C@_1BG@EAKMMACD@?$AAb?$AAs?$AA?9?$AAb?$AAa?$AA?9?$AAl?$AAa?$AAt?$AAn?$AA?$AA@ 0000000180006070     libucrt:lcidtoname_downlevel.obj
 0001:00005088       ??_C@_1M@KGADAODK@?$AAc?$AAa?$AA?9?$AAe?$AAs?$AA?$AA@ 0000000180006088     libucrt:lcidtoname_downlevel.obj
 0001:00005098       ??_C@_1M@COAJPDHI@?$AAc?$AAs?$AA?9?$AAc?$AAz?$AA?$AA@ 0000000180006098     libucrt:lcidtoname_downlevel.obj
 0001:000050a8       ??_C@_1M@DHBHFONH@?$AAc?$AAy?$AA?9?$AAg?$AAb?$AA?$AA@ 00000001800060a8     libucrt:lcidtoname_downlevel.obj
 0001:000050b8       ??_C@_1M@IMGKELGA@?$AAd?$AAa?$AA?9?$AAd?$AAk?$AA?$AA@ 00000001800060b8     libucrt:lcidtoname_downlevel.obj
 0001:000050c8       ??_C@_1M@NNDGDNGA@?$AAd?$AAe?$AA?9?$AAa?$AAt?$AA?$AA@ 00000001800060c8     libucrt:lcidtoname_downlevel.obj
 0001:000050d8       ??_C@_1M@IKDBHEEM@?$AAd?$AAe?$AA?9?$AAc?$AAh?$AA?$AA@ 00000001800060d8     libucrt:lcidtoname_downlevel.obj
 0001:000050e8       ??_C@_1M@GFFOJMCJ@?$AAd?$AAe?$AA?9?$AAd?$AAe?$AA?$AA@ 00000001800060e8     libucrt:lcidtoname_downlevel.obj
 0001:000050f8       ??_C@_1M@MDNLKBPM@?$AAd?$AAe?$AA?9?$AAl?$AAi?$AA?$AA@ 00000001800060f8     libucrt:lcidtoname_downlevel.obj
 0001:00005108       ??_C@_1M@NJBEEJNL@?$AAd?$AAe?$AA?9?$AAl?$AAu?$AA?$AA@ 0000000180006108     libucrt:lcidtoname_downlevel.obj
 0001:00005118       ??_C@_1O@GNNELBAP@?$AAd?$AAi?$AAv?$AA?9?$AAm?$AAv?$AA?$AA@ 0000000180006118     libucrt:lcidtoname_downlevel.obj
 0001:00005128       ??_C@_1M@EJLEOGAE@?$AAe?$AAl?$AA?9?$AAg?$AAr?$AA?$AA@ 0000000180006128     libucrt:lcidtoname_downlevel.obj
 0001:00005138       ??_C@_1M@GMPONJN@?$AAe?$AAn?$AA?9?$AAa?$AAu?$AA?$AA@ 0000000180006138     libucrt:lcidtoname_downlevel.obj
 0001:00005148       ??_C@_1M@NIDIIPGF@?$AAe?$AAn?$AA?9?$AAb?$AAz?$AA?$AA@ 0000000180006148     libucrt:lcidtoname_downlevel.obj
 0001:00005158       ??_C@_1M@JEHMIMFO@?$AAe?$AAn?$AA?9?$AAc?$AAa?$AA?$AA@ 0000000180006158     libucrt:lcidtoname_downlevel.obj
 0001:00005168       ??_C@_1M@IGMJCDLA@?$AAe?$AAn?$AA?9?$AAc?$AAb?$AA?$AA@ 0000000180006168     libucrt:lcidtoname_downlevel.obj
 0001:00005178       ??_C@_1M@BNFIGBKG@?$AAe?$AAn?$AA?9?$AAg?$AAb?$AA?$AA@ 0000000180006178     libucrt:lcidtoname_downlevel.obj
 0001:00005188       ??_C@_1M@LKIFDIGP@?$AAe?$AAn?$AA?9?$AAi?$AAe?$AA?$AA@ 0000000180006188     libucrt:lcidtoname_downlevel.obj
 0001:00005198       ??_C@_1M@PJKFGCCO@?$AAe?$AAn?$AA?9?$AAj?$AAm?$AA?$AA@ 0000000180006198     libucrt:lcidtoname_downlevel.obj
 0001:000051a8       ??_C@_1M@KPPKEPBO@?$AAe?$AAn?$AA?9?$AAn?$AAz?$AA?$AA@ 00000001800061a8     libucrt:lcidtoname_downlevel.obj
 0001:000051b8       ??_C@_1M@GMDGLDOB@?$AAe?$AAn?$AA?9?$AAp?$AAh?$AA?$AA@ 00000001800061b8     libucrt:lcidtoname_downlevel.obj
 0001:000051c8       ??_C@_1M@ONGIBJNA@?$AAe?$AAn?$AA?9?$AAt?$AAt?$AA?$AA@ 00000001800061c8     libucrt:lcidtoname_downlevel.obj
 0001:000051d8       ??_C@_1M@LLODPCMM@?$AAe?$AAn?$AA?9?$AAu?$AAs?$AA?$AA@ 00000001800061d8     libucrt:lcidtoname_downlevel.obj
 0001:000051e8       ??_C@_1M@LAKFNPAN@?$AAe?$AAn?$AA?9?$AAz?$AAa?$AA?$AA@ 00000001800061e8     libucrt:lcidtoname_downlevel.obj
 0001:000051f8       ??_C@_1M@MFNHNHEO@?$AAe?$AAn?$AA?9?$AAz?$AAw?$AA?$AA@ 00000001800061f8     libucrt:lcidtoname_downlevel.obj
 0001:00005208       ??_C@_1M@EJEINPHM@?$AAe?$AAs?$AA?9?$AAa?$AAr?$AA?$AA@ 0000000180006208     libucrt:lcidtoname_downlevel.obj
 0001:00005218       ??_C@_1M@GNKPCCJA@?$AAe?$AAs?$AA?9?$AAb?$AAo?$AA?$AA@ 0000000180006218     libucrt:lcidtoname_downlevel.obj
 0001:00005228       ??_C@_1M@LEEGFONL@?$AAe?$AAs?$AA?9?$AAc?$AAl?$AA?$AA@ 0000000180006228     libucrt:lcidtoname_downlevel.obj
 0001:00005238       ??_C@_1M@KGPDPBDF@?$AAe?$AAs?$AA?9?$AAc?$AAo?$AA?$AA@ 0000000180006238     libucrt:lcidtoname_downlevel.obj
 0001:00005248       ??_C@_1M@EIAHOHH@?$AAe?$AAs?$AA?9?$AAc?$AAr?$AA?$AA@ 0000000180006248     libucrt:lcidtoname_downlevel.obj
 0001:00005258       ??_C@_1M@LLPGMBIN@?$AAe?$AAs?$AA?9?$AAd?$AAo?$AA?$AA@ 0000000180006258     libucrt:lcidtoname_downlevel.obj
 0001:00005268       ??_C@_1M@DKHMKNJA@?$AAe?$AAs?$AA?9?$AAe?$AAc?$AA?$AA@ 0000000180006268     libucrt:lcidtoname_downlevel.obj
 0001:00005278       ??_C@_1M@GKGFPKAP@?$AAe?$AAs?$AA?9?$AAe?$AAs?$AA?$AA@ 0000000180006278     libucrt:lcidtoname_downlevel.obj
 0001:00005288       ??_C@_1M@LKHKGDLN@?$AAe?$AAs?$AA?9?$AAg?$AAt?$AA?$AA@ 0000000180006288     libucrt:lcidtoname_downlevel.obj
 0001:00005298       ??_C@_1M@HEIIGGJD@?$AAe?$AAs?$AA?9?$AAh?$AAn?$AA?$AA@ 0000000180006298     libucrt:lcidtoname_downlevel.obj
 0001:000052a8       ??_C@_1M@FBDHPPGD@?$AAe?$AAs?$AA?9?$AAm?$AAx?$AA?$AA@ 00000001800062a8     libucrt:lcidtoname_downlevel.obj
 0001:000052b8       ??_C@_1M@DPAGLNDH@?$AAe?$AAs?$AA?9?$AAn?$AAi?$AA?$AA@ 00000001800062b8     libucrt:lcidtoname_downlevel.obj
 0001:000052c8       ??_C@_1M@MDGOPGDD@?$AAe?$AAs?$AA?9?$AAp?$AAa?$AA?$AA@ 00000001800062c8     libucrt:lcidtoname_downlevel.obj
 0001:000052d8       ??_C@_1M@EMAMGBGE@?$AAe?$AAs?$AA?9?$AAp?$AAe?$AA?$AA@ 00000001800062d8     libucrt:lcidtoname_downlevel.obj
 0001:000052e8       ??_C@_1M@IBMCAOEC@?$AAe?$AAs?$AA?9?$AAp?$AAr?$AA?$AA@ 00000001800062e8     libucrt:lcidtoname_downlevel.obj
 0001:000052f8       ??_C@_1M@FGMDIJED@?$AAe?$AAs?$AA?9?$AAp?$AAy?$AA?$AA@ 00000001800062f8     libucrt:lcidtoname_downlevel.obj
 0001:00005308       ??_C@_1M@IIDEOLLL@?$AAe?$AAs?$AA?9?$AAs?$AAv?$AA?$AA@ 0000000180006308     libucrt:lcidtoname_downlevel.obj
 0001:00005318       ??_C@_1M@GAOBIPA@?$AAe?$AAs?$AA?9?$AAu?$AAy?$AA?$AA@ 0000000180006318     libucrt:lcidtoname_downlevel.obj
 0001:00005328       ??_C@_1M@JKFFICHJ@?$AAe?$AAs?$AA?9?$AAv?$AAe?$AA?$AA@ 0000000180006328     libucrt:lcidtoname_downlevel.obj
 0001:00005338       ??_C@_1M@PNMLOJDF@?$AAe?$AAt?$AA?9?$AAe?$AAe?$AA?$AA@ 0000000180006338     libucrt:lcidtoname_downlevel.obj
 0001:00005348       ??_C@_1M@GHHLIKEI@?$AAe?$AAu?$AA?9?$AAe?$AAs?$AA?$AA@ 0000000180006348     libucrt:lcidtoname_downlevel.obj
 0001:00005358       ??_C@_1M@PBNONODE@?$AAf?$AAa?$AA?9?$AAi?$AAr?$AA?$AA@ 0000000180006358     libucrt:lcidtoname_downlevel.obj
 0001:00005368       ??_C@_1M@JEEHPMIL@?$AAf?$AAi?$AA?9?$AAf?$AAi?$AA?$AA@ 0000000180006368     libucrt:lcidtoname_downlevel.obj
 0001:00005378       ??_C@_1M@LMDCNDBA@?$AAf?$AAo?$AA?9?$AAf?$AAo?$AA?$AA@ 0000000180006378     libucrt:lcidtoname_downlevel.obj
 0001:00005388       ??_C@_1M@JKEOHLDK@?$AAf?$AAr?$AA?9?$AAb?$AAe?$AA?$AA@ 0000000180006388     libucrt:lcidtoname_downlevel.obj
 0001:00005398       ??_C@_1M@NOHADPMI@?$AAf?$AAr?$AA?9?$AAc?$AAa?$AA?$AA@ 0000000180006398     libucrt:lcidtoname_downlevel.obj
 0001:000053a8       ??_C@_1M@KDHIHAEC@?$AAf?$AAr?$AA?9?$AAc?$AAh?$AA?$AA@ 00000001800063a8     libucrt:lcidtoname_downlevel.obj
 0001:000053b8       ??_C@_1M@MMBBFGAK@?$AAf?$AAr?$AA?9?$AAf?$AAr?$AA?$AA@ 00000001800063b8     libucrt:lcidtoname_downlevel.obj
 0001:000053c8       ??_C@_1M@PAFNENNF@?$AAf?$AAr?$AA?9?$AAl?$AAu?$AA?$AA@ 00000001800063c8     libucrt:lcidtoname_downlevel.obj
 0001:000053d8       ??_C@_1M@EOHDJGDD@?$AAf?$AAr?$AA?9?$AAm?$AAc?$AA?$AA@ 00000001800063d8     libucrt:lcidtoname_downlevel.obj
 0001:000053e8       ??_C@_1M@FAPLLOPF@?$AAg?$AAl?$AA?9?$AAe?$AAs?$AA?$AA@ 00000001800063e8     libucrt:lcidtoname_downlevel.obj
 0001:000053f8       ??_C@_1M@FOPBFLOO@?$AAg?$AAu?$AA?9?$AAi?$AAn?$AA?$AA@ 00000001800063f8     libucrt:lcidtoname_downlevel.obj
 0001:00005408       ??_C@_1M@KBMCINPM@?$AAh?$AAe?$AA?9?$AAi?$AAl?$AA?$AA@ 0000000180006408     libucrt:lcidtoname_downlevel.obj
 0001:00005418       ??_C@_1M@BBPHKFPJ@?$AAh?$AAi?$AA?9?$AAi?$AAn?$AA?$AA@ 0000000180006418     libucrt:lcidtoname_downlevel.obj
 0001:00005428       ??_C@_1M@PMBNDPHD@?$AAh?$AAr?$AA?9?$AAb?$AAa?$AA?$AA@ 0000000180006428     libucrt:lcidtoname_downlevel.obj
 0001:00005438       ??_C@_1M@BPCKOEGE@?$AAh?$AAr?$AA?9?$AAh?$AAr?$AA?$AA@ 0000000180006438     libucrt:lcidtoname_downlevel.obj
 0001:00005448       ??_C@_1M@GACBMHKE@?$AAh?$AAu?$AA?9?$AAh?$AAu?$AA?$AA@ 0000000180006448     libucrt:lcidtoname_downlevel.obj
 0001:00005458       ??_C@_1M@MILPAJJC@?$AAh?$AAy?$AA?9?$AAa?$AAm?$AA?$AA@ 0000000180006458     libucrt:lcidtoname_downlevel.obj
 0001:00005468       ??_C@_1M@BABBICEC@?$AAi?$AAd?$AA?9?$AAi?$AAd?$AA?$AA@ 0000000180006468     libucrt:lcidtoname_downlevel.obj
 0001:00005478       ??_C@_1M@BIKNHHPF@?$AAi?$AAs?$AA?9?$AAi?$AAs?$AA?$AA@ 0000000180006478     libucrt:lcidtoname_downlevel.obj
 0001:00005488       ??_C@_1M@NMPCJPHE@?$AAi?$AAt?$AA?9?$AAc?$AAh?$AA?$AA@ 0000000180006488     libucrt:lcidtoname_downlevel.obj
 0001:00005498       ??_C@_1M@GHKGFEDF@?$AAi?$AAt?$AA?9?$AAi?$AAt?$AA?$AA@ 0000000180006498     libucrt:lcidtoname_downlevel.obj
 0001:000054a8       ??_C@_1M@NIEJCJJA@?$AAj?$AAa?$AA?9?$AAj?$AAp?$AA?$AA@ 00000001800064a8     libucrt:lcidtoname_downlevel.obj
 0001:000054b8       ??_C@_1M@JILFNBIM@?$AAk?$AAa?$AA?9?$AAg?$AAe?$AA?$AA@ 00000001800064b8     libucrt:lcidtoname_downlevel.obj
 0001:000054c8       ??_C@_1M@PACPMGPH@?$AAk?$AAk?$AA?9?$AAk?$AAz?$AA?$AA@ 00000001800064c8     libucrt:lcidtoname_downlevel.obj
 0001:000054d8       ??_C@_1M@IELFGMHA@?$AAk?$AAn?$AA?9?$AAi?$AAn?$AA?$AA@ 00000001800064d8     libucrt:lcidtoname_downlevel.obj
 0001:000054e8       ??_C@_1O@IBBJHCH@?$AAk?$AAo?$AAk?$AA?9?$AAi?$AAn?$AA?$AA@ 00000001800064e8     libucrt:lcidtoname_downlevel.obj
 0001:000054f8       ??_C@_1M@DMHAEOGC@?$AAk?$AAo?$AA?9?$AAk?$AAr?$AA?$AA@ 00000001800064f8     libucrt:lcidtoname_downlevel.obj
 0001:00005508       ??_C@_1M@HBAHBIGA@?$AAk?$AAy?$AA?9?$AAk?$AAg?$AA?$AA@ 0000000180006508     libucrt:lcidtoname_downlevel.obj
 0001:00005518       ??_C@_1M@KPMILCJG@?$AAl?$AAt?$AA?9?$AAl?$AAt?$AA?$AA@ 0000000180006518     libucrt:lcidtoname_downlevel.obj
 0001:00005528       ??_C@_1M@BDEKKCA@?$AAl?$AAv?$AA?9?$AAl?$AAv?$AA?$AA@ 0000000180006528     libucrt:lcidtoname_downlevel.obj
 0001:00005538       ??_C@_1M@ELCKCCJJ@?$AAm?$AAi?$AA?9?$AAn?$AAz?$AA?$AA@ 0000000180006538     libucrt:lcidtoname_downlevel.obj
 0001:00005548       ??_C@_1M@CBOOLAPA@?$AAm?$AAk?$AA?9?$AAm?$AAk?$AA?$AA@ 0000000180006548     libucrt:lcidtoname_downlevel.obj
 0001:00005558       ??_C@_1M@GPHNBJKN@?$AAm?$AAl?$AA?9?$AAi?$AAn?$AA?$AA@ 0000000180006558     libucrt:lcidtoname_downlevel.obj
 0001:00005568       ??_C@_1M@PABJILIG@?$AAm?$AAn?$AA?9?$AAm?$AAn?$AA?$AA@ 0000000180006568     libucrt:lcidtoname_downlevel.obj
 0001:00005578       ??_C@_1M@FGBKKIPG@?$AAm?$AAr?$AA?9?$AAi?$AAn?$AA?$AA@ 0000000180006578     libucrt:lcidtoname_downlevel.obj
 0001:00005588       ??_C@_1M@NDBPDDAL@?$AAm?$AAs?$AA?9?$AAb?$AAn?$AA?$AA@ 0000000180006588     libucrt:lcidtoname_downlevel.obj
 0001:00005598       ??_C@_1M@OPIHOOPI@?$AAm?$AAs?$AA?9?$AAm?$AAy?$AA?$AA@ 0000000180006598     libucrt:lcidtoname_downlevel.obj
 0001:000055a8       ??_C@_1M@PPDBCNFM@?$AAm?$AAt?$AA?9?$AAm?$AAt?$AA?$AA@ 00000001800065a8     libucrt:lcidtoname_downlevel.obj
 0001:000055b8       ??_C@_1M@KDJDKMDD@?$AAn?$AAb?$AA?9?$AAn?$AAo?$AA?$AA@ 00000001800065b8     libucrt:lcidtoname_downlevel.obj
 0001:000055c8       ??_C@_1M@KFCFLMJP@?$AAn?$AAl?$AA?9?$AAb?$AAe?$AA?$AA@ 00000001800065c8     libucrt:lcidtoname_downlevel.obj
 0001:000055d8       ??_C@_1M@KPOPDDGO@?$AAn?$AAl?$AA?9?$AAn?$AAl?$AA?$AA@ 00000001800065d8     libucrt:lcidtoname_downlevel.obj
 0001:000055e8       ??_C@_1M@LJKPEMLN@?$AAn?$AAn?$AA?9?$AAn?$AAo?$AA?$AA@ 00000001800065e8     libucrt:lcidtoname_downlevel.obj
 0001:000055f8       ??_C@_1M@BDGHHBFL@?$AAn?$AAs?$AA?9?$AAz?$AAa?$AA?$AA@ 00000001800065f8     libucrt:lcidtoname_downlevel.obj
 0001:00005608       ??_C@_1M@IDEHOAP@?$AAp?$AAa?$AA?9?$AAi?$AAn?$AA?$AA@ 0000000180006608     libucrt:lcidtoname_downlevel.obj
 0001:00005618       ??_C@_1M@HDBKGOGH@?$AAp?$AAl?$AA?9?$AAp?$AAl?$AA?$AA@ 0000000180006618     libucrt:lcidtoname_downlevel.obj
 0001:00005628       ??_C@_1M@LJLLCMEH@?$AAp?$AAt?$AA?9?$AAb?$AAr?$AA?$AA@ 0000000180006628     libucrt:lcidtoname_downlevel.obj
 0001:00005638       ??_C@_1M@NCMONAAL@?$AAp?$AAt?$AA?9?$AAp?$AAt?$AA?$AA@ 0000000180006638     libucrt:lcidtoname_downlevel.obj
 0001:00005648       ??_C@_1O@EAKMAJDN@?$AAq?$AAu?$AAz?$AA?9?$AAb?$AAo?$AA?$AA@ 0000000180006648     libucrt:lcidtoname_downlevel.obj
 0001:00005658       ??_C@_1O@BHHPIGDN@?$AAq?$AAu?$AAz?$AA?9?$AAe?$AAc?$AA?$AA@ 0000000180006658     libucrt:lcidtoname_downlevel.obj
 0001:00005668       ??_C@_1O@GBAPEKMJ@?$AAq?$AAu?$AAz?$AA?9?$AAp?$AAe?$AA?$AA@ 0000000180006668     libucrt:lcidtoname_downlevel.obj
 0001:00005678       ??_C@_1M@CLGLEFBO@?$AAr?$AAo?$AA?9?$AAr?$AAo?$AA?$AA@ 0000000180006678     libucrt:lcidtoname_downlevel.obj
 0001:00005688       ??_C@_1M@CEEDODME@?$AAr?$AAu?$AA?9?$AAr?$AAu?$AA?$AA@ 0000000180006688     libucrt:lcidtoname_downlevel.obj
 0001:00005698       ??_C@_1M@HPKKKMPP@?$AAs?$AAa?$AA?9?$AAi?$AAn?$AA?$AA@ 0000000180006698     libucrt:lcidtoname_downlevel.obj
 0001:000056a8       ??_C@_1M@BKMAIGOJ@?$AAs?$AAe?$AA?9?$AAf?$AAi?$AA?$AA@ 00000001800066a8     libucrt:lcidtoname_downlevel.obj
 0001:000056b8       ??_C@_1M@NDPIFLFI@?$AAs?$AAe?$AA?9?$AAn?$AAo?$AA?$AA@ 00000001800066b8     libucrt:lcidtoname_downlevel.obj
 0001:000056c8       ??_C@_1M@DANKKHJ@?$AAs?$AAe?$AA?9?$AAs?$AAe?$AA?$AA@ 00000001800066c8     libucrt:lcidtoname_downlevel.obj
 0001:000056d8       ??_C@_1M@PNBLONPJ@?$AAs?$AAk?$AA?9?$AAs?$AAk?$AA?$AA@ 00000001800066d8     libucrt:lcidtoname_downlevel.obj
 0001:000056e8       ??_C@_1M@LFMODOAL@?$AAs?$AAl?$AA?9?$AAs?$AAi?$AA?$AA@ 00000001800066e8     libucrt:lcidtoname_downlevel.obj
 0001:000056f8       ??_C@_1O@DFKOMPG@?$AAs?$AAm?$AAa?$AA?9?$AAn?$AAo?$AA?$AA@ 00000001800066f8     libucrt:lcidtoname_downlevel.obj
 0001:00005708       ??_C@_1O@NDKPBNNH@?$AAs?$AAm?$AAa?$AA?9?$AAs?$AAe?$AA?$AA@ 0000000180006708     libucrt:lcidtoname_downlevel.obj
 0001:00005718       ??_C@_1O@PLLKBHAB@?$AAs?$AAm?$AAj?$AA?9?$AAn?$AAo?$AA?$AA@ 0000000180006718     libucrt:lcidtoname_downlevel.obj
 0001:00005728       ??_C@_1O@CLEPOGCA@?$AAs?$AAm?$AAj?$AA?9?$AAs?$AAe?$AA?$AA@ 0000000180006728     libucrt:lcidtoname_downlevel.obj
 0001:00005738       ??_C@_1O@DLGJGKMK@?$AAs?$AAm?$AAn?$AA?9?$AAf?$AAi?$AA?$AA@ 0000000180006738     libucrt:lcidtoname_downlevel.obj
 0001:00005748       ??_C@_1O@OJDJGAJC@?$AAs?$AAm?$AAs?$AA?9?$AAf?$AAi?$AA?$AA@ 0000000180006748     libucrt:lcidtoname_downlevel.obj
 0001:00005758       ??_C@_1M@BOFOGHPB@?$AAs?$AAq?$AA?9?$AAa?$AAl?$AA?$AA@ 0000000180006758     libucrt:lcidtoname_downlevel.obj
 0001:00005768       ??_C@_1BG@LJBBIPGB@?$AAs?$AAr?$AA?9?$AAb?$AAa?$AA?9?$AAc?$AAy?$AAr?$AAl?$AA?$AA@ 0000000180006768     libucrt:lcidtoname_downlevel.obj
 0001:00005780       ??_C@_1BG@JLBENFOE@?$AAs?$AAr?$AA?9?$AAb?$AAa?$AA?9?$AAl?$AAa?$AAt?$AAn?$AA?$AA@ 0000000180006780     libucrt:lcidtoname_downlevel.obj
 0001:00005798       ??_C@_1BG@KODPNHE@?$AAs?$AAr?$AA?9?$AAs?$AAp?$AA?9?$AAc?$AAy?$AAr?$AAl?$AA?$AA@ 0000000180006798     libucrt:lcidtoname_downlevel.obj
 0001:000057b0       ??_C@_1BG@CIOGKHPB@?$AAs?$AAr?$AA?9?$AAs?$AAp?$AA?9?$AAl?$AAa?$AAt?$AAn?$AA?$AA@ 00000001800067b0     libucrt:lcidtoname_downlevel.obj
 0001:000057c8       ??_C@_1M@NGFJLMAC@?$AAs?$AAv?$AA?9?$AAf?$AAi?$AA?$AA@ 00000001800067c8     libucrt:lcidtoname_downlevel.obj
 0001:000057d8       ??_C@_1M@MPJEJAJC@?$AAs?$AAv?$AA?9?$AAs?$AAe?$AA?$AA@ 00000001800067d8     libucrt:lcidtoname_downlevel.obj
 0001:000057e8       ??_C@_1M@MPNDHLFK@?$AAs?$AAw?$AA?9?$AAk?$AAe?$AA?$AA@ 00000001800067e8     libucrt:lcidtoname_downlevel.obj
 0001:000057f8       ??_C@_1O@KOHBJJI@?$AAs?$AAy?$AAr?$AA?9?$AAs?$AAy?$AA?$AA@ 00000001800067f8     libucrt:lcidtoname_downlevel.obj
 0001:00005808       ??_C@_1M@LDCEFHA@?$AAt?$AAa?$AA?9?$AAi?$AAn?$AA?$AA@ 0000000180006808     libucrt:lcidtoname_downlevel.obj
 0001:00005818       ??_C@_1M@CNJOFAK@?$AAt?$AAe?$AA?9?$AAi?$AAn?$AA?$AA@ 0000000180006818     libucrt:lcidtoname_downlevel.obj
 0001:00005828       ??_C@_1M@GNAECACD@?$AAt?$AAh?$AA?9?$AAt?$AAh?$AA?$AA@ 0000000180006828     libucrt:lcidtoname_downlevel.obj
 0001:00005838       ??_C@_1M@CHBIHOJO@?$AAt?$AAn?$AA?9?$AAz?$AAa?$AA?$AA@ 0000000180006838     libucrt:lcidtoname_downlevel.obj
 0001:00005848       ??_C@_1M@GCCMIGPJ@?$AAt?$AAr?$AA?9?$AAt?$AAr?$AA?$AA@ 0000000180006848     libucrt:lcidtoname_downlevel.obj
 0001:00005858       ??_C@_1M@CELMCNBK@?$AAt?$AAt?$AA?9?$AAr?$AAu?$AA?$AA@ 0000000180006858     libucrt:lcidtoname_downlevel.obj
 0001:00005868       ??_C@_1M@KLMCELGA@?$AAu?$AAk?$AA?9?$AAu?$AAa?$AA?$AA@ 0000000180006868     libucrt:lcidtoname_downlevel.obj
 0001:00005878       ??_C@_1M@EPAJJAJF@?$AAu?$AAr?$AA?9?$AAp?$AAk?$AA?$AA@ 0000000180006878     libucrt:lcidtoname_downlevel.obj
 0001:00005888       ??_C@_1BG@GEGPMCDJ@?$AAu?$AAz?$AA?9?$AAu?$AAz?$AA?9?$AAc?$AAy?$AAr?$AAl?$AA?$AA@ 0000000180006888     libucrt:lcidtoname_downlevel.obj
 0001:000058a0       ??_C@_1BG@EGGKJILM@?$AAu?$AAz?$AA?9?$AAu?$AAz?$AA?9?$AAl?$AAa?$AAt?$AAn?$AA?$AA@ 00000001800068a0     libucrt:lcidtoname_downlevel.obj
 0001:000058b8       ??_C@_1M@GFOCLFF@?$AAv?$AAi?$AA?9?$AAv?$AAn?$AA?$AA@ 00000001800068b8     libucrt:lcidtoname_downlevel.obj
 0001:000058c8       ??_C@_1M@CPAMEDFI@?$AAx?$AAh?$AA?9?$AAz?$AAa?$AA?$AA@ 00000001800068c8     libucrt:lcidtoname_downlevel.obj
 0001:000058d8       ??_C@_1O@EBKIFIGN@?$AAz?$AAh?$AA?9?$AAc?$AAh?$AAs?$AA?$AA@ 00000001800068d8     libucrt:lcidtoname_downlevel.obj
 0001:000058e8       ??_C@_1O@NMHPGANE@?$AAz?$AAh?$AA?9?$AAc?$AAh?$AAt?$AA?$AA@ 00000001800068e8     libucrt:lcidtoname_downlevel.obj
 0001:000058f8       ??_C@_1M@LPINJOMC@?$AAz?$AAh?$AA?9?$AAc?$AAn?$AA?$AA@ 00000001800068f8     libucrt:lcidtoname_downlevel.obj
 0001:00005908       ??_C@_1M@OCJEJODD@?$AAz?$AAh?$AA?9?$AAh?$AAk?$AA?$AA@ 0000000180006908     libucrt:lcidtoname_downlevel.obj
 0001:00005918       ??_C@_1M@DNDLJINH@?$AAz?$AAh?$AA?9?$AAm?$AAo?$AA?$AA@ 0000000180006918     libucrt:lcidtoname_downlevel.obj
 0001:00005928       ??_C@_1M@MBFDNDND@?$AAz?$AAh?$AA?9?$AAs?$AAg?$AA?$AA@ 0000000180006928     libucrt:lcidtoname_downlevel.obj
 0001:00005938       ??_C@_1M@IMEPLEPE@?$AAz?$AAh?$AA?9?$AAt?$AAw?$AA?$AA@ 0000000180006938     libucrt:lcidtoname_downlevel.obj
 0001:00005948       ??_C@_1M@BBGHNHJP@?$AAz?$AAu?$AA?9?$AAz?$AAa?$AA?$AA@ 0000000180006948     libucrt:lcidtoname_downlevel.obj
 0001:00005bb0       __log10_256_lead           0000000180006bb0     libucrt:log10_256_lead_tail_table.obj
 0001:000063c0       __log10_256_tail           00000001800073c0     libucrt:log10_256_lead_tail_table.obj
 0001:00006bd0       __log_F_inv_qword          0000000180007bd0     libucrt:log_f_inv_qword_table.obj
 0001:000073e0       ??_C@_05HGHHAHAP@log10?$AA@ 00000001800083e0     libucrt:log_special.obj
 0001:000073e8       ??_C@_1BA@BALFACEM@?$AAC?$AAO?$AAN?$AAO?$AAU?$AAT?$AA$?$AA?$AA@ 00000001800083e8     libucrt:initcon.obj
 0001:00007440       _load_config_used          0000000180008440     LIBCMT:loadcfg.obj
 0001:000074d8       ??_R4exception@std@@6B@    00000001800084d8     LIBCMT:throw_bad_alloc.obj
 0001:00007500       ??_R3exception@std@@8      0000000180008500     LIBCMT:throw_bad_alloc.obj
 0001:00007518       ??_R2exception@std@@8      0000000180008518     LIBCMT:throw_bad_alloc.obj
 0001:00007528       ??_R1A@?0A@EA@exception@std@@8 0000000180008528     LIBCMT:throw_bad_alloc.obj
 0001:00007550       ??_R4bad_alloc@std@@6B@    0000000180008550     LIBCMT:throw_bad_alloc.obj
 0001:00007578       ??_R3bad_alloc@std@@8      0000000180008578     LIBCMT:throw_bad_alloc.obj
 0001:00007590       ??_R2bad_alloc@std@@8      0000000180008590     LIBCMT:throw_bad_alloc.obj
 0001:000075a8       ??_R1A@?0A@EA@bad_alloc@std@@8 00000001800085a8     LIBCMT:throw_bad_alloc.obj
 0001:000075d0       ??_R4bad_array_new_length@std@@6B@ 00000001800085d0     LIBCMT:throw_bad_alloc.obj
 0001:000075f8       ??_R3bad_array_new_length@std@@8 00000001800085f8     LIBCMT:throw_bad_alloc.obj
 0001:00007610       ??_R2bad_array_new_length@std@@8 0000000180008610     LIBCMT:throw_bad_alloc.obj
 0001:00007630       ??_R1A@?0A@EA@bad_array_new_length@std@@8 0000000180008630     LIBCMT:throw_bad_alloc.obj
 0001:00007658       ??_R4type_info@@6B@        0000000180008658     LIBCMT:std_type_info_static.obj
 0001:00007680       ??_R3type_info@@8          0000000180008680     LIBCMT:std_type_info_static.obj
 0001:00007698       ??_R2type_info@@8          0000000180008698     LIBCMT:std_type_info_static.obj
 0001:000076a8       ??_R1A@?0A@EA@type_info@@8 00000001800086a8     LIBCMT:std_type_info_static.obj
 0001:000076d0       ?_TraceLoggingMetadata@?1??_TlgWrite@__vcrt_trace_logging_provider@@YAJPEBU_TlgProvider_t@2@PEFBXPEBU_GUID@@2IPEAU_EVENT_DATA_DESCRIPTOR@@@Z@4U_TraceLoggingMetadata_t@2@B 00000001800086d0     libvcruntime:telemetry.obj
 0001:00007783       ?_TraceLoggingMetadataEnd@?1??_TlgWrite@__vcrt_trace_logging_provider@@YAJPEBU_TlgProvider_t@2@PEFBXPEBU_GUID@@2IPEAU_EVENT_DATA_DESCRIPTOR@@@Z@4EB 0000000180008783     libvcruntime:telemetry.obj
 0001:00007ad0       __rtc_iaa                  0000000180008ad0     LIBCMT:_initsect_.obj
 0001:00007ad8       __rtc_izz                  0000000180008ad8     LIBCMT:_initsect_.obj
 0001:00007ae0       __rtc_taa                  0000000180008ae0     LIBCMT:_initsect_.obj
 0001:00007ae8       __rtc_tzz                  0000000180008ae8     LIBCMT:_initsect_.obj
 0001:00007af0       ?TraceLoggingRegister@__vcrt_trace_logging_provider@@YAJPEBU_TlgProvider_t@1@PEBU_GUID@@P6AX1KE_K2PEAU_EVENT_FILTER_DESCRIPTOR@@PEAX@Z4@Z 0000000180008af0 f i libvcruntime:telemetry.obj
 0001:00007b6c       ?_TlgEnableCallback@__vcrt_trace_logging_provider@@YAXPEBU_GUID@@KE_K1PEAU_EVENT_FILTER_DESCRIPTOR@@PEAX@Z 0000000180008b6c f i libvcruntime:telemetry.obj
 0001:00007c30       ?_TlgWrite@__vcrt_trace_logging_provider@@YAJPEBU_TlgProvider_t@1@PEFBXPEBU_GUID@@2IPEAU_EVENT_DATA_DESCRIPTOR@@@Z 0000000180008c30 f i libvcruntime:telemetry.obj
 0001:00007ce0       __chkstk                   0000000180008ce0 f   chkstk.obj
 0001:00007ce0       _alloca_probe              0000000180008ce0 f   chkstk.obj
 0001:00007d40       ??0PluginIntEditFieldBinding@@QEAA@AEBUPluginStartupInfo@@PEAPEAXHPEAHH@Z 0000000180008d40 f i Brackets.obj
 0001:00007e00       ??0PluginUIntEditFieldBinding@@QEAA@AEBUPluginStartupInfo@@PEAPEAXHPEAIH@Z 0000000180008e00 f i Brackets.obj
 0001:00007ec0       ??1?$DialogBuilderBase@UFarDialogItem@@@@MEAA@XZ 0000000180008ec0 f i Brackets.obj
 0001:00007f40       ??_G?$DialogBuilderBase@UFarDialogItem@@@@MEAAPEAXI@Z 0000000180008f40 f i Brackets.obj
 0001:00007f40       ??_E?$DialogBuilderBase@UFarDialogItem@@@@MEAAPEAXI@Z 0000000180008f40 f i Brackets.obj
 0001:00007f80       ??_E?$DialogItemBinding@UFarDialogItem@@@@UEAAPEAXI@Z 0000000180008f80 f i Brackets.obj
 0001:00007f80       ??_G?$DialogItemBinding@UFarDialogItem@@@@UEAAPEAXI@Z 0000000180008f80 f i Brackets.obj
 0001:00007fb0       ??_GPluginDialogBuilder@@UEAAPEAXI@Z 0000000180008fb0 f i Brackets.obj
 0001:00007fb0       ??_EPluginDialogBuilder@@UEAAPEAXI@Z 0000000180008fb0 f i Brackets.obj
 0001:00008000       ??_EPluginEditFieldBinding@@UEAAPEAXI@Z 0000000180009000 f i Brackets.obj
 0001:00008000       ??_GPluginCheckBoxBinding@@UEAAPEAXI@Z 0000000180009000 f i Brackets.obj
 0001:00008000       ??_EPluginCheckBoxBinding@@UEAAPEAXI@Z 0000000180009000 f i Brackets.obj
 0001:00008000       ??_GPluginEditFieldBinding@@UEAAPEAXI@Z 0000000180009000 f i Brackets.obj
 0001:00008030       ??_EPluginRadioButtonBinding@@UEAAPEAXI@Z 0000000180009030 f i Brackets.obj
 0001:00008030       ??_GPluginRadioButtonBinding@@UEAAPEAXI@Z 0000000180009030 f i Brackets.obj
 0001:00008060       ??_EPluginIntEditFieldBinding@@UEAAPEAXI@Z 0000000180009060 f i Brackets.obj
 0001:00008060       ??_EPluginUIntEditFieldBinding@@UEAAPEAXI@Z 0000000180009060 f i Brackets.obj
 0001:00008060       ??_GPluginIntEditFieldBinding@@UEAAPEAXI@Z 0000000180009060 f i Brackets.obj
 0001:00008060       ??_GPluginUIntEditFieldBinding@@UEAAPEAXI@Z 0000000180009060 f i Brackets.obj
 0001:00008090       ?AddButtons@?$DialogBuilderBase@UFarDialogItem@@@@QEAAXHPEBHHH@Z 0000000180009090 f i Brackets.obj
 0001:000081f0       ?AddIntEditField@PluginDialogBuilder@@UEAAPEAUFarDialogItem@@PEAHH@Z 00000001800091f0 f i Brackets.obj
 0001:00008300       ?AddUIntEditField@PluginDialogBuilder@@UEAAPEAUFarDialogItem@@PEAIH@Z 0000000180009300 f i Brackets.obj
 0001:00008410       ?Config@@YAHXZ             0000000180009410 f   Brackets.obj
 0001:00009540       ?CreateCheckBoxBinding@PluginDialogBuilder@@MEAAPEAU?$DialogItemBinding@UFarDialogItem@@@@PEAHH@Z 000000018000a540 f i Brackets.obj
 0001:000095c0       ?AddIntEditField@?$DialogBuilderBase@UFarDialogItem@@@@UEAAPEAUFarDialogItem@@PEAHH@Z 000000018000a5c0 f i Brackets.obj
 0001:000095c0       ?CreateRadioButtonBinding@?$DialogBuilderBase@UFarDialogItem@@@@MEAAPEAU?$DialogItemBinding@UFarDialogItem@@@@PEAH@Z 000000018000a5c0 f i Brackets.obj
 0001:000095c0       ?GetLangString@?$DialogBuilderBase@UFarDialogItem@@@@MEAAPEB_WH@Z 000000018000a5c0 f i Brackets.obj
 0001:000095c0       ?CreateCheckBoxBinding@?$DialogBuilderBase@UFarDialogItem@@@@MEAAPEAU?$DialogItemBinding@UFarDialogItem@@@@PEAHH@Z 000000018000a5c0 f i Brackets.obj
 0001:000095c0       ?AddUIntEditField@?$DialogBuilderBase@UFarDialogItem@@@@UEAAPEAUFarDialogItem@@PEAIH@Z 000000018000a5c0 f i Brackets.obj
 0001:000095d0       ?CreateRadioButtonBinding@PluginDialogBuilder@@MEAAPEAU?$DialogItemBinding@UFarDialogItem@@@@PEAH@Z 000000018000a5d0 f i Brackets.obj
 0001:00009640       ?DoShowDialog@?$DialogBuilderBase@UFarDialogItem@@@@MEAA_JXZ 000000018000a640 f i Brackets.obj
 0001:00009650       ?DoShowDialog@PluginDialogBuilder@@MEAA_JXZ 000000018000a650 f i Brackets.obj
 0001:00009700       ?GetLangString@PluginDialogBuilder@@MEAAPEB_WH@Z 000000018000a700 f i Brackets.obj
 0001:00009710       ?InitDialogItem@PluginDialogBuilder@@MEAAXPEAUFarDialogItem@@PEB_W@Z 000000018000a710 f i Brackets.obj
 0001:00009740       ?ItemWidth@?$DialogBuilderBase@UFarDialogItem@@@@IEAA_JAEBUFarDialogItem@@@Z 000000018000a740 f i Brackets.obj
 0001:000097e0       ?MaxTextWidth@?$DialogBuilderBase@UFarDialogItem@@@@IEAA_JXZ 000000018000a7e0 f i Brackets.obj
 0001:00009910       ?ReallocDialogItems@?$DialogBuilderBase@UFarDialogItem@@@@IEAAXXZ 000000018000a910 f i Brackets.obj
 0001:00009a70       ?SaveValue@PluginCheckBoxBinding@@UEAAXPEAUFarDialogItem@@H@Z 000000018000aa70 f i Brackets.obj
 0001:00009ad0       ?SaveValue@PluginEditFieldBinding@@UEAAXPEAUFarDialogItem@@H@Z 000000018000aad0 f i Brackets.obj
 0001:00009b10       ?SaveValue@PluginIntEditFieldBinding@@UEAAXPEAUFarDialogItem@@H@Z 000000018000ab10 f i Brackets.obj
 0001:00009b60       ?SaveValue@PluginRadioButtonBinding@@UEAAXPEAUFarDialogItem@@H@Z 000000018000ab60 f i Brackets.obj
 0001:00009bb0       ?SaveValue@PluginUIntEditFieldBinding@@UEAAXPEAUFarDialogItem@@H@Z 000000018000abb0 f i Brackets.obj
 0001:00009c00       ?SaveValues@?$DialogBuilderBase@UFarDialogItem@@@@IEAAXXZ 000000018000ac00 f i Brackets.obj
 0001:00009c90       ?ShowMenu@@YAHH@Z          000000018000ac90 f   Brackets.obj
 0001:00009e20       ?TextWidth@?$DialogBuilderBase@UFarDialogItem@@@@MEAAHAEBUFarDialogItem@@@Z 000000018000ae20 f i Brackets.obj
 0001:00009e30       ?TextWidth@PluginDialogBuilder@@MEAAHAEBUFarDialogItem@@@Z 000000018000ae30 f i Brackets.obj
 0001:00009e40       ?UpdateBorderSize@?$DialogBuilderBase@UFarDialogItem@@@@IEAAXXZ 000000018000ae40 f i Brackets.obj
 0001:00009f00       ConfigureW                 000000018000af00 f   Brackets.obj
 0001:00009f10       GetGlobalInfoW             000000018000af10 f   Brackets.obj
 0001:00009f90       GetPluginInfoW             000000018000af90 f   Brackets.obj
 0001:0000a000       OpenW                      000000018000b000 f   Brackets.obj
 0001:0000ab60       SetStartupInfoW            000000018000bb60 f   Brackets.obj
 0001:0000aea8       ??2@YAPEAX_K@Z             000000018000bea8 f   LIBCMT:new_scalar.obj
 0001:0000aee4       ??_V@YAXPEAX@Z             000000018000bee4 f   LIBCMT:delete_array.obj
 0001:0000aee4       ??3@YAXPEAX_K@Z            000000018000bee4 f   LIBCMT:delete_scalar_size.obj
 0001:0000aeec       ??_U@YAPEAX_K@Z            000000018000beec f   LIBCMT:new_array.obj
 0001:0000b250       _DllMainCRTStartup         000000018000c250 f   LIBCMT:dll_dllmain.obj
 0001:0000b290       ??0bad_alloc@std@@QEAA@AEBV01@@Z 000000018000c290 f i LIBCMT:throw_bad_alloc.obj
 0001:0000b2d0       ??0bad_alloc@std@@QEAA@XZ  000000018000c2d0 f i LIBCMT:throw_bad_alloc.obj
 0001:0000b2f0       ??0bad_array_new_length@std@@QEAA@AEBV01@@Z 000000018000c2f0 f i LIBCMT:throw_bad_alloc.obj
 0001:0000b330       ??0bad_array_new_length@std@@QEAA@XZ 000000018000c330 f i LIBCMT:throw_bad_alloc.obj
 0001:0000b350       ??0exception@std@@QEAA@AEBV01@@Z 000000018000c350 f i LIBCMT:throw_bad_alloc.obj
 0001:0000b388       ??1bad_alloc@std@@UEAA@XZ  000000018000c388 f i LIBCMT:throw_bad_alloc.obj
 0001:0000b388       ??1bad_array_new_length@std@@UEAA@XZ 000000018000c388 f i LIBCMT:throw_bad_alloc.obj
 0001:0000b39c       ??_Ebad_alloc@std@@UEAAPEAXI@Z 000000018000c39c f i LIBCMT:throw_bad_alloc.obj
 0001:0000b39c       ??_Gbad_array_new_length@std@@UEAAPEAXI@Z 000000018000c39c f i LIBCMT:throw_bad_alloc.obj
 0001:0000b39c       ??_Gbad_alloc@std@@UEAAPEAXI@Z 000000018000c39c f i LIBCMT:throw_bad_alloc.obj
 0001:0000b39c       ??_Eexception@std@@UEAAPEAXI@Z 000000018000c39c f i LIBCMT:throw_bad_alloc.obj
 0001:0000b39c       ??_Ebad_array_new_length@std@@UEAAPEAXI@Z 000000018000c39c f i LIBCMT:throw_bad_alloc.obj
 0001:0000b39c       ??_Gexception@std@@UEAAPEAXI@Z 000000018000c39c f i LIBCMT:throw_bad_alloc.obj
 0001:0000b3e0       ?__scrt_throw_std_bad_alloc@@YAXXZ 000000018000c3e0 f   LIBCMT:throw_bad_alloc.obj
 0001:0000b400       ?__scrt_throw_std_bad_array_new_length@@YAXXZ 000000018000c400 f   LIBCMT:throw_bad_alloc.obj
 0001:0000b420       ?what@exception@std@@UEBAPEBDXZ 000000018000c420 f i LIBCMT:throw_bad_alloc.obj
 0001:0000b434       ??3@YAXPEAX@Z              000000018000c434 f   LIBCMT:delete_scalar.obj
 0001:0000b43c       __scrt_acquire_startup_lock 000000018000c43c f   LIBCMT:utility.obj
 0001:0000b478       __scrt_dllmain_after_initialize_c 000000018000c478 f   LIBCMT:utility.obj
 0001:0000b498       __scrt_dllmain_before_initialize_c 000000018000c498 f   LIBCMT:utility.obj
 0001:0000b4b0       __scrt_dllmain_crt_thread_attach 000000018000c4b0 f   LIBCMT:utility.obj
 0001:0000b4d8       __scrt_dllmain_crt_thread_detach 000000018000c4d8 f   LIBCMT:utility.obj
 0001:0000b4f0       __scrt_dllmain_exception_filter 000000018000c4f0 f   LIBCMT:utility.obj
 0001:0000b554       __scrt_dllmain_uninitialize_c 000000018000c554 f   LIBCMT:utility.obj
 0001:0000b584       __scrt_dllmain_uninitialize_critical 000000018000c584 f   LIBCMT:utility.obj
 0001:0000b598       __scrt_initialize_crt      000000018000c598 f   LIBCMT:utility.obj
 0001:0000b5e4       __scrt_initialize_onexit_tables 000000018000c5e4 f   LIBCMT:utility.obj
 0001:0000b6b0       __scrt_is_nonwritable_in_current_image 000000018000c6b0 f   LIBCMT:utility.obj
 0001:0000b74c       __scrt_release_startup_lock 000000018000c74c f   LIBCMT:utility.obj
 0001:0000b770       __scrt_uninitialize_crt    000000018000c770 f   LIBCMT:utility.obj
 0001:0000b79c       _onexit                    000000018000c79c f   LIBCMT:utility.obj
 0001:0000b7ec       atexit                     000000018000c7ec f   LIBCMT:utility.obj
 0001:0000b804       __security_init_cookie     000000018000c804 f   LIBCMT:gs_support.obj
 0001:0000b8b0       DllMain                    000000018000c8b0 f   LIBCMT:dll_dllmain_stub.obj
 0001:0000b8b8       ?__scrt_initialize_type_info@@YAXXZ 000000018000c8b8 f   LIBCMT:tncleanup.obj
 0001:0000b8c8       ?__scrt_uninitialize_type_info@@YAXXZ 000000018000c8c8 f   LIBCMT:tncleanup.obj
 0001:0000b8d4       __local_stdio_printf_options 000000018000c8d4 f i LIBCMT:default_local_stdio_options.obj
 0001:0000b8dc       __local_stdio_scanf_options 000000018000c8dc f i LIBCMT:default_local_stdio_options.obj
 0001:0000b8e4       __scrt_initialize_default_local_stdio_options 000000018000c8e4 f   LIBCMT:default_local_stdio_options.obj
 0001:0000b900       __scrt_get_dyn_tls_init_callback 000000018000c900 f   LIBCMT:dyn_tls_init.obj
 0001:0000b908       __crt_debugger_hook        000000018000c908 f   LIBCMT:utility_desktop.obj
 0001:0000b910       __scrt_fastfail            000000018000c910 f   LIBCMT:utility_desktop.obj
 0001:0000ba58       _RTC_Initialize            000000018000ca58 f   LIBCMT:_initsect_.obj
 0001:0000baa4       _RTC_Terminate             000000018000caa4 f   LIBCMT:_initsect_.obj
 0001:0000baf0       _guard_check_icall         000000018000caf0 f i LIBCMT:checkcfg.obj
 0001:0000baf8       ??_Gtype_info@@UEAAPEAXI@Z 000000018000caf8 f i LIBCMT:std_type_info_static.obj
 0001:0000baf8       ??_Etype_info@@UEAAPEAXI@Z 000000018000caf8 f i LIBCMT:std_type_info_static.obj
 0001:0000bb24       __isa_available_init       000000018000cb24 f   LIBCMT:_cpu_disp_.obj
 0001:0000bce8       __scrt_is_ucrt_dll_in_use  000000018000cce8 f   LIBCMT:ucrt_detection.obj
 0001:0000bd10       memset                     000000018000cd10 f   libvcruntime:memset.obj
 0001:0000beb4       __telemetry_main_invoke_trigger 000000018000ceb4 f   libvcruntime:telemetry.obj
 0001:0000bfcc       __telemetry_main_return_trigger 000000018000cfcc f   libvcruntime:telemetry.obj
 0001:0000c0e4       __vcrt_initialize_telemetry_provider 000000018000d0e4 f   libvcruntime:telemetry.obj
 0001:0000c0f8       __vcrt_uninitialize_telemetry_provider 000000018000d0f8 f   libvcruntime:telemetry.obj
 0001:0000c118       __C_specific_handler       000000018000d118 f   libvcruntime:_chandler_.obj
 0001:0000c308       __std_exception_copy       000000018000d308 f   libvcruntime:std_exception.obj
 0001:0000c398       __std_exception_destroy    000000018000d398 f   libvcruntime:std_exception.obj
 0001:0000c3c0       _CxxThrowException         000000018000d3c0 f   libvcruntime:throw.obj
 0001:0000c498       __vcrt_initialize          000000018000d498 f   libvcruntime:initialization.obj
 0001:0000c4d0       __vcrt_thread_attach       000000018000d4d0 f   libvcruntime:initialization.obj
 0001:0000c4e4       __vcrt_thread_detach       000000018000d4e4 f   libvcruntime:initialization.obj
 0001:0000c4f8       __vcrt_uninitialize        000000018000d4f8 f   libvcruntime:initialization.obj
 0001:0000c524       __vcrt_uninitialize_critical 000000018000d524 f   libvcruntime:initialization.obj
 0001:0000c534       __std_type_info_destroy_list 000000018000d534 f   libvcruntime:std_type_info.obj
 0001:0000c728       __vcrt_EventRegister       000000018000d728 f   libvcruntime:winapi_downlevel.obj
 0001:0000c7ac       __vcrt_EventSetInformation 000000018000d7ac f   libvcruntime:winapi_downlevel.obj
 0001:0000c830       __vcrt_EventUnregister     000000018000d830 f   libvcruntime:winapi_downlevel.obj
 0001:0000c884       __vcrt_EventWriteTransfer  000000018000d884 f   libvcruntime:winapi_downlevel.obj
 0001:0000c91c       __vcrt_FlsAlloc            000000018000d91c f   libvcruntime:winapi_downlevel.obj
 0001:0000c970       __vcrt_FlsFree             000000018000d970 f   libvcruntime:winapi_downlevel.obj
 0001:0000c9c4       __vcrt_FlsGetValue         000000018000d9c4 f   libvcruntime:winapi_downlevel.obj
 0001:0000ca18       __vcrt_FlsSetValue         000000018000da18 f   libvcruntime:winapi_downlevel.obj
 0001:0000ca80       __vcrt_InitializeCriticalSectionEx 000000018000da80 f   libvcruntime:winapi_downlevel.obj
 0001:0000caf8       __vcrt_initialize_winapi_thunks 000000018000daf8 f   libvcruntime:winapi_downlevel.obj
 0001:0000cb30       __vcrt_uninitialize_winapi_thunks 000000018000db30 f   libvcruntime:winapi_downlevel.obj
 0001:0000cb80       _local_unwind              000000018000db80 f   libvcruntime:_jmpuwind_.obj
 0001:0000cbb0       _NLG_Notify                000000018000dbb0 f   libvcruntime:_jmpuwind_.obj
 0001:0000cbd0       __NLG_Dispatch2            000000018000dbd0 f   libvcruntime:_jmpuwind_.obj
 0001:0000cbe0       __NLG_Return2              000000018000dbe0 f   libvcruntime:_jmpuwind_.obj
 0001:0000cbf0       __except_validate_context_record 000000018000dbf0 f   libvcruntime:jbcxrval.obj
 0001:0000cbf0       _guard_check_icall_nop     000000018000dbf0 f   LIBCMT:guard_support.obj
 0001:0000cbf0       ?InitDialogItem@?$DialogBuilderBase@UFarDialogItem@@@@MEAAXPEAUFarDialogItem@@PEB_W@Z 000000018000dbf0 f   Brackets.obj
 0001:0000cbf0       ?SaveValue@?$DialogItemBinding@UFarDialogItem@@@@UEAAXPEAUFarDialogItem@@H@Z 000000018000dbf0 f   Brackets.obj
 0001:0000cbf4       __vcrt_freefls             000000018000dbf4 f   libvcruntime:per_thread_data.obj
 0001:0000cc14       __vcrt_freeptd             000000018000dc14 f   libvcruntime:per_thread_data.obj
 0001:0000cc64       __vcrt_getptd_noexit       000000018000dc64 f   libvcruntime:per_thread_data.obj
 0001:0000cd0c       __vcrt_initialize_ptd      000000018000dd0c f   libvcruntime:per_thread_data.obj
 0001:0000cd4c       __vcrt_uninitialize_ptd    000000018000dd4c f   libvcruntime:per_thread_data.obj
 0001:0000cd70       __vcrt_initialize_locks    000000018000dd70 f   libvcruntime:locks.obj
 0001:0000cdb8       __vcrt_uninitialize_locks  000000018000ddb8 f   libvcruntime:locks.obj
 0001:0000cdf0       __vcrt_initialize_pure_virtual_call_handler 000000018000ddf0 f   libvcruntime:purevirt_data.obj
 0001:0000ce14       __acrt_initialize_new_handler 000000018000de14 f   libucrt:new_handler.obj
 0001:0000ce1c       _callnewh                  000000018000de1c f   libucrt:new_handler.obj
 0001:0000ce5c       _query_new_handler         000000018000de5c f   libucrt:new_handler.obj
 0001:0000ce90       malloc                     000000018000de90 f   libucrt:malloc.obj
 0001:0000ce98       _initterm                  000000018000de98 f   libucrt:initterm.obj
 0001:0000cf10       _initterm_e                000000018000df10 f   libucrt:initterm.obj
 0001:0000cf5c       free                       000000018000df5c f   libucrt:free.obj
 0001:0000cf64       _seh_filter_dll            000000018000df64 f   libucrt:exception_filter.obj
 0001:0000cf78       _seh_filter_exe            000000018000df78 f   libucrt:exception_filter.obj
 0001:0000d338       __acrt_initialize_thread_local_exit_callback 000000018000e338 f   libucrt:exit.obj
 0001:0000d340       _cexit                     000000018000e340 f   libucrt:exit.obj
 0001:0000d350       _exit                      000000018000e350 f   libucrt:exit.obj
 0001:0000d35c       _is_c_termination_complete 000000018000e35c f   libucrt:exit.obj
 0001:0000d548       __dcrt_uninitialize_environments_nolock 000000018000e548 f   libucrt:environment_initialization.obj
 0001:0000d580       _initialize_narrow_environment 000000018000e580 f   libucrt:environment_initialization.obj
 0001:0000d588       ??$?RV<lambda_b8c45f8f788dd370798f47cfe8ac3a86>@@AEAV<lambda_4e60a939b0d047cfe11ddc22648dfba9>@@V<lambda_332c3edc96d0294ec56c57d38c1cdfd5>@@@?$__crt_seh_guarded_call@H@@QEAAH$$QEAV<lambda_b8c45f8f788dd370798f47cfe8ac3a86>@@AEAV<lambda_4e60a939b0d047cfe11ddc22648dfba9>@@$$QEAV<lambda_332c3edc96d0294ec56c57d38c1cdfd5>@@@Z 000000018000e588 f i libucrt:onexit.obj
 0001:0000d5c4       ??$?RV<lambda_e24bbb7b643b32fcea6fa61b31d4c984>@@AEAV<lambda_275893d493268fdec8709772e3fcec0e>@@V<lambda_9d71df4d7cf3f480f8d633942495c3b0>@@@?$__crt_seh_guarded_call@H@@QEAAH$$QEAV<lambda_e24bbb7b643b32fcea6fa61b31d4c984>@@AEAV<lambda_275893d493268fdec8709772e3fcec0e>@@$$QEAV<lambda_9d71df4d7cf3f480f8d633942495c3b0>@@@Z 000000018000e5c4 f i libucrt:onexit.obj
 0001:0000d940       _crt_atexit                000000018000e940 f   libucrt:onexit.obj
 0001:0000d950       _execute_onexit_table      000000018000e950 f   libucrt:onexit.obj
 0001:0000d98c       _initialize_onexit_table   000000018000e98c f   libucrt:onexit.obj
 0001:0000d9cc       _register_onexit_function  000000018000e9cc f   libucrt:onexit.obj
 0001:0000da4c       __acrt_uninitialize_command_line 000000018000ea4c f   libucrt:argv_data.obj
 0001:0000db4c       __acrt_initialize          000000018000eb4c f   libucrt:initialization.obj
 0001:0000db60       __acrt_thread_attach       000000018000eb60 f   libucrt:initialization.obj
 0001:0000db74       __acrt_thread_detach       000000018000eb74 f   libucrt:initialization.obj
 0001:0000db84       __acrt_uninitialize        000000018000eb84 f   libucrt:initialization.obj
 0001:0000db98       __acrt_uninitialize_critical 000000018000eb98 f   libucrt:initialization.obj
 0001:0000dba8       terminate                  000000018000eba8 f   libucrt:terminate.obj
 0001:0000dbd0       strcpy_s                   000000018000ebd0 f   libucrt:strcpy_s.obj
 0001:0000dc30       _free_base                 000000018000ec30 f   libucrt:free_base.obj
 0001:0000dc70       _malloc_base               000000018000ec70 f   libucrt:malloc_base.obj
 0001:0000dcd0       abort                      000000018000ecd0 f   libucrt:abort.obj
 0001:0000dd28       _calloc_base               000000018000ed28 f   libucrt:calloc_base.obj
 0001:0000dda0       ??0_LocaleUpdate@@QEAA@QEAU__crt_locale_pointers@@@Z 000000018000eda0 f i libucrt:output.obj
 0001:0000de30       __acrt_initialize_locks    000000018000ee30 f   libucrt:locks.obj
 0001:0000de78       __acrt_lock                000000018000ee78 f   libucrt:locks.obj
 0001:0000de94       __acrt_uninitialize_locks  000000018000ee94 f   libucrt:locks.obj
 0001:0000decc       __acrt_unlock              000000018000eecc f   libucrt:locks.obj
 0001:0000dee8       ??$?RV<lambda_46352004c1216016012b18bd6f87e700>@@AEAV<lambda_3bd07e1a1191394380780325891bf33f>@@V<lambda_334532d3f185bcaa59b5be82d7d22bff>@@@?$__crt_seh_guarded_call@X@@QEAAX$$QEAV<lambda_46352004c1216016012b18bd6f87e700>@@AEAV<lambda_3bd07e1a1191394380780325891bf33f>@@$$QEAV<lambda_334532d3f185bcaa59b5be82d7d22bff>@@@Z 000000018000eee8 f i libucrt:per_thread_data.obj
 0001:0000df48       ??$?RV<lambda_5e887d1dcbef67a5eb4283622ba103bf>@@AEAV<lambda_4466841279450cc726390878d4a41900>@@V<lambda_341c25c0346d94847f1f3c463c57e077>@@@?$__crt_seh_guarded_call@X@@QEAAX$$QEAV<lambda_5e887d1dcbef67a5eb4283622ba103bf>@@AEAV<lambda_4466841279450cc726390878d4a41900>@@$$QEAV<lambda_341c25c0346d94847f1f3c463c57e077>@@@Z 000000018000ef48 f i libucrt:per_thread_data.obj
 0001:0000df90       ??$?RV<lambda_72d1df2b273a38828b1ce30cbf4cdab5>@@AEAV<lambda_876a65b173b8412d3a47c70a915b0cf4>@@V<lambda_41932305e351933ebe8f8be3ed8bb5dc>@@@?$__crt_seh_guarded_call@X@@QEAAX$$QEAV<lambda_72d1df2b273a38828b1ce30cbf4cdab5>@@AEAV<lambda_876a65b173b8412d3a47c70a915b0cf4>@@$$QEAV<lambda_41932305e351933ebe8f8be3ed8bb5dc>@@@Z 000000018000ef90 f i libucrt:per_thread_data.obj
 0001:0000dfd0       ??$?RV<lambda_fb3a7dec4e47f37f22dae91bb15c9095>@@AEAV<lambda_698284760c8add0bfb0756c19673e34b>@@V<lambda_dfb8eca1e75fef3034a8fb18dd509707>@@@?$__crt_seh_guarded_call@X@@QEAAX$$QEAV<lambda_fb3a7dec4e47f37f22dae91bb15c9095>@@AEAV<lambda_698284760c8add0bfb0756c19673e34b>@@$$QEAV<lambda_dfb8eca1e75fef3034a8fb18dd509707>@@@Z 000000018000efd0 f i libucrt:per_thread_data.obj
 0001:0000e260       __acrt_freeptd             000000018000f260 f   libucrt:per_thread_data.obj
 0001:0000e2a4       __acrt_getptd              000000018000f2a4 f   libucrt:per_thread_data.obj
 0001:0000e338       __acrt_getptd_noexit       000000018000f338 f   libucrt:per_thread_data.obj
 0001:0000e3d8       __acrt_initialize_ptd      000000018000f3d8 f   libucrt:per_thread_data.obj
 0001:0000e414       __acrt_uninitialize_ptd    000000018000f414 f   libucrt:per_thread_data.obj
 0001:0000e5d8       __acrt_FlsAlloc            000000018000f5d8 f   libucrt:winapi_thunks.obj
 0001:0000e630       __acrt_FlsFree             000000018000f630 f   libucrt:winapi_thunks.obj
 0001:0000e688       __acrt_FlsGetValue         000000018000f688 f   libucrt:winapi_thunks.obj
 0001:0000e6e0       __acrt_FlsSetValue         000000018000f6e0 f   libucrt:winapi_thunks.obj
 0001:0000e748       __acrt_InitializeCriticalSectionEx 000000018000f748 f   libucrt:winapi_thunks.obj
 0001:0000e7c0       __acrt_LCMapStringEx       000000018000f7c0 f   libucrt:winapi_thunks.obj
 0001:0000e8b0       __acrt_LocaleNameToLCID    000000018000f8b0 f   libucrt:winapi_thunks.obj
 0001:0000e918       __acrt_initialize_winapi_thunks 000000018000f918 f   libucrt:winapi_thunks.obj
 0001:0000e950       __acrt_is_packaged_app     000000018000f950 f   libucrt:winapi_thunks.obj
 0001:0000e9d8       __acrt_uninitialize_winapi_thunks 000000018000f9d8 f   libucrt:winapi_thunks.obj
 0001:0000ea1c       __acrt_call_reportfault    000000018000fa1c f   libucrt:invalid_parameter.obj
 0001:0000eb78       __acrt_initialize_invalid_parameter_handler 000000018000fb78 f   libucrt:invalid_parameter.obj
 0001:0000eb80       _invalid_parameter         000000018000fb80 f   libucrt:invalid_parameter.obj
 0001:0000ec28       _invalid_parameter_noinfo  000000018000fc28 f   libucrt:invalid_parameter.obj
 0001:0000ec48       _invoke_watson             000000018000fc48 f   libucrt:invalid_parameter.obj
 0001:0000ec90       ??$?RV<lambda_99476a1ad63dd22509b5d3e65b0ffc95>@@AEAV<lambda_ad1ced32f4ac17aa236e5ef05d6b3b7c>@@V<lambda_f7424dd8d45958661754dc4f2697e9c3>@@@?$__crt_seh_guarded_call@X@@QEAAX$$QEAV<lambda_99476a1ad63dd22509b5d3e65b0ffc95>@@AEAV<lambda_ad1ced32f4ac17aa236e5ef05d6b3b7c>@@$$QEAV<lambda_f7424dd8d45958661754dc4f2697e9c3>@@@Z 000000018000fc90 f i libucrt:mbctype.obj
 0001:0000f38c       __acrt_initialize_multibyte 000000018001038c f   libucrt:mbctype.obj
 0001:0000f3b4       __acrt_update_thread_multibyte_data 00000001800103b4 f   libucrt:mbctype.obj
 0001:0000f474       _setmbcp_nolock            0000000180010474 f   libucrt:mbctype.obj
 0001:0000f71c       __dcrt_get_narrow_environment_from_os 000000018001071c f   libucrt:get_environment_from_os.obj
 0001:0000f820       _recalloc                  0000000180010820 f   libucrt:recalloc.obj
 0001:0000f828       _recalloc_base             0000000180010828 f   libucrt:recalloc.obj
 0001:0000f8c0       __acrt_initialize_heap     00000001800108c0 f   libucrt:heap_handle.obj
 0001:0000f8dc       __acrt_uninitialize_heap   00000001800108dc f   libucrt:heap_handle.obj
 0001:0000fad0       __acrt_initialize_lowio    0000000180010ad0 f   libucrt:ioinit.obj
 0001:0000fb0c       __acrt_uninitialize_lowio  0000000180010b0c f   libucrt:ioinit.obj
 0001:0000fb4c       __acrt_initialize_command_line 0000000180010b4c f   libucrt:argv_data.obj
 0001:0000fb74       __acrt_execute_initializers 0000000180010b74 f   libucrt:shared_initialization.obj
 0001:0000fc08       __acrt_execute_uninitializers 0000000180010c08 f   libucrt:shared_initialization.obj
 0001:0000fc58       ??$?RV<lambda_c36588078e9f5dfd39652860aa6b3aaf>@@AEAV<lambda_ec61778202f4f5fc7e7711acc23c3bca>@@V<lambda_dc9d2797ccde5d239b4a0efae8ebd7db>@@@?$__crt_seh_guarded_call@P6AXH@Z@@QEAAP6AXH@Z$$QEAV<lambda_c36588078e9f5dfd39652860aa6b3aaf>@@AEAV<lambda_ec61778202f4f5fc7e7711acc23c3bca>@@$$QEAV<lambda_dc9d2797ccde5d239b4a0efae8ebd7db>@@@Z 0000000180010c58 f i libucrt:signal.obj
 0001:0000fca0       __acrt_get_sigabrt_handler 0000000180010ca0 f   libucrt:signal.obj
 0001:0000fcd0       __acrt_initialize_signal_handlers 0000000180010cd0 f   libucrt:signal.obj
 0001:0000fcf0       raise                      0000000180010cf0 f   libucrt:signal.obj
 0001:0000ff8c       __acrt_has_user_matherr    0000000180010f8c f   libucrt:matherr.obj
 0001:0000ffac       __acrt_initialize_user_matherr 0000000180010fac f   libucrt:matherr.obj
 0001:0000ffb4       __acrt_invoke_user_matherr 0000000180010fb4 f   libucrt:matherr.obj
 0001:0000fffc       __acrt_errno_from_os_error 0000000180010ffc f   libucrt:errno.obj
 0001:00010044       __acrt_errno_map_os_error  0000000180011044 f   libucrt:errno.obj
 0001:00010094       __doserrno                 0000000180011094 f   libucrt:errno.obj
 0001:000100b4       _errno                     00000001800110b4 f   libucrt:errno.obj
 0001:000100d4       _query_new_mode            00000001800110d4 f   libucrt:new_mode.obj
 0001:000100dc       _mbtowc_l                  00000001800110dc f   libucrt:mbtowc.obj
 0001:00010224       mbtowc                     0000000180011224 f   libucrt:mbtowc.obj
 0001:0001022c       __acrt_update_locale_info  000000018001122c f   libucrt:locale_update.obj
 0001:00010260       __acrt_update_multibyte_info 0000000180011260 f   libucrt:locale_update.obj
 0001:00010294       _fileno                    0000000180011294 f   libucrt:fileno.obj
 0001:000102bc       __acrt_initialize_stdio    00000001800112bc f   libucrt:_file.obj
 0001:000103dc       __acrt_uninitialize_stdio  00000001800113dc f   libucrt:_file.obj
 0001:00010438       _lock_file                 0000000180011438 f   libucrt:_file.obj
 0001:00010444       _unlock_file               0000000180011444 f   libucrt:_file.obj
 0001:00010450       __acrt_set_locale_changed  0000000180011450 f   libucrt:wsetlocale.obj
 0001:0001045c       __acrt_uninitialize_locale 000000018001145c f   libucrt:wsetlocale.obj
 0001:000104a4       __pctype_func              00000001800114a4 f   libucrt:ctype.obj
 0001:000104d4       __acrt_add_locale_ref      00000001800114d4 f   libucrt:locale_refcounting.obj
 0001:00010560       __acrt_free_locale         0000000180011560 f   libucrt:locale_refcounting.obj
 0001:000106d8       __acrt_locale_add_lc_time_reference 00000001800116d8 f   libucrt:locale_refcounting.obj
 0001:00010700       __acrt_locale_free_lc_time_if_unreferenced 0000000180011700 f   libucrt:locale_refcounting.obj
 0001:00010738       __acrt_locale_release_lc_time_reference 0000000180011738 f   libucrt:locale_refcounting.obj
 0001:00010760       __acrt_release_locale_ref  0000000180011760 f   libucrt:locale_refcounting.obj
 0001:00010808       __acrt_update_thread_locale_data 0000000180011808 f   libucrt:locale_refcounting.obj
 0001:00010878       _updatetlocinfoEx_nolock   0000000180011878 f   libucrt:locale_refcounting.obj
 0001:000109a8       __acrt_DownlevelLocaleNameToLCID 00000001800119a8 f   libucrt:lcidtoname_downlevel.obj
 0001:000109f4       __acrt_GetStringTypeA      00000001800119f4 f   libucrt:getstringtypea.obj
 0001:00010f04       __acrt_LCMapStringA        0000000180011f04 f   libucrt:lcmapstringa.obj
 0001:00010f9c       _msize                     0000000180011f9c f   libucrt:msize.obj
 0001:00010fd8       _realloc_base              0000000180011fd8 f   libucrt:realloc_base.obj
 0001:0001105c       __acrt_lowio_create_handle_array 000000018001205c f   libucrt:osfinfo.obj
 0001:000110f4       __acrt_lowio_destroy_handle_array 00000001800120f4 f   libucrt:osfinfo.obj
 0001:00011144       __acrt_lowio_ensure_fh_exists 0000000180012144 f   libucrt:osfinfo.obj
 0001:000111fc       __acrt_lowio_lock_fh       00000001800121fc f   libucrt:osfinfo.obj
 0001:00011220       __acrt_lowio_unlock_fh     0000000180012220 f   libucrt:osfinfo.obj
 0001:00011244       _free_osfhnd               0000000180012244 f   libucrt:osfinfo.obj
 0001:00011300       _get_osfhandle             0000000180012300 f   libucrt:osfinfo.obj
 0001:00011378       _isatty                    0000000180012378 f   libucrt:isatty.obj
 0001:000113d8       __acrt_stdio_flush_nolock  00000001800123d8 f   libucrt:fflush.obj
 0001:00011450       _fflush_nolock             0000000180012450 f   libucrt:fflush.obj
 0001:0001149c       _flushall                  000000018001249c f   libucrt:fflush.obj
 0001:0001158c       _isleadbyte_l              000000018001258c f i libucrt:_wctype.obj
 0001:000115cc       _fcloseall                 00000001800125cc f   libucrt:closeall.obj
 0001:00011680       __acrt_stdio_free_buffer_nolock 0000000180012680 f   libucrt:_freebuf.obj
 0001:000116c0       __acrt_locale_free_monetary 00000001800126c0 f   libucrt:initmon.obj
 0001:000117cc       __acrt_locale_free_numeric 00000001800127cc f   libucrt:initnum.obj
 0001:00011890       __acrt_locale_free_time    0000000180012890 f   libucrt:inittime.obj
 0001:00011998       __strncnt                  0000000180012998 f   libucrt:strncnt.obj
 0001:000119b0       _query_app_type            00000001800129b0 f   libucrt:report_runtime_error.obj
 0001:000119b8       ??$?RV<lambda_b521505b218e5242e90febf6bfebc422>@@AEAV<lambda_6978c1fb23f02e42e1d9e99668cc68aa>@@V<lambda_314360699dd331753a4119843814e9a7>@@@?$__crt_seh_guarded_call@H@@QEAAH$$QEAV<lambda_b521505b218e5242e90febf6bfebc422>@@AEAV<lambda_6978c1fb23f02e42e1d9e99668cc68aa>@@$$QEAV<lambda_314360699dd331753a4119843814e9a7>@@@Z 00000001800129b8 f i libucrt:commit.obj
 0001:00011a44       _commit                    0000000180012a44 f   libucrt:commit.obj
 0001:00012078       _write                     0000000180013078 f   libucrt:write.obj
 0001:00012164       _write_nolock              0000000180013164 f   libucrt:write.obj
 0001:00012450       log10                      0000000180013450 f   libucrt:log10.obj
 0001:00012a98       _lseeki64_nolock           0000000180013a98 f   libucrt:lseek.obj
 0001:00012aa0       _fclose_nolock             0000000180013aa0 f   libucrt:fclose.obj
 0001:00012b24       fclose                     0000000180013b24 f   libucrt:fclose.obj
 0001:00012b90       _putwch_nolock             0000000180013b90 f   libucrt:putwch.obj
 0001:00012d10       _handle_error              0000000180013d10 f   libucrt:libm_error.obj
 0001:00012e40       __acrt_initialize_fma3     0000000180013e40 f   libucrt:fma3_available.obj
 0001:00012eb0       _log10_special             0000000180013eb0 f   libucrt:log_special.obj
 0001:00012f68       ??$?RV<lambda_bfedae4ebbf01fab1bb6dcc6a9e276e0>@@AEAV<lambda_2fe9b910cf3cbf4a0ab98a02ba45b3ec>@@V<lambda_237c231691f317818eb88cc1d5d642d6>@@@?$__crt_seh_guarded_call@H@@QEAAH$$QEAV<lambda_bfedae4ebbf01fab1bb6dcc6a9e276e0>@@AEAV<lambda_2fe9b910cf3cbf4a0ab98a02ba45b3ec>@@$$QEAV<lambda_237c231691f317818eb88cc1d5d642d6>@@@Z 0000000180013f68 f i libucrt:close.obj
 0001:00012fdc       _close                     0000000180013fdc f   libucrt:close.obj
 0001:00013080       _close_nolock              0000000180014080 f   libucrt:close.obj
 0001:0001313c       ?__acrt_stdio_free_stream@@YAXV__crt_stdio_stream@@@Z 000000018001413c f   libucrt:stream.obj
 0001:00013180       __dcrt_lowio_initialize_console_output 0000000180014180 f   libucrt:initcon.obj
 0001:000131bc       __dcrt_terminate_console_output 00000001800141bc f   libucrt:initcon.obj
 0001:000131f0       _get_fpsr                  00000001800141f0 f   libucrt:fpsr.obj
 0001:00013200       _set_fpsr                  0000000180014200 f   libucrt:fpsr.obj
 0001:0001320a       _fclrf                     000000018001420a f   libucrt:fpsr.obj
 0001:0001321e       _frnd                      000000018001421e f   libucrt:fpsr.obj
 0001:00013240       _raise_exc                 0000000180014240 f   libucrt:fpexcept.obj
 0001:00013268       _raise_exc_ex              0000000180014268 f   libucrt:fpexcept.obj
 0001:00013570       _set_errno_from_matherr    0000000180014570 f   libucrt:fpexcept.obj
 0001:000135a0       _clrfp                     00000001800145a0 f   libucrt:fpctrl.obj
 0001:000135c0       _ctrlfp                    00000001800145c0 f   libucrt:fpctrl.obj
 0001:0001363c       _set_statfp                000000018001463c f   libucrt:fpctrl.obj
 0001:0001365c       _statfp                    000000018001465c f   libucrt:fpctrl.obj
 0001:0001366e       IsProcessorFeaturePresent  000000018001466e f   kernel32:KERNEL32.dll
 0001:00013674       RtlUnwindEx                0000000180014674 f   kernel32:KERNEL32.dll
 0001:0001367a       SystemFunction036          000000018001467a f   advapi32:ADVAPI32.dll
 0001:00013680       __GSHandlerCheck           0000000180014680 f   LIBCMT:_gshandler_.obj
 0001:000136a0       __GSHandlerCheckCommon     00000001800146a0 f   LIBCMT:_gshandler_.obj
 0001:00013710       __security_check_cookie    0000000180014710 f   LIBCMT:_amdsecgs_.obj
 0001:00013740       _FindPESection             0000000180014740 f   LIBCMT:pesect.obj
 0001:00013790       _IsNonwritableInCurrentImage 0000000180014790 f   LIBCMT:pesect.obj
 0001:000137e0       _ValidateImageBase         00000001800147e0 f   LIBCMT:pesect.obj
 0001:00013810       __raise_securityfailure    0000000180014810 f   LIBCMT:gs_report.obj
 0001:00013844       __report_gsfailure         0000000180014844 f   LIBCMT:gs_report.obj
 0001:000139a0       memcpy                     00000001800149a0 f   libvcruntime:memcpy.obj
 0001:000139a0       memmove                    00000001800149a0 f   libvcruntime:memcpy.obj
 0001:00013df0       memcmp                     0000000180014df0 f   libvcruntime:memcmp.obj
 0001:00013ed0       _guard_dispatch_icall_nop  0000000180014ed0 f   LIBCMT:_guard_dispatch_.obj
 0001:00014b98       _TI2?AVbad_alloc@std@@     0000000180015b98     LIBCMT:throw_bad_alloc.obj
 0001:00014bb8       _CTA2?AVbad_alloc@std@@    0000000180015bb8     LIBCMT:throw_bad_alloc.obj
 0001:00014bd0       _CT??_R0?AVbad_alloc@std@@@8??0bad_alloc@std@@QEAA@AEBV01@@Z24 0000000180015bd0     LIBCMT:throw_bad_alloc.obj
 0001:00014bf8       _CT??_R0?AVexception@std@@@8??0exception@std@@QEAA@AEBV01@@Z24 0000000180015bf8     LIBCMT:throw_bad_alloc.obj
 0001:00014c20       _TI3?AVbad_array_new_length@std@@ 0000000180015c20     LIBCMT:throw_bad_alloc.obj
 0001:00014c40       _CTA3?AVbad_array_new_length@std@@ 0000000180015c40     LIBCMT:throw_bad_alloc.obj
 0001:00014c60       _CT??_R0?AVbad_array_new_length@std@@@8??0bad_array_new_length@std@@QEAA@AEBV01@@Z24 0000000180015c60     LIBCMT:throw_bad_alloc.obj
 0002:00000070       __scrt_native_dllmain_reason 0000000180016070     LIBCMT:utility.obj
 0002:00000078       __isa_available            0000000180016078     LIBCMT:_cpu_disp_.obj
 0002:0000007c       __isa_enabled              000000018001607c     LIBCMT:_cpu_disp_.obj
 0002:00000080       __memcpy_nt_iters          0000000180016080     LIBCMT:_cpu_disp_.obj
 0002:00000088       __security_cookie          0000000180016088     LIBCMT:gs_cookie.obj
 0002:00000090       __security_cookie_complement 0000000180016090     LIBCMT:gs_cookie.obj
 0002:000000f4       __abort_behavior           00000001800160f4     libucrt:abort.obj
 0002:00000100       __acrt_initial_multibyte_data 0000000180016100     libucrt:mbctype.obj
 0002:00000328       __acrt_current_multibyte_data 0000000180016328     libucrt:mbctype.obj
 0002:00000430       _mbctype                   0000000180016430     libucrt:mbctype.obj
 0002:00000540       _mbcasemap                 0000000180016540     libucrt:mbctype.obj
 0002:00000640       __acrt_initial_locale_data 0000000180016640     libucrt:nlsdata.obj
 0002:00000798       __acrt_initial_locale_pointers 0000000180016798     libucrt:nlsdata.obj
 0002:000007a8       __acrt_wide_c_locale_string 00000001800167a8     libucrt:nlsdata.obj
 0002:000007c0       _iob                       00000001800167c0     libucrt:_file.obj
 0002:000008c8       __globallocalestatus       00000001800168c8     libucrt:glstatus.obj
 0002:000008d0       __acrt_lconv_c             00000001800168d0     libucrt:localeconv.obj
 0002:00000968       __acrt_lconv_static_decimal 0000000180016968     libucrt:localeconv.obj
 0002:0000096c       __acrt_lconv_static_W_decimal 000000018001696c     libucrt:localeconv.obj
 0002:00000970       __dcrt_lowio_console_output_handle 0000000180016970     libucrt:initcon.obj
 0002:00000990       _fltused                   0000000180016990     LIBCMT:fltused.obj
 0002:000009a0       ??_R0?AVbad_alloc@std@@@8  00000001800169a0     LIBCMT:throw_bad_alloc.obj
 0002:000009c8       ??_R0?AVexception@std@@@8  00000001800169c8     LIBCMT:throw_bad_alloc.obj
 0002:000009f0       ??_R0?AVbad_array_new_length@std@@@8 00000001800169f0     LIBCMT:throw_bad_alloc.obj
 0002:00000a20       ??_R0?AVtype_info@@@8      0000000180016a20     LIBCMT:std_type_info_static.obj
 0002:00000c20       __scrt_current_native_startup_state 0000000180016c20     LIBCMT:utility.obj
 0002:00000c28       __scrt_native_startup_lock 0000000180016c28     LIBCMT:utility.obj
 0002:00000c70       ?__type_info_root_node@@3U__type_info_node@@A 0000000180016c70     LIBCMT:tncleanup.obj
 0002:00000c80       ?_OptionsStorage@?1??__local_stdio_printf_options@@9@4_KA 0000000180016c80     LIBCMT:default_local_stdio_options.obj
 0002:00000c88       ?_OptionsStorage@?1??__local_stdio_scanf_options@@9@4_KA 0000000180016c88     LIBCMT:default_local_stdio_options.obj
 0002:00000c90       __scrt_debugger_hook_flag  0000000180016c90     LIBCMT:utility_desktop.obj
 0002:00000c94       __favor                    0000000180016c94     LIBCMT:_cpu_disp_.obj
 0002:00000db8       __pPurecall                0000000180016db8     libvcruntime:purevirt_data.obj
 0002:00000dc0       ?pArgList@UnDecorator@@0PEAVReplicator@@EA 0000000180016dc0     libvcruntime:undname.obj
 0002:00000dc8       ?pZNameList@UnDecorator@@0PEAVReplicator@@EA 0000000180016dc8     libvcruntime:undname.obj
 0002:00000dd0       ?pTemplateArgList@UnDecorator@@0PEAVReplicator@@EA 0000000180016dd0     libvcruntime:undname.obj
 0002:00000dd8       ?gName@UnDecorator@@0PEBDEB 0000000180016dd8     libvcruntime:undname.obj
 0002:00000de0       ?name@UnDecorator@@0PEBDEB 0000000180016de0     libvcruntime:undname.obj
 0002:00000de8       ?outputString@UnDecorator@@0PEADEA 0000000180016de8     libvcruntime:undname.obj
 0002:00000df0       ?maxStringLength@UnDecorator@@0HA 0000000180016df0     libvcruntime:undname.obj
 0002:00000df4       ?disableFlags@UnDecorator@@0KA 0000000180016df4     libvcruntime:undname.obj
 0002:00000df8       ?fExplicitTemplateParams@UnDecorator@@0_NA 0000000180016df8     libvcruntime:undname.obj
 0002:00000df9       ?fGetTemplateArgumentList@UnDecorator@@0_NA 0000000180016df9     libvcruntime:undname.obj
 0002:00000e00       ?m_pGetParameter@UnDecorator@@0P6APEADJ@ZEA 0000000180016e00     libvcruntime:undname.obj
 0002:00000e50       _environ_table             0000000180016e50     libucrt:environment_initialization.obj
 0002:00000e58       _wenviron_table            0000000180016e58     libucrt:environment_initialization.obj
 0002:00000e60       __dcrt_initial_wide_environment 0000000180016e60     libucrt:environment_initialization.obj
 0002:00000e68       __dcrt_initial_narrow_environment 0000000180016e68     libucrt:environment_initialization.obj
 0002:00000e70       __acrt_atexit_table        0000000180016e70     libucrt:onexit.obj
 0002:00000e88       __acrt_at_quick_exit_table 0000000180016e88     libucrt:onexit.obj
 0002:00001260       __mbcodepage               0000000180017260     libucrt:mbctype.obj
 0002:00001264       __ismbcodepage             0000000180017264     libucrt:mbctype.obj
 0002:00001268       __mbulinfo                 0000000180017268     libucrt:mbctype.obj
 0002:00001278       __mblocalename             0000000180017278     libucrt:mbctype.obj
 0002:00001288       __acrt_heap                0000000180017288     libucrt:heap_handle.obj
 0002:00001290       __pioinfo                  0000000180017290     libucrt:ioinit.obj
 0002:00001690       _nhandle                   0000000180017690     libucrt:ioinit.obj
 0002:00001698       __argv                     0000000180017698     libucrt:argv_data.obj
 0002:000016a0       __wargv                    00000001800176a0     libucrt:argv_data.obj
 0002:000016a8       _acmdln                    00000001800176a8     libucrt:argv_data.obj
 0002:000016b0       _wcmdln                    00000001800176b0     libucrt:argv_data.obj
 0002:000016e0       __acrt_current_locale_data 00000001800176e0     libucrt:nlsdata.obj
 0002:000016e8       __acrt_stdout_buffer       00000001800176e8     libucrt:_sftbuf.obj
 0002:000016f0       __acrt_stderr_buffer       00000001800176f0     libucrt:_sftbuf.obj
 0002:00001700       _nstream                   0000000180017700     libucrt:_file.obj
 0002:00001708       __piob                     0000000180017708     libucrt:_file.obj
 0002:00001710       __acrt_locale_changed_data 0000000180017710     libucrt:wsetlocale.obj
 0002:00001714       __acrt_lconv_static_null   0000000180017714     libucrt:localeconv.obj
 0002:00001718       __acrt_lconv_static_W_null 0000000180017718     libucrt:localeconv.obj
 0002:00001720       __fma3_is_available        0000000180017720     libucrt:fma3_available.obj
 0002:00001724       __use_fma3_lib             0000000180017724     libucrt:fma3_available.obj
 0002:00001ca0       __scrt_ucrt_dll_is_in_use  0000000180017ca0     <common>
 0002:00001ca8       __dyn_tls_init_callback    0000000180017ca8     <common>
 0002:00001cb0       _pDestructExceptionObject  0000000180017cb0     <common>
 0004:00000000       __imp_SystemFunction036    0000000180019000     advapi32:ADVAPI32.dll
 0004:00000008       \177ADVAPI32_NULL_THUNK_DATA 0000000180019008     advapi32:ADVAPI32.dll
 0004:00000010       __imp_lstrlenW             0000000180019010     kernel32:KERNEL32.dll
 0004:00000018       __imp_lstrcpynW            0000000180019018     kernel32:KERNEL32.dll
 0004:00000020       __imp_CreateFileW          0000000180019020     kernel32:KERNEL32.dll
 0004:00000028       __imp_QueryPerformanceCounter 0000000180019028     kernel32:KERNEL32.dll
 0004:00000030       __imp_GetCurrentProcessId  0000000180019030     kernel32:KERNEL32.dll
 0004:00000038       __imp_GetCurrentThreadId   0000000180019038     kernel32:KERNEL32.dll
 0004:00000040       __imp_GetSystemTimeAsFileTime 0000000180019040     kernel32:KERNEL32.dll
 0004:00000048       __imp_InitializeSListHead  0000000180019048     kernel32:KERNEL32.dll
 0004:00000050       __imp_RtlCaptureContext    0000000180019050     kernel32:KERNEL32.dll
 0004:00000058       __imp_RtlLookupFunctionEntry 0000000180019058     kernel32:KERNEL32.dll
 0004:00000060       __imp_RtlVirtualUnwind     0000000180019060     kernel32:KERNEL32.dll
 0004:00000068       __imp_IsDebuggerPresent    0000000180019068     kernel32:KERNEL32.dll
 0004:00000070       __imp_UnhandledExceptionFilter 0000000180019070     kernel32:KERNEL32.dll
 0004:00000078       __imp_SetUnhandledExceptionFilter 0000000180019078     kernel32:KERNEL32.dll
 0004:00000080       __imp_GetStartupInfoW      0000000180019080     kernel32:KERNEL32.dll
 0004:00000088       __imp_IsProcessorFeaturePresent 0000000180019088     kernel32:KERNEL32.dll
 0004:00000090       __imp_GetModuleHandleW     0000000180019090     kernel32:KERNEL32.dll
 0004:00000098       __imp_GetLastError         0000000180019098     kernel32:KERNEL32.dll
 0004:000000a0       __imp_GetModuleFileNameW   00000001800190a0     kernel32:KERNEL32.dll
 0004:000000a8       __imp_RtlUnwindEx          00000001800190a8     kernel32:KERNEL32.dll
 0004:000000b0       __imp_RtlPcToFileHeader    00000001800190b0     kernel32:KERNEL32.dll
 0004:000000b8       __imp_RaiseException       00000001800190b8     kernel32:KERNEL32.dll
 0004:000000c0       __imp_InterlockedFlushSList 00000001800190c0     kernel32:KERNEL32.dll
 0004:000000c8       __imp_InitializeCriticalSectionAndSpinCount 00000001800190c8     kernel32:KERNEL32.dll
 0004:000000d0       __imp_TlsAlloc             00000001800190d0     kernel32:KERNEL32.dll
 0004:000000d8       __imp_TlsGetValue          00000001800190d8     kernel32:KERNEL32.dll
 0004:000000e0       __imp_TlsSetValue          00000001800190e0     kernel32:KERNEL32.dll
 0004:000000e8       __imp_TlsFree              00000001800190e8     kernel32:KERNEL32.dll
 0004:000000f0       __imp_FreeLibrary          00000001800190f0     kernel32:KERNEL32.dll
 0004:000000f8       __imp_GetProcAddress       00000001800190f8     kernel32:KERNEL32.dll
 0004:00000100       __imp_LoadLibraryExW       0000000180019100     kernel32:KERNEL32.dll
 0004:00000108       __imp_SetLastError         0000000180019108     kernel32:KERNEL32.dll
 0004:00000110       __imp_EnterCriticalSection 0000000180019110     kernel32:KERNEL32.dll
 0004:00000118       __imp_LeaveCriticalSection 0000000180019118     kernel32:KERNEL32.dll
 0004:00000120       __imp_DeleteCriticalSection 0000000180019120     kernel32:KERNEL32.dll
 0004:00000128       __imp_GetCurrentProcess    0000000180019128     kernel32:KERNEL32.dll
 0004:00000130       __imp_ExitProcess          0000000180019130     kernel32:KERNEL32.dll
 0004:00000138       __imp_TerminateProcess     0000000180019138     kernel32:KERNEL32.dll
 0004:00000140       __imp_GetModuleHandleExW   0000000180019140     kernel32:KERNEL32.dll
 0004:00000148       __imp_MultiByteToWideChar  0000000180019148     kernel32:KERNEL32.dll
 0004:00000150       __imp_WideCharToMultiByte  0000000180019150     kernel32:KERNEL32.dll
 0004:00000158       __imp_HeapFree             0000000180019158     kernel32:KERNEL32.dll
 0004:00000160       __imp_HeapAlloc            0000000180019160     kernel32:KERNEL32.dll
 0004:00000168       __imp_LCMapStringW         0000000180019168     kernel32:KERNEL32.dll
 0004:00000170       __imp_IsValidCodePage      0000000180019170     kernel32:KERNEL32.dll
 0004:00000178       __imp_GetACP               0000000180019178     kernel32:KERNEL32.dll
 0004:00000180       __imp_GetOEMCP             0000000180019180     kernel32:KERNEL32.dll
 0004:00000188       __imp_GetCPInfo            0000000180019188     kernel32:KERNEL32.dll
 0004:00000190       __imp_GetEnvironmentStringsW 0000000180019190     kernel32:KERNEL32.dll
 0004:00000198       __imp_FreeEnvironmentStringsW 0000000180019198     kernel32:KERNEL32.dll
 0004:000001a0       __imp_GetProcessHeap       00000001800191a0     kernel32:KERNEL32.dll
 0004:000001a8       __imp_GetStdHandle         00000001800191a8     kernel32:KERNEL32.dll
 0004:000001b0       __imp_GetFileType          00000001800191b0     kernel32:KERNEL32.dll
 0004:000001b8       __imp_GetCommandLineA      00000001800191b8     kernel32:KERNEL32.dll
 0004:000001c0       __imp_GetCommandLineW      00000001800191c0     kernel32:KERNEL32.dll
 0004:000001c8       __imp_GetStringTypeW       00000001800191c8     kernel32:KERNEL32.dll
 0004:000001d0       __imp_HeapSize             00000001800191d0     kernel32:KERNEL32.dll
 0004:000001d8       __imp_HeapReAlloc          00000001800191d8     kernel32:KERNEL32.dll
 0004:000001e0       __imp_SetStdHandle         00000001800191e0     kernel32:KERNEL32.dll
 0004:000001e8       __imp_WriteFile            00000001800191e8     kernel32:KERNEL32.dll
 0004:000001f0       __imp_FlushFileBuffers     00000001800191f0     kernel32:KERNEL32.dll
 0004:000001f8       __imp_GetConsoleCP         00000001800191f8     kernel32:KERNEL32.dll
 0004:00000200       __imp_GetConsoleMode       0000000180019200     kernel32:KERNEL32.dll
 0004:00000208       __imp_SetFilePointerEx     0000000180019208     kernel32:KERNEL32.dll
 0004:00000210       __imp_CloseHandle          0000000180019210     kernel32:KERNEL32.dll
 0004:00000218       __imp_WriteConsoleW        0000000180019218     kernel32:KERNEL32.dll
 0004:00000220       __imp_lstrcmpiW            0000000180019220     kernel32:KERNEL32.dll
 0004:00000228       \177KERNEL32_NULL_THUNK_DATA 0000000180019228     kernel32:KERNEL32.dll
 0004:00000230       __imp_MessageBeep          0000000180019230     user32:USER32.dll
 0004:00000238       \177USER32_NULL_THUNK_DATA 0000000180019238     user32:USER32.dll
 0004:00000240       __IMPORT_DESCRIPTOR_KERNEL32 0000000180019240     kernel32:KERNEL32.dll
 0004:00000254       __IMPORT_DESCRIPTOR_USER32 0000000180019254     user32:USER32.dll
 0004:00000268       __IMPORT_DESCRIPTOR_ADVAPI32 0000000180019268     advapi32:ADVAPI32.dll
 0004:0000027c       __NULL_IMPORT_DESCRIPTOR   000000018001927c     kernel32:KERNEL32.dll

 entry point at        0001:0000b250

 Static symbols

 0001:00000500       ?ExceptionTemplate@?1??_CxxThrowException@@9@4UEHExceptionRecord@@B 0000000180001500     libvcruntime:throw.obj
 0001:00000540       ?module_names@?A0x61ce2399@@3QBQEB_WB 0000000180001540     libvcruntime:winapi_downlevel.obj
 0001:0000060c       ?candidate_modules@?1??try_get_EventRegister@@YAP6AKPEBU_GUID@@P6AX0KE_K1PEAU_EVENT_FILTER_DESCRIPTOR@@PEAX@Z3PEA_K@ZXZ@4QBW4module_id@?A0x61ce2399@@B 000000018000160c     libvcruntime:winapi_downlevel.obj
 0001:00000620       ?candidate_modules@?1??try_get_EventSetInformation@@YAP6AK_KW4_EVENT_INFO_CLASS@@PEAXK@ZXZ@4QBW4module_id@?A0x61ce2399@@B 0000000180001620     libvcruntime:winapi_downlevel.obj
 0001:0000063c       ?candidate_modules@?1??try_get_EventUnregister@@YAP6AK_K@ZXZ@4QBW4module_id@?A0x61ce2399@@B 000000018000163c     libvcruntime:winapi_downlevel.obj
 0001:00000650       ?candidate_modules@?1??try_get_EventWriteTransfer@@YAP6AK_KPEBU_EVENT_DESCRIPTOR@@PEBU_GUID@@2KPEAU_EVENT_DATA_DESCRIPTOR@@@ZXZ@4QBW4module_id@?A0x61ce2399@@B 0000000180001650     libvcruntime:winapi_downlevel.obj
 0001:00000670       ?candidate_modules@?1??try_get_FlsAlloc@@YAP6AKP6AXPEAX@Z@ZXZ@4QBW4module_id@?A0x61ce2399@@B 0000000180001670     libvcruntime:winapi_downlevel.obj
 0001:00000688       ?candidate_modules@?1??try_get_FlsFree@@YAP6AHK@ZXZ@4QBW4module_id@?A0x61ce2399@@B 0000000180001688     libvcruntime:winapi_downlevel.obj
 0001:00000698       ?candidate_modules@?1??try_get_FlsGetValue@@YAP6APEAXK@ZXZ@4QBW4module_id@?A0x61ce2399@@B 0000000180001698     libvcruntime:winapi_downlevel.obj
 0001:000006b0       ?candidate_modules@?1??try_get_FlsSetValue@@YAP6AHKPEAX@ZXZ@4QBW4module_id@?A0x61ce2399@@B 00000001800016b0     libvcruntime:winapi_downlevel.obj
 0001:000006c8       ?candidate_modules@?1??try_get_InitializeCriticalSectionEx@@YAP6AHPEAU_RTL_CRITICAL_SECTION@@KK@ZXZ@4QBW4module_id@?A0x61ce2399@@B 00000001800016c8     libvcruntime:winapi_downlevel.obj
 0001:00000bb0       ?rttiTable@@3QBQEBDB       0000000180001bb0     libvcruntime:undname.obj
 0001:00000be0       ?tokenTable@@3QBQEBDB      0000000180001be0     libvcruntime:undname.obj
 0001:00000c50       ?nameTable@@3QBQEBDB       0000000180001c50     libvcruntime:undname.obj
 0001:00001170       __acrt_initializers        0000000180002170     libucrt:initialization.obj
 0001:00001260       module_names               0000000180002260     libucrt:winapi_thunks.obj
 0001:00001790       ?candidate_modules@?1??try_get_FlsAlloc@@YAP6AKP6AXPEAX@Z@ZXZ@4QBW4module_id@?A0x63058377@@B 0000000180002790     libucrt:winapi_thunks.obj
 0001:00001798       ?candidate_modules@?1??try_get_FlsFree@@YAP6AHK@ZXZ@4QBW4module_id@?A0x63058377@@B 0000000180002798     libucrt:winapi_thunks.obj
 0001:000017a0       ?candidate_modules@?1??try_get_FlsGetValue@@YAP6APEAXK@ZXZ@4QBW4module_id@?A0x63058377@@B 00000001800027a0     libucrt:winapi_thunks.obj
 0001:000017a8       ?candidate_modules@?1??try_get_FlsSetValue@@YAP6AHKPEAX@ZXZ@4QBW4module_id@?A0x63058377@@B 00000001800027a8     libucrt:winapi_thunks.obj
 0001:000017b0       ?candidate_modules@?1??try_get_GetCurrentPackageId@@YAP6AJPEAIPEAE@ZXZ@4QBW4module_id@?A0x63058377@@B 00000001800027b0     libucrt:winapi_thunks.obj
 0001:000017d0       ?candidate_modules@?1??try_get_InitializeCriticalSectionEx@@YAP6AHPEAU_RTL_CRITICAL_SECTION@@KK@ZXZ@4QBW4module_id@?A0x63058377@@B 00000001800027d0     libucrt:winapi_thunks.obj
 0001:000017d8       ?candidate_modules@?1??try_get_LCMapStringEx@@YAP6AHPEB_WK0HPEA_WHPEAU_nlsversioninfo@@PEAX_J@ZXZ@4QBW4module_id@?A0x63058377@@B 00000001800027d8     libucrt:winapi_thunks.obj
 0001:000017f0       ?candidate_modules@?1??try_get_LocaleNameToLCID@@YAP6AKPEB_WK@ZXZ@4QBW4module_id@?A0x63058377@@B 00000001800027f0     libucrt:winapi_thunks.obj
 0001:00001810       _mb_locale_names           0000000180002810     libucrt:mbctype.obj
 0001:00001ef0       errtable                   0000000180002ef0     libucrt:errno.obj
 0001:00002660       LcidToLocaleNameTable      0000000180003660     libucrt:lcidtoname_downlevel.obj
 0001:000040c0       LocaleNameToIndexTable     00000001800050c0     libucrt:lcidtoname_downlevel.obj
 0001:00005960       __real_ninf                0000000180006960     libucrt:log10.obj
 0001:00005970       __real_inf                 0000000180006970     libucrt:log10.obj
 0001:00005980       __real_neg_qnan            0000000180006980     libucrt:log10.obj
 0001:00005990       __real_qnanbit             0000000180006990     libucrt:log10.obj
 0001:000059a0       __int_1023                 00000001800069a0     libucrt:log10.obj
 0001:000059b0       __mask_001                 00000001800069b0     libucrt:log10.obj
 0001:000059c0       __mask_mant                00000001800069c0     libucrt:log10.obj
 0001:000059d0       __mask_mant_top8           00000001800069d0     libucrt:log10.obj
 0001:000059e0       __mask_mant9               00000001800069e0     libucrt:log10.obj
 0001:000059f0       __real_log10_e             00000001800069f0     libucrt:log10.obj
 0001:00005a00       __real_log10_e_lead        0000000180006a00     libucrt:log10.obj
 0001:00005a10       __real_log10_e_tail        0000000180006a10     libucrt:log10.obj
 0001:00005a20       __real_log10_2_lead        0000000180006a20     libucrt:log10.obj
 0001:00005a30       __real_log10_2_tail        0000000180006a30     libucrt:log10.obj
 0001:00005a40       __real_two                 0000000180006a40     libucrt:log10.obj
 0001:00005a50       __real_one                 0000000180006a50     libucrt:log10.obj
 0001:00005a60       __real_half                0000000180006a60     libucrt:log10.obj
 0001:00005a70       __mask_100                 0000000180006a70     libucrt:log10.obj
 0001:00005a80       __real_1_over_512          0000000180006a80     libucrt:log10.obj
 0001:00005a90       __real_1_over_2            0000000180006a90     libucrt:log10.obj
 0001:00005aa0       __real_1_over_3            0000000180006aa0     libucrt:log10.obj
 0001:00005ab0       __real_1_over_4            0000000180006ab0     libucrt:log10.obj
 0001:00005ac0       __real_1_over_5            0000000180006ac0     libucrt:log10.obj
 0001:00005ad0       __real_1_over_6            0000000180006ad0     libucrt:log10.obj
 0001:00005ae0       __real_neg_1023            0000000180006ae0     libucrt:log10.obj
 0001:00005af0       __mask_2045                0000000180006af0     libucrt:log10.obj
 0001:00005b00       __real_threshold           0000000180006b00     libucrt:log10.obj
 0001:00005b10       __real_near_one_lt         0000000180006b10     libucrt:log10.obj
 0001:00005b20       __real_near_one_gt         0000000180006b20     libucrt:log10.obj
 0001:00005b30       __real_min_norm            0000000180006b30     libucrt:log10.obj
 0001:00005b40       __real_notsign             0000000180006b40     libucrt:log10.obj
 0001:00005b50       __real_ca1                 0000000180006b50     libucrt:log10.obj
 0001:00005b60       __real_ca2                 0000000180006b60     libucrt:log10.obj
 0001:00005b70       __real_ca3                 0000000180006b70     libucrt:log10.obj
 0001:00005b80       __real_ca4                 0000000180006b80     libucrt:log10.obj
 0001:00005b90       __mask_lower               0000000180006b90     libucrt:log10.obj
 0001:00005ba0       __flag_x_zero              0000000180006ba0     libucrt:log10.obj
 0001:00005ba4       __flag_x_neg               0000000180006ba4     libucrt:log10.obj
 0001:00005ba8       __flag_x_nan               0000000180006ba8     libucrt:log10.obj
 0001:00007400       __real@433fffffffffffff    0000000180008400     libucrt:fpsr.obj
 0001:00007408       __real@c33fffffffffffff    0000000180008408     libucrt:fpsr.obj
 0001:00007410       GS_ExceptionPointers       0000000180008410     LIBCMT:gs_report.obj
 0001:000076e0       ?_TlgEvent@?3??__telemetry_main_invoke_trigger@@9@4U<unnamed-type-_TlgEvent>@?3??1@YAXQEAUHINSTANCE__@@@Z@B 00000001800086e0     libvcruntime:telemetry.obj
 0001:0000771c       ?_TlgEvent@?3??__telemetry_main_return_trigger@@9@4U<unnamed-type-_TlgEvent>@?3??1@YAXQEAUHINSTANCE__@@@Z@B 000000018000871c     libvcruntime:telemetry.obj
 0001:00007757       ?_Tlg_Microsoft_CRTProviderProv_Meta@@3U<unnamed-type-_Tlg_Microsoft_CRTProviderProv_Meta>@@B 0000000180008757     libvcruntime:telemetry.obj
 0001:00007cd0       $$000000                   0000000180008cd0     chkstk.obj
 0001:00009450       $LN313                     000000018000a450     Brackets.obj
 0001:00009480       $LN312                     000000018000a480     Brackets.obj
 0001:000094b0       $LN311                     000000018000a4b0     Brackets.obj
 0001:000094e0       $LN310                     000000018000a4e0     Brackets.obj
 0001:00009510       $LN309                     000000018000a510     Brackets.obj
 0001:000097a4       $LN10                      000000018000a7a4     Brackets.obj
 0001:000098d8       $LN22                      000000018000a8d8     Brackets.obj
 0001:0000aef4       ?dllmain_crt_dispatch@@YAHQEAUHINSTANCE__@@KQEAX@Z 000000018000bef4 f   LIBCMT:dll_dllmain.obj
 0001:0000af44       ?dllmain_crt_process_attach@@YAHQEAUHINSTANCE__@@QEAX@Z 000000018000bf44 f   LIBCMT:dll_dllmain.obj
 0001:0000b070       ?dllmain_crt_process_detach@@YAH_N@Z 000000018000c070 f   LIBCMT:dll_dllmain.obj
 0001:0000b0f4       ?dllmain_dispatch@@YAHQEAUHINSTANCE__@@KQEAX@Z 000000018000c0f4 f   LIBCMT:dll_dllmain.obj
 0001:0000b1fc       ?dllmain_raw@@YAHQEAUHINSTANCE__@@KQEAX@Z 000000018000c1fc f   LIBCMT:dll_dllmain.obj
 0001:0000bd00       $$000000                   000000018000cd00     libvcruntime:memset.obj
 0001:0000bdec       MsetTab                    000000018000cdec     libvcruntime:memset.obj
 0001:0000beb0       _TlgDefineProvider_annotation__Tlg_Microsoft_CRTProviderProv 000000018000ceb0 f   libvcruntime:telemetry.obj
 0001:0000c560       ?try_get_function@@YAPEAXW4function_id@?A0x61ce2399@@QEBDQEBW4module_id@2@2@Z 000000018000d560 f   libvcruntime:winapi_downlevel.obj
 0001:0000cb70       $$000000                   000000018000db70     libvcruntime:_jmpuwind_.obj
 0001:0000d108       ?atexit_exception_filter@@YAHK@Z 000000018000e108 f   libucrt:exit.obj
 0001:0000d114       ?common_exit@@YAXHW4_crt_exit_cleanup_mode@@W4_crt_exit_return_mode@@@Z 000000018000e114 f   libucrt:exit.obj
 0001:0000d280       ?exit_or_terminate_process@@YAXI@Z 000000018000e280 f   libucrt:exit.obj
 0001:0000d2cc       ?try_cor_exit_process@@YAXI@Z 000000018000e2cc f   libucrt:exit.obj
 0001:0000d364       ??$common_initialize_environment_nolock@D@@YAHXZ 000000018000e364 f   libucrt:environment_initialization.obj
 0001:0000d3d0       ??$create_environment@D@@YAQEAPEADQEAD@Z 000000018000e3d0 f   libucrt:environment_initialization.obj
 0001:0000d4cc       ??$free_environment@D@@YAXQEAPEAD@Z 000000018000e4cc f   libucrt:environment_initialization.obj
 0001:0000d4cc       ??$free_environment@_W@@YAXQEAPEA_W@Z 000000018000e4cc f   libucrt:environment_initialization.obj
 0001:0000d510       ??$uninitialize_environment_internal@D@@YAXAEAPEAPEAD@Z 000000018000e510 f   libucrt:environment_initialization.obj
 0001:0000d52c       ??$uninitialize_environment_internal@_W@@YAXAEAPEAPEA_W@Z 000000018000e52c f   libucrt:environment_initialization.obj
 0001:0000d764       ??R<lambda_4e60a939b0d047cfe11ddc22648dfba9>@@QEBAHXZ 000000018000e764 f   libucrt:onexit.obj
 0001:0000da14       initialize_global_variables 000000018000ea14 f   libucrt:initialization.obj
 0001:0000da28       initialize_c               000000018000ea28 f   libucrt:initialization.obj
 0001:0000da4c       initialize_environment     000000018000ea4c f   libucrt:initialization.obj
 0001:0000da4c       uninitialize_c             000000018000ea4c f   libucrt:initialization.obj
 0001:0000da4c       initialize_global_state_isolation 000000018000ea4c f   libucrt:initialization.obj
 0001:0000da4c       uninitialize_global_state_isolation 000000018000ea4c f   libucrt:initialization.obj
 0001:0000da4c       report_memory_leaks        000000018000ea4c f   libucrt:initialization.obj
 0001:0000da50       uninitialize_environment   000000018000ea50 f   libucrt:initialization.obj
 0001:0000da60       initialize_pointers        000000018000ea60 f   libucrt:initialization.obj
 0001:0000dab4       uninitialize_vcruntime     000000018000eab4 f   libucrt:initialization.obj
 0001:0000dabc       uninitialize_allocated_memory 000000018000eabc f   libucrt:initialization.obj
 0001:0000e010       ?construct_ptd_array@@YAXQEAU__acrt_ptd@@@Z 000000018000f010 f   libucrt:per_thread_data.obj
 0001:0000e0e0       ?destroy_fls@@YAXPEAX@Z    000000018000f0e0 f   libucrt:per_thread_data.obj
 0001:0000e100       ?destroy_ptd_array@@YAXQEAU__acrt_ptd@@@Z 000000018000f100 f   libucrt:per_thread_data.obj
 0001:0000e1f8       ?replace_current_thread_locale_nolock@@YAXQEAU__acrt_ptd@@QEAU__crt_locale_data@@@Z 000000018000f1f8 f   libucrt:per_thread_data.obj
 0001:0000e438       ?try_get_function@@YAPEAXW4function_id@?A0x63058377@@QEBDQEBW4module_id@2@2@Z 000000018000f438 f   libucrt:winapi_thunks.obj
 0001:0000ecc8       ??R<lambda_ad1ced32f4ac17aa236e5ef05d6b3b7c>@@QEBAXXZ 000000018000fcc8 f   libucrt:mbctype.obj
 0001:0000eee0       ?getSystemCP@@YAHH@Z       000000018000fee0 f   libucrt:mbctype.obj
 0001:0000ef60       ?setSBCS@@YAXPEAU__crt_multibyte_data@@@Z 000000018000ff60 f   libucrt:mbctype.obj
 0001:0000eff0       ?setSBUpLow@@YAXPEAU__crt_multibyte_data@@@Z 000000018000fff0 f   libucrt:mbctype.obj
 0001:0000f1d4       ?setmbcp_internal@@YAHH_N@Z 00000001800101d4 f   libucrt:mbctype.obj
 0001:0000f8e8       ?initialize_inherited_file_handles_nolock@@YAXXZ 00000001800108e8 f   libucrt:ioinit.obj
 0001:0000f9d4       ?initialize_stdio_handles_nolock@@YAXXZ 00000001800109d4 f   libucrt:ioinit.obj
 0001:000108e0       ?GetTableIndexFromLocaleName@@YAHPEB_W@Z 00000001800118e0 f   libucrt:lcidtoname_downlevel.obj
 0001:000109dc       ?initialize_multibyte@@YAHXZ 00000001800119dc f   libucrt:multibyte_initializer.obj
 0001:00010ba8       ?__acrt_LCMapStringA_stat@@YAHPEAU__crt_locale_pointers@@PEB_WKPEBDHPEADHHH@Z 0000000180011ba8 f   libucrt:lcmapstringa.obj
 0001:000114a8       common_flush_all           00000001800124a8 f   libucrt:fflush.obj
 0001:00011838       ?free_crt_array_internal@@YAXQEAPEBX_K@Z 0000000180012838 f   libucrt:inittime.obj
 0001:00011ad8       ?write_double_translated_ansi_nolock@@YA?AUwrite_result@?A0x9c548279@@HQEBDI@Z 0000000180012ad8 f   libucrt:write.obj
 0001:00011ce0       ?write_text_ansi_nolock@@YA?AUwrite_result@?A0x9c548279@@HQEBDI@Z 0000000180012ce0 f   libucrt:write.obj
 0001:00011de8       ?write_text_utf16le_nolock@@YA?AUwrite_result@?A0x9c548279@@HQEBDI@Z 0000000180012de8 f   libucrt:write.obj
 0001:00011f04       ?write_text_utf8_nolock@@YA?AUwrite_result@?A0x9c548279@@HQEBDI@Z 0000000180012f04 f   libucrt:write.obj
 0001:00012450       $$000000                   0000000180013450     libucrt:log10.obj
 0001:000129fc       ??$common_lseek_nolock@_J@@YA_JH_JH@Z 00000001800139fc f   libucrt:lseek.obj
 0001:00012bec       _call_matherr              0000000180013bec f   libucrt:libm_error.obj
 0001:00012c54       _exception_enabled         0000000180013c54 f   libucrt:libm_error.obj
 0001:00012ed0       _log_special_common        0000000180013ed0 f   libucrt:log_special.obj
 0001:000131e0       $$000000                   00000001800141e0     libucrt:fpsr.obj
 0001:00013700       $$000000                   0000000180014700     LIBCMT:_amdsecgs_.obj
 0001:00013918       capture_previous_context   0000000180014918 f   LIBCMT:gs_report.obj
 0001:00013990       $$000000                   0000000180014990     libvcruntime:memcpy.obj
 0001:00013a37       MoveSmall                  0000000180014a37     libvcruntime:memcpy.obj
 0001:00013de0       $$000000                   0000000180014de0     libvcruntime:memcmp.obj
 0001:00013ec0       $$000000                   0000000180014ec0     LIBCMT:_guard_dispatch_.obj
 0001:00013ee0       ?fin$0@?0??dllmain_crt_process_attach@@YAHQEAUHINSTANCE__@@QEAX@Z@4HA 0000000180014ee0 f   LIBCMT:dll_dllmain.obj
 0001:00013ef7       ?fin$0@?0??dllmain_crt_process_detach@@YAH_N@Z@4HA 0000000180014ef7 f   LIBCMT:dll_dllmain.obj
 0001:00013f13       ?filt$0@?0??dllmain_dispatch@@YAHQEAUHINSTANCE__@@KQEAX@Z@4HA 0000000180014f13 f   LIBCMT:dll_dllmain.obj
 0001:00013f49       __scrt_is_nonwritable_in_current_image$filt$0 0000000180014f49 f   LIBCMT:utility.obj
 0001:00013f61       _query_new_handler$fin$0   0000000180014f61 f   libucrt:new_handler.obj
 0001:00013f77       ?filt$0@?0??common_exit@@YAXHW4_crt_exit_cleanup_mode@@W4_crt_exit_return_mode@@@Z@4HA 0000000180014f77 f   libucrt:exit.obj
 0001:00013f92       ?fin$1@?0??common_exit@@YAXHW4_crt_exit_cleanup_mode@@W4_crt_exit_return_mode@@@Z@4HA 0000000180014f92 f   libucrt:exit.obj
 0001:00013fab       ?fin$0@?0???$?RV<lambda_e24bbb7b643b32fcea6fa61b31d4c984>@@AEAV<lambda_275893d493268fdec8709772e3fcec0e>@@V<lambda_9d71df4d7cf3f480f8d633942495c3b0>@@@?$__crt_seh_guarded_call@H@@QEAAH$$QEAV<lambda_e24bbb7b643b32fcea6fa61b31d4c984>@@AEAV<lambda_275893d493268fdec8709772e3fcec0e>@@$$QEAV<lambda_9d71df4d7cf3f480f8d633942495c3b0>@@@Z@4HA 0000000180014fab f   libucrt:onexit.obj
 0001:00013fc8       ?fin$0@?0???$?RV<lambda_c36588078e9f5dfd39652860aa6b3aaf>@@AEAV<lambda_ec61778202f4f5fc7e7711acc23c3bca>@@V<lambda_dc9d2797ccde5d239b4a0efae8ebd7db>@@@?$__crt_seh_guarded_call@P6AXH@Z@@QEAAP6AXH@Z$$QEAV<lambda_c36588078e9f5dfd39652860aa6b3aaf>@@AEAV<lambda_ec61778202f4f5fc7e7711acc23c3bca>@@$$QEAV<lambda_dc9d2797ccde5d239b4a0efae8ebd7db>@@@Z@4HA 0000000180014fc8 f   libucrt:signal.obj
 0001:00013fc8       ?fin$0@?0???$?RV<lambda_fb3a7dec4e47f37f22dae91bb15c9095>@@AEAV<lambda_698284760c8add0bfb0756c19673e34b>@@V<lambda_dfb8eca1e75fef3034a8fb18dd509707>@@@?$__crt_seh_guarded_call@X@@QEAAX$$QEAV<lambda_fb3a7dec4e47f37f22dae91bb15c9095>@@AEAV<lambda_698284760c8add0bfb0756c19673e34b>@@$$QEAV<lambda_dfb8eca1e75fef3034a8fb18dd509707>@@@Z@4HA 0000000180014fc8 f   libucrt:per_thread_data.obj
 0001:00013fc8       ?fin$0@?0???$?RV<lambda_72d1df2b273a38828b1ce30cbf4cdab5>@@AEAV<lambda_876a65b173b8412d3a47c70a915b0cf4>@@V<lambda_41932305e351933ebe8f8be3ed8bb5dc>@@@?$__crt_seh_guarded_call@X@@QEAAX$$QEAV<lambda_72d1df2b273a38828b1ce30cbf4cdab5>@@AEAV<lambda_876a65b173b8412d3a47c70a915b0cf4>@@$$QEAV<lambda_41932305e351933ebe8f8be3ed8bb5dc>@@@Z@4HA 0000000180014fc8 f   libucrt:per_thread_data.obj
 0001:00013fc8       ?fin$0@?0???$?RV<lambda_b8c45f8f788dd370798f47cfe8ac3a86>@@AEAV<lambda_4e60a939b0d047cfe11ddc22648dfba9>@@V<lambda_332c3edc96d0294ec56c57d38c1cdfd5>@@@?$__crt_seh_guarded_call@H@@QEAAH$$QEAV<lambda_b8c45f8f788dd370798f47cfe8ac3a86>@@AEAV<lambda_4e60a939b0d047cfe11ddc22648dfba9>@@$$QEAV<lambda_332c3edc96d0294ec56c57d38c1cdfd5>@@@Z@4HA 0000000180014fc8 f   libucrt:onexit.obj
 0001:00013fc8       ?fin$0@?0???$?RV<lambda_99476a1ad63dd22509b5d3e65b0ffc95>@@AEAV<lambda_ad1ced32f4ac17aa236e5ef05d6b3b7c>@@V<lambda_f7424dd8d45958661754dc4f2697e9c3>@@@?$__crt_seh_guarded_call@X@@QEAAX$$QEAV<lambda_99476a1ad63dd22509b5d3e65b0ffc95>@@AEAV<lambda_ad1ced32f4ac17aa236e5ef05d6b3b7c>@@$$QEAV<lambda_f7424dd8d45958661754dc4f2697e9c3>@@@Z@4HA 0000000180014fc8 f   libucrt:mbctype.obj
 0001:00013fc8       ?fin$0@?0???$?RV<lambda_5e887d1dcbef67a5eb4283622ba103bf>@@AEAV<lambda_4466841279450cc726390878d4a41900>@@V<lambda_341c25c0346d94847f1f3c463c57e077>@@@?$__crt_seh_guarded_call@X@@QEAAX$$QEAV<lambda_5e887d1dcbef67a5eb4283622ba103bf>@@AEAV<lambda_4466841279450cc726390878d4a41900>@@$$QEAV<lambda_341c25c0346d94847f1f3c463c57e077>@@@Z@4HA 0000000180014fc8 f   libucrt:per_thread_data.obj
 0001:00013fc8       ?fin$0@?0???$?RV<lambda_46352004c1216016012b18bd6f87e700>@@AEAV<lambda_3bd07e1a1191394380780325891bf33f>@@V<lambda_334532d3f185bcaa59b5be82d7d22bff>@@@?$__crt_seh_guarded_call@X@@QEAAX$$QEAV<lambda_46352004c1216016012b18bd6f87e700>@@AEAV<lambda_3bd07e1a1191394380780325891bf33f>@@$$QEAV<lambda_334532d3f185bcaa59b5be82d7d22bff>@@@Z@4HA 0000000180014fc8 f   libucrt:per_thread_data.obj
 0001:00013fe2       __acrt_update_thread_multibyte_data$fin$0 0000000180014fe2 f   libucrt:mbctype.obj
 0001:00013ffb       __acrt_initialize_lowio$fin$0 0000000180014ffb f   libucrt:ioinit.obj
 0001:00013ffb       __acrt_lowio_ensure_fh_exists$fin$0 0000000180014ffb f   libucrt:osfinfo.obj
 0001:00014014       raise$fin$0                0000000180015014 f   libucrt:signal.obj
 0001:00014038       __acrt_uninitialize_locale$fin$0 0000000180015038 f   libucrt:wsetlocale.obj
 0001:00014038       __acrt_update_thread_locale_data$fin$0 0000000180015038 f   libucrt:locale_refcounting.obj
 0001:00014051       common_flush_all$fin$0     0000000180015051 f   libucrt:fflush.obj
 0001:0001406b       common_flush_all$fin$1     000000018001506b f   libucrt:fflush.obj
 0001:00014084       _fcloseall$fin$0           0000000180015084 f   libucrt:closeall.obj
 0001:0001409d       ?fin$0@?0???$?RV<lambda_b521505b218e5242e90febf6bfebc422>@@AEAV<lambda_6978c1fb23f02e42e1d9e99668cc68aa>@@V<lambda_314360699dd331753a4119843814e9a7>@@@?$__crt_seh_guarded_call@H@@QEAAH$$QEAV<lambda_b521505b218e5242e90febf6bfebc422>@@AEAV<lambda_6978c1fb23f02e42e1d9e99668cc68aa>@@$$QEAV<lambda_314360699dd331753a4119843814e9a7>@@@Z@4HA 000000018001509d f   libucrt:commit.obj
 0001:0001409d       ?fin$0@?0???$?RV<lambda_bfedae4ebbf01fab1bb6dcc6a9e276e0>@@AEAV<lambda_2fe9b910cf3cbf4a0ab98a02ba45b3ec>@@V<lambda_237c231691f317818eb88cc1d5d642d6>@@@?$__crt_seh_guarded_call@H@@QEAAH$$QEAV<lambda_bfedae4ebbf01fab1bb6dcc6a9e276e0>@@AEAV<lambda_2fe9b910cf3cbf4a0ab98a02ba45b3ec>@@$$QEAV<lambda_237c231691f317818eb88cc1d5d642d6>@@@Z@4HA 000000018001509d f   libucrt:close.obj
 0001:000140b7       _write$fin$0               00000001800150b7 f   libucrt:write.obj
 0001:000140ce       fclose$fin$0               00000001800150ce f   libucrt:fclose.obj
 0001:000140e6       _ctrlfp$filt$0             00000001800150e6 f   libucrt:fpctrl.obj
 0001:00014120       _IsNonwritableInCurrentImage$filt$0 0000000180015120 f   LIBCMT:pesect.obj
 0001:00014140       $xdatasym                  0000000180015140     chkstk.obj
 0001:00014148       $unwind$__acrt_uninitialize_critical 0000000180015148     libucrt:initialization.obj
 0001:00014148       $unwind$__acrt_thread_attach 0000000180015148     libucrt:initialization.obj
 0001:00014148       $unwind$_fileno            0000000180015148     libucrt:fileno.obj
 0001:00014148       $unwind$__acrt_release_locale_ref 0000000180015148     libucrt:locale_refcounting.obj
 0001:00014148       $unwind$__dcrt_uninitialize_environments_nolock 0000000180015148     libucrt:environment_initialization.obj
 0001:00014148       $unwind$__dcrt_terminate_console_output 0000000180015148     libucrt:initcon.obj
 0001:00014148       $unwind$__vcrt_initialize  0000000180015148     libvcruntime:initialization.obj
 0001:00014148       $unwind$?initialize_multibyte@@YAHXZ 0000000180015148     libucrt:multibyte_initializer.obj
 0001:00014148       $unwind$??$uninitialize_environment_internal@D@@YAXAEAPEAPEAD@Z 0000000180015148     libucrt:environment_initialization.obj
 0001:00014148       $unwind$__acrt_uninitialize_ptd 0000000180015148     libucrt:per_thread_data.obj
 0001:00014148       $unwind$_invoke_watson     0000000180015148     libucrt:invalid_parameter.obj
 0001:00014148       $unwind$??$uninitialize_environment_internal@_W@@YAXAEAPEAPEA_W@Z 0000000180015148     libucrt:environment_initialization.obj
 0001:00014148       $unwind$__acrt_initialize_heap 0000000180015148     libucrt:heap_handle.obj
 0001:00014148       $unwind$__GSHandlerCheck   0000000180015148     LIBCMT:_gshandler_.obj
 0001:00014148       $unwind$_get_osfhandle     0000000180015148     libucrt:osfinfo.obj
 0001:00014148       $unwind$__vcrt_thread_attach 0000000180015148     libvcruntime:initialization.obj
 0001:00014148       $unwind$__acrt_thread_detach 0000000180015148     libucrt:initialization.obj
 0001:00014148       $unwind$__acrt_initialize_multibyte 0000000180015148     libucrt:mbctype.obj
 0001:00014148       $unwind$__scrt_dllmain_crt_thread_detach 0000000180015148     LIBCMT:utility.obj
 0001:00014148       $unwind$ConfigureW         0000000180015148     Brackets.obj
 0001:00014148       $unwind$__scrt_dllmain_crt_thread_attach 0000000180015148     LIBCMT:utility.obj
 0001:00014148       $unwind$_set_errno_from_matherr 0000000180015148     libucrt:fpexcept.obj
 0001:00014148       $unwind$__vcrt_thread_detach 0000000180015148     libvcruntime:initialization.obj
 0001:00014148       $unwind$GetGlobalInfoW     0000000180015148     Brackets.obj
 0001:00014148       $unwind$abort              0000000180015148     libucrt:abort.obj
 0001:00014148       $unwind$initialize_c       0000000180015148     libucrt:initialization.obj
 0001:00014148       $unwind$__pctype_func      0000000180015148     libucrt:ctype.obj
 0001:00014148       $unwind$atexit             0000000180015148     LIBCMT:utility.obj
 0001:00014148       $unwind$__acrt_DownlevelLocaleNameToLCID 0000000180015148     libucrt:lcidtoname_downlevel.obj
 0001:00014148       $unwind$__vcrt_freefls     0000000180015148     libvcruntime:per_thread_data.obj
 0001:00014148       $unwind$__acrt_initialize_ptd 0000000180015148     libucrt:per_thread_data.obj
 0001:00014148       $unwind$__scrt_dllmain_uninitialize_critical 0000000180015148     LIBCMT:utility.obj
 0001:00014148       $unwind$uninitialize_environment 0000000180015148     libucrt:initialization.obj
 0001:00014148       $unwind$_errno             0000000180015148     libucrt:errno.obj
 0001:00014148       $unwind$_statfp            0000000180015148     libucrt:fpctrl.obj
 0001:00014148       $unwind$__scrt_acquire_startup_lock 0000000180015148     LIBCMT:utility.obj
 0001:00014148       $unwind$__scrt_dllmain_uninitialize_c 0000000180015148     LIBCMT:utility.obj
 0001:00014148       $unwind$__vcrt_uninitialize_telemetry_provider 0000000180015148     libvcruntime:telemetry.obj
 0001:00014148       $unwind$?dllmain_crt_dispatch@@YAHQEAUHINSTANCE__@@KQEAX@Z 0000000180015148     LIBCMT:dll_dllmain.obj
 0001:00014148       $unwind$__vcrt_uninitialize_ptd 0000000180015148     libvcruntime:per_thread_data.obj
 0001:00014148       $unwind$_isatty            0000000180015148     libucrt:isatty.obj
 0001:00014148       $unwind$__doserrno         0000000180015148     libucrt:errno.obj
 0001:00014148       $unwind$_msize             0000000180015148     libucrt:msize.obj
 0001:00014148       $unwind$__scrt_dllmain_after_initialize_c 0000000180015148     LIBCMT:utility.obj
 0001:00014148       $unwind$__scrt_initialize_default_local_stdio_options 0000000180015148     LIBCMT:default_local_stdio_options.obj
 0001:00014148       $unwind$?ItemWidth@?$DialogBuilderBase@UFarDialogItem@@@@IEAA_JAEBUFarDialogItem@@@Z 0000000180015148     Brackets.obj
 0001:00014148       $unwind$__acrt_initialize_command_line 0000000180015148     libucrt:argv_data.obj
 0001:00014148       $unwind$__scrt_dllmain_before_initialize_c 0000000180015148     LIBCMT:utility.obj
 0001:00014148       $unwind$__vcrt_uninitialize_critical 0000000180015148     libvcruntime:initialization.obj
 0001:00014148       $unwind$__vcrt_initialize_ptd 0000000180015148     libvcruntime:per_thread_data.obj
 0001:00014150       $unwind$OpenW              0000000180015150     Brackets.obj
 0001:00014168       $unwind$SetStartupInfoW    0000000180015168     Brackets.obj
 0001:0001417c       $unwind$?ReallocDialogItems@?$DialogBuilderBase@UFarDialogItem@@@@IEAAXXZ 000000018001517c     Brackets.obj
 0001:0001418c       $unwind$?MaxTextWidth@?$DialogBuilderBase@UFarDialogItem@@@@IEAA_JXZ 000000018001518c     Brackets.obj
 0001:0001419c       $chain$1$?MaxTextWidth@?$DialogBuilderBase@UFarDialogItem@@@@IEAA_JXZ 000000018001519c     Brackets.obj
 0001:000141b4       $chain$2$?MaxTextWidth@?$DialogBuilderBase@UFarDialogItem@@@@IEAA_JXZ 00000001800151b4     Brackets.obj
 0001:000141c4       $unwind$?SaveValues@?$DialogBuilderBase@UFarDialogItem@@@@IEAAXXZ 00000001800151c4     Brackets.obj
 0001:000141d4       $chain$1$?SaveValues@?$DialogBuilderBase@UFarDialogItem@@@@IEAAXXZ 00000001800151d4     Brackets.obj
 0001:000141ec       $chain$2$?SaveValues@?$DialogBuilderBase@UFarDialogItem@@@@IEAAXXZ 00000001800151ec     Brackets.obj
 0001:000141fc       $chain$0$??1?$DialogBuilderBase@UFarDialogItem@@@@MEAA@XZ 00000001800151fc     Brackets.obj
 0001:00014210       $chain$1$??1?$DialogBuilderBase@UFarDialogItem@@@@MEAA@XZ 0000000180015210     Brackets.obj
 0001:00014220       $unwind$?AddButtons@?$DialogBuilderBase@UFarDialogItem@@@@QEAAXHPEBHHH@Z 0000000180015220     Brackets.obj
 0001:00014230       $chain$3$?AddButtons@?$DialogBuilderBase@UFarDialogItem@@@@QEAAXHPEBHHH@Z 0000000180015230     Brackets.obj
 0001:00014250       $chain$4$?AddButtons@?$DialogBuilderBase@UFarDialogItem@@@@QEAAXHPEBHHH@Z 0000000180015250     Brackets.obj
 0001:00014260       $unwind$?DoShowDialog@PluginDialogBuilder@@MEAA_JXZ 0000000180015260     Brackets.obj
 0001:0001426c       $unwind$?AddUIntEditField@PluginDialogBuilder@@UEAAPEAUFarDialogItem@@PEAIH@Z 000000018001526c     Brackets.obj
 0001:0001426c       $unwind$?AddIntEditField@PluginDialogBuilder@@UEAAPEAUFarDialogItem@@PEAHH@Z 000000018001526c     Brackets.obj
 0001:0001426c       $unwind$??$create_environment@D@@YAQEAPEADQEAD@Z 000000018001526c     libucrt:environment_initialization.obj
 0001:00014284       $unwind$?Config@@YAHXZ     0000000180015284     Brackets.obj
 0001:000142a4       $unwind$?ShowMenu@@YAHH@Z  00000001800152a4     Brackets.obj
 0001:000142b8       $unwind$?dllmain_crt_process_attach@@YAHQEAUHINSTANCE__@@QEAX@Z 00000001800152b8     LIBCMT:dll_dllmain.obj
 0001:000142e4       $unwind$?dllmain_crt_process_detach@@YAH_N@Z 00000001800152e4     LIBCMT:dll_dllmain.obj
 0001:0001430c       $unwind$?dllmain_dispatch@@YAHQEAUHINSTANCE__@@KQEAX@Z 000000018001530c     LIBCMT:dll_dllmain.obj
 0001:00014334       $unwind$?filt$0@?0??dllmain_dispatch@@YAHQEAUHINSTANCE__@@KQEAX@Z@4HA 0000000180015334     LIBCMT:dll_dllmain.obj
 0001:0001433c       $unwind$_raise_exc         000000018001533c     libucrt:fpexcept.obj
 0001:0001433c       $unwind$?__scrt_throw_std_bad_array_new_length@@YAXXZ 000000018001533c     LIBCMT:throw_bad_alloc.obj
 0001:0001433c       $unwind$__dcrt_lowio_initialize_console_output 000000018001533c     libucrt:initcon.obj
 0001:0001433c       $unwind$?__scrt_throw_std_bad_alloc@@YAXXZ 000000018001533c     LIBCMT:throw_bad_alloc.obj
 0001:00014344       $unwind$__scrt_is_nonwritable_in_current_image 0000000180015344     LIBCMT:utility.obj
 0001:00014364       $unwind$__scrt_is_nonwritable_in_current_image$filt$0 0000000180015364     LIBCMT:utility.obj
 0001:0001436c       $unwind$__scrt_initialize_onexit_tables 000000018001536c     LIBCMT:utility.obj
 0001:00014378       $unwind$__security_init_cookie 0000000180015378     LIBCMT:gs_support.obj
 0001:00014384       $unwind$__scrt_fastfail    0000000180015384     LIBCMT:utility_desktop.obj
 0001:00014394       $unwind$__acrt_stdio_flush_nolock 0000000180015394     libucrt:fflush.obj
 0001:00014394       $unwind$?CreateCheckBoxBinding@PluginDialogBuilder@@MEAAPEAU?$DialogItemBinding@UFarDialogItem@@@@PEAHH@Z 0000000180015394     Brackets.obj
 0001:00014394       $unwind$_RTC_Terminate     0000000180015394     LIBCMT:_initsect_.obj
 0001:00014394       $unwind$__acrt_FlsSetValue 0000000180015394     libucrt:winapi_thunks.obj
 0001:00014394       $unwind$__acrt_LocaleNameToLCID 0000000180015394     libucrt:winapi_thunks.obj
 0001:00014394       $unwind$__acrt_getptd_noexit 0000000180015394     libucrt:per_thread_data.obj
 0001:00014394       $unwind$??R<lambda_ad1ced32f4ac17aa236e5ef05d6b3b7c>@@QEBAXXZ 0000000180015394     libucrt:mbctype.obj
 0001:00014394       $unwind$_initterm_e        0000000180015394     libucrt:initterm.obj
 0001:00014394       $unwind$?free_crt_array_internal@@YAXQEAPEBX_K@Z 0000000180015394     libucrt:inittime.obj
 0001:00014394       $unwind$__vcrt_FlsSetValue 0000000180015394     libvcruntime:winapi_downlevel.obj
 0001:00014394       $unwind$?TraceLoggingRegister@__vcrt_trace_logging_provider@@YAJPEBU_TlgProvider_t@1@PEBU_GUID@@P6AX1KE_K2PEAU_EVENT_FILTER_DESCRIPTOR@@PEAX@Z4@Z 0000000180015394     libvcruntime:telemetry.obj
 0001:00014394       $unwind$_exception_enabled 0000000180015394     libucrt:libm_error.obj
 0001:00014394       $unwind$__vcrt_getptd_noexit 0000000180015394     libvcruntime:per_thread_data.obj
 0001:00014394       $unwind$_DllMainCRTStartup 0000000180015394     LIBCMT:dll_dllmain.obj
 0001:00014394       $unwind$??$common_lseek_nolock@_J@@YA_JH_JH@Z 0000000180015394     libucrt:lseek.obj
 0001:00014394       $unwind$__acrt_execute_uninitializers 0000000180015394     libucrt:shared_initialization.obj
 0001:00014394       $unwind$_RTC_Initialize    0000000180015394     LIBCMT:_initsect_.obj
 0001:000143a4       $unwind$__isa_available_init 00000001800153a4     LIBCMT:_cpu_disp_.obj
 0001:000143b0       $xdatasym                  00000001800153b0     LIBCMT:_guard_dispatch_.obj
 0001:000143b8       $xdatasym                  00000001800153b8     libvcruntime:memset.obj
 0001:000143bc       $unwind$__telemetry_main_return_trigger 00000001800153bc     libvcruntime:telemetry.obj
 0001:000143bc       $unwind$__telemetry_main_invoke_trigger 00000001800153bc     libvcruntime:telemetry.obj
 0001:000143d4       $unwind$?_TlgEnableCallback@__vcrt_trace_logging_provider@@YAXPEBU_GUID@@KE_K1PEAU_EVENT_FILTER_DESCRIPTOR@@PEAX@Z 00000001800153d4     libvcruntime:telemetry.obj
 0001:000143f0       $unwind$__C_specific_handler 00000001800153f0     libvcruntime:_chandler_.obj
 0001:0001440c       $unwind$?initialize_stdio_handles_nolock@@YAXXZ 000000018001540c     libucrt:ioinit.obj
 0001:0001440c       $unwind$_free_osfhnd       000000018001540c     libucrt:osfinfo.obj
 0001:0001440c       $unwind$__std_exception_copy 000000018001540c     libvcruntime:std_exception.obj
 0001:00014420       $unwind$_CxxThrowException 0000000180015420     libvcruntime:throw.obj
 0001:00014434       $unwind$__acrt_initialize_stdio 0000000180015434     libucrt:_file.obj
 0001:00014434       $unwind$_initterm          0000000180015434     libucrt:initterm.obj
 0001:00014434       $unwind$__vcrt_EventSetInformation 0000000180015434     libvcruntime:winapi_downlevel.obj
 0001:00014434       $unwind$__vcrt_EventRegister 0000000180015434     libvcruntime:winapi_downlevel.obj
 0001:0001444c       $unwind$__vcrt_EventWriteTransfer 000000018001544c     libvcruntime:winapi_downlevel.obj
 0001:0001444c       $unwind$_invalid_parameter 000000018001544c     libucrt:invalid_parameter.obj
 0001:00014464       $unwind$__vcrt_uninitialize_winapi_thunks 0000000180015464     libvcruntime:winapi_downlevel.obj
 0001:00014470       $xdatasym                  0000000180015470     libvcruntime:_jmpuwind_.obj
 0001:00014484       $unwind$_query_new_handler 0000000180015484     libucrt:new_handler.obj
 0001:000144a4       $unwind$?common_exit@@YAXHW4_crt_exit_cleanup_mode@@W4_crt_exit_return_mode@@@Z 00000001800154a4     libucrt:exit.obj
 0001:000144e4       $unwind$??_G?$DialogBuilderBase@UFarDialogItem@@@@MEAAPEAXI@Z 00000001800154e4     Brackets.obj
 0001:000144e4       $unwind$__vcrt_FlsAlloc    00000001800154e4     libvcruntime:winapi_downlevel.obj
 0001:000144e4       $unwind$__acrt_getptd      00000001800154e4     libucrt:per_thread_data.obj
 0001:000144e4       $unwind$__vcrt_FlsFree     00000001800154e4     libvcruntime:winapi_downlevel.obj
 0001:000144e4       $unwind$__acrt_FlsAlloc    00000001800154e4     libucrt:winapi_thunks.obj
 0001:000144e4       $unwind$??_Gbad_alloc@std@@UEAAPEAXI@Z 00000001800154e4     LIBCMT:throw_bad_alloc.obj
 0001:000144e4       $unwind$_close_nolock      00000001800154e4     libucrt:close.obj
 0001:000144e4       $unwind$__acrt_FlsFree     00000001800154e4     libucrt:winapi_thunks.obj
 0001:000144e4       $unwind$__vcrt_EventUnregister 00000001800154e4     libvcruntime:winapi_downlevel.obj
 0001:000144e4       $unwind$__acrt_FlsGetValue 00000001800154e4     libucrt:winapi_thunks.obj
 0001:000144e4       $unwind$?UpdateBorderSize@?$DialogBuilderBase@UFarDialogItem@@@@IEAAXXZ 00000001800154e4     Brackets.obj
 0001:000144e4       $unwind$_updatetlocinfoEx_nolock 00000001800154e4     libucrt:locale_refcounting.obj
 0001:000144e4       $unwind$??0PluginIntEditFieldBinding@@QEAA@AEBUPluginStartupInfo@@PEAPEAXHPEAHH@Z 00000001800154e4     Brackets.obj
 0001:000144e4       $unwind$??_Gexception@std@@UEAAPEAXI@Z 00000001800154e4     LIBCMT:throw_bad_alloc.obj
 0001:000144e4       $unwind$__acrt_uninitialize_lowio 00000001800154e4     libucrt:ioinit.obj
 0001:000144e4       $unwind$?try_cor_exit_process@@YAXI@Z 00000001800154e4     libucrt:exit.obj
 0001:000144e4       $unwind$?CreateRadioButtonBinding@PluginDialogBuilder@@MEAAPEAU?$DialogItemBinding@UFarDialogItem@@@@PEAH@Z 00000001800154e4     Brackets.obj
 0001:000144e4       $unwind$_fclose_nolock     00000001800154e4     libucrt:fclose.obj
 0001:000144e4       $unwind$??_Gbad_array_new_length@std@@UEAAPEAXI@Z 00000001800154e4     LIBCMT:throw_bad_alloc.obj
 0001:000144e4       $unwind$??_GPluginDialogBuilder@@UEAAPEAXI@Z 00000001800154e4     Brackets.obj
 0001:000144e4       $unwind$?SaveValue@PluginRadioButtonBinding@@UEAAXPEAUFarDialogItem@@H@Z 00000001800154e4     Brackets.obj
 0001:000144e4       $unwind$__acrt_invoke_user_matherr 00000001800154e4     libucrt:matherr.obj
 0001:000144e4       $unwind$_realloc_base      00000001800154e4     libucrt:realloc_base.obj
 0001:000144e4       $unwind$??0PluginUIntEditFieldBinding@@QEAA@AEBUPluginStartupInfo@@PEAPEAXHPEAIH@Z 00000001800154e4     Brackets.obj
 0001:000144e4       $unwind$?replace_current_thread_locale_nolock@@YAXQEAU__acrt_ptd@@QEAU__crt_locale_data@@@Z 00000001800154e4     libucrt:per_thread_data.obj
 0001:000144e4       $unwind$??0_LocaleUpdate@@QEAA@QEAU__crt_locale_pointers@@@Z 00000001800154e4     libucrt:output.obj
 0001:000144e4       $unwind$_callnewh          00000001800154e4     libucrt:new_handler.obj
 0001:000144e4       $unwind$?InitDialogItem@PluginDialogBuilder@@MEAAXPEAUFarDialogItem@@PEB_W@Z 00000001800154e4     Brackets.obj
 0001:000144e4       $unwind$??$common_initialize_environment_nolock@D@@YAHXZ 00000001800154e4     libucrt:environment_initialization.obj
 0001:000144e4       $unwind$__acrt_errno_map_os_error 00000001800154e4     libucrt:errno.obj
 0001:000144e4       $unwind$__vcrt_FlsGetValue 00000001800154e4     libvcruntime:winapi_downlevel.obj
 0001:000144f0       $unwind$??$free_environment@_W@@YAXQEAPEA_W@Z 00000001800154f0     libucrt:environment_initialization.obj
 0001:000144f0       $unwind$??$free_environment@D@@YAXQEAPEAD@Z 00000001800154f0     libucrt:environment_initialization.obj
 0001:000144fc       $unwind$_register_onexit_function 00000001800154fc     libucrt:onexit.obj
 0001:00014504       $unwind$_execute_onexit_table 0000000180015504     libucrt:onexit.obj
 0001:0001450c       $unwind$??R<lambda_4e60a939b0d047cfe11ddc22648dfba9>@@QEBAHXZ 000000018001550c     libucrt:onexit.obj
 0001:00014528       $unwind$??$?RV<lambda_b8c45f8f788dd370798f47cfe8ac3a86>@@AEAV<lambda_4e60a939b0d047cfe11ddc22648dfba9>@@V<lambda_332c3edc96d0294ec56c57d38c1cdfd5>@@@?$__crt_seh_guarded_call@H@@QEAAH$$QEAV<lambda_b8c45f8f788dd370798f47cfe8ac3a86>@@AEAV<lambda_4e60a939b0d047cfe11ddc22648dfba9>@@$$QEAV<lambda_332c3edc96d0294ec56c57d38c1cdfd5>@@@Z 0000000180015528     libucrt:onexit.obj
 0001:0001454c       $unwind$??$?RV<lambda_e24bbb7b643b32fcea6fa61b31d4c984>@@AEAV<lambda_275893d493268fdec8709772e3fcec0e>@@V<lambda_9d71df4d7cf3f480f8d633942495c3b0>@@@?$__crt_seh_guarded_call@H@@QEAAH$$QEAV<lambda_e24bbb7b643b32fcea6fa61b31d4c984>@@AEAV<lambda_275893d493268fdec8709772e3fcec0e>@@$$QEAV<lambda_9d71df4d7cf3f480f8d633942495c3b0>@@@Z 000000018001554c     libucrt:onexit.obj
 0001:0001457c       $unwind$terminate          000000018001557c     libucrt:terminate.obj
 0001:0001459c       $unwind$?construct_ptd_array@@YAXQEAU__acrt_ptd@@@Z 000000018001559c     libucrt:per_thread_data.obj
 0001:000145a4       $unwind$?destroy_ptd_array@@YAXQEAU__acrt_ptd@@@Z 00000001800155a4     libucrt:per_thread_data.obj
 0001:000145ac       $unwind$??$?RV<lambda_72d1df2b273a38828b1ce30cbf4cdab5>@@AEAV<lambda_876a65b173b8412d3a47c70a915b0cf4>@@V<lambda_41932305e351933ebe8f8be3ed8bb5dc>@@@?$__crt_seh_guarded_call@X@@QEAAX$$QEAV<lambda_72d1df2b273a38828b1ce30cbf4cdab5>@@AEAV<lambda_876a65b173b8412d3a47c70a915b0cf4>@@$$QEAV<lambda_41932305e351933ebe8f8be3ed8bb5dc>@@@Z 00000001800155ac     libucrt:per_thread_data.obj
 0001:000145d0       $unwind$??$?RV<lambda_5e887d1dcbef67a5eb4283622ba103bf>@@AEAV<lambda_4466841279450cc726390878d4a41900>@@V<lambda_341c25c0346d94847f1f3c463c57e077>@@@?$__crt_seh_guarded_call@X@@QEAAX$$QEAV<lambda_5e887d1dcbef67a5eb4283622ba103bf>@@AEAV<lambda_4466841279450cc726390878d4a41900>@@$$QEAV<lambda_341c25c0346d94847f1f3c463c57e077>@@@Z 00000001800155d0     libucrt:per_thread_data.obj
 0001:000145f4       $unwind$??$?RV<lambda_46352004c1216016012b18bd6f87e700>@@AEAV<lambda_3bd07e1a1191394380780325891bf33f>@@V<lambda_334532d3f185bcaa59b5be82d7d22bff>@@@?$__crt_seh_guarded_call@X@@QEAAX$$QEAV<lambda_46352004c1216016012b18bd6f87e700>@@AEAV<lambda_3bd07e1a1191394380780325891bf33f>@@$$QEAV<lambda_334532d3f185bcaa59b5be82d7d22bff>@@@Z 00000001800155f4     libucrt:per_thread_data.obj
 0001:00014618       $unwind$??$?RV<lambda_fb3a7dec4e47f37f22dae91bb15c9095>@@AEAV<lambda_698284760c8add0bfb0756c19673e34b>@@V<lambda_dfb8eca1e75fef3034a8fb18dd509707>@@@?$__crt_seh_guarded_call@X@@QEAAX$$QEAV<lambda_fb3a7dec4e47f37f22dae91bb15c9095>@@AEAV<lambda_698284760c8add0bfb0756c19673e34b>@@$$QEAV<lambda_dfb8eca1e75fef3034a8fb18dd509707>@@@Z 0000000180015618     libucrt:per_thread_data.obj
 0001:0001463c       $unwind$__vcrt_initialize_winapi_thunks 000000018001563c     libvcruntime:winapi_downlevel.obj
 0001:0001463c       $unwind$__acrt_initialize_winapi_thunks 000000018001563c     libucrt:winapi_thunks.obj
 0001:00014644       $unwind$??1?$DialogBuilderBase@UFarDialogItem@@@@MEAA@XZ 0000000180015644     Brackets.obj
 0001:00014644       $unwind$__acrt_is_packaged_app 0000000180015644     libucrt:winapi_thunks.obj
 0001:00014650       $unwind$?try_get_function@@YAPEAXW4function_id@?A0x63058377@@QEBDQEBW4module_id@2@2@Z 0000000180015650     libucrt:winapi_thunks.obj
 0001:00014650       $unwind$?try_get_function@@YAPEAXW4function_id@?A0x61ce2399@@QEBDQEBW4module_id@2@2@Z 0000000180015650     libvcruntime:winapi_downlevel.obj
 0001:0001466c       $unwind$__acrt_call_reportfault 000000018001566c     libucrt:invalid_parameter.obj
 0001:0001468c       $unwind$__acrt_update_thread_multibyte_data 000000018001568c     libucrt:mbctype.obj
 0001:000146b0       $unwind$_setmbcp_nolock    00000001800156b0     libucrt:mbctype.obj
 0001:000146d0       $unwind$?setSBUpLow@@YAXPEAU__crt_multibyte_data@@@Z 00000001800156d0     libucrt:mbctype.obj
 0001:000146ec       $unwind$?setmbcp_internal@@YAHH_N@Z 00000001800156ec     libucrt:mbctype.obj
 0001:000146fc       $unwind$??$?RV<lambda_99476a1ad63dd22509b5d3e65b0ffc95>@@AEAV<lambda_ad1ced32f4ac17aa236e5ef05d6b3b7c>@@V<lambda_f7424dd8d45958661754dc4f2697e9c3>@@@?$__crt_seh_guarded_call@X@@QEAAX$$QEAV<lambda_99476a1ad63dd22509b5d3e65b0ffc95>@@AEAV<lambda_ad1ced32f4ac17aa236e5ef05d6b3b7c>@@$$QEAV<lambda_f7424dd8d45958661754dc4f2697e9c3>@@@Z 00000001800156fc     libucrt:mbctype.obj
 0001:00014720       $unwind$__dcrt_get_narrow_environment_from_os 0000000180015720     libucrt:get_environment_from_os.obj
 0001:00014738       $unwind$__acrt_initialize_lowio 0000000180015738     libucrt:ioinit.obj
 0001:00014758       $unwind$?initialize_inherited_file_handles_nolock@@YAXXZ 0000000180015758     libucrt:ioinit.obj
 0001:00014774       $unwind$__acrt_get_sigabrt_handler 0000000180015774     libucrt:signal.obj
 0001:0001477c       $unwind$raise              000000018001577c     libucrt:signal.obj
 0001:000147a8       $unwind$??$?RV<lambda_c36588078e9f5dfd39652860aa6b3aaf>@@AEAV<lambda_ec61778202f4f5fc7e7711acc23c3bca>@@V<lambda_dc9d2797ccde5d239b4a0efae8ebd7db>@@@?$__crt_seh_guarded_call@P6AXH@Z@@QEAAP6AXH@Z$$QEAV<lambda_c36588078e9f5dfd39652860aa6b3aaf>@@AEAV<lambda_ec61778202f4f5fc7e7711acc23c3bca>@@$$QEAV<lambda_dc9d2797ccde5d239b4a0efae8ebd7db>@@@Z 00000001800157a8     libucrt:signal.obj
 0001:000147cc       $unwind$_mbtowc_l          00000001800157cc     libucrt:mbtowc.obj
 0001:000147cc       $unwind$__acrt_LCMapStringEx 00000001800157cc     libucrt:winapi_thunks.obj
 0001:000147e4       $unwind$__acrt_uninitialize_locale 00000001800157e4     libucrt:wsetlocale.obj
 0001:00014804       $unwind$_free_base         0000000180015804     libucrt:free_base.obj
 0001:00014804       $unwind$__acrt_locale_free_numeric 0000000180015804     libucrt:initnum.obj
 0001:00014804       $unwind$?destroy_fls@@YAXPEAX@Z 0000000180015804     libucrt:per_thread_data.obj
 0001:00014804       $unwind$__acrt_locale_free_lc_time_if_unreferenced 0000000180015804     libucrt:locale_refcounting.obj
 0001:0001480c       $unwind$__acrt_update_thread_locale_data 000000018001580c     libucrt:locale_refcounting.obj
 0001:00014830       $unwind$?GetTableIndexFromLocaleName@@YAHPEB_W@Z 0000000180015830     libucrt:lcidtoname_downlevel.obj
 0001:00014848       $unwind$__acrt_GetStringTypeA 0000000180015848     libucrt:getstringtypea.obj
 0001:00014870       $unwind$__acrt_LCMapStringA 0000000180015870     libucrt:lcmapstringa.obj
 0001:00014880       $unwind$?__acrt_LCMapStringA_stat@@YAHPEAU__crt_locale_pointers@@PEB_WKPEBDHPEADHHH@Z 0000000180015880     libucrt:lcmapstringa.obj
 0001:000148a8       $unwind$_recalloc_base     00000001800158a8     libucrt:recalloc.obj
 0001:000148a8       $unwind$__scrt_dllmain_exception_filter 00000001800158a8     LIBCMT:utility.obj
 0001:000148a8       $unwind$__acrt_execute_initializers 00000001800158a8     libucrt:shared_initialization.obj
 0001:000148a8       $unwind$__acrt_lowio_create_handle_array 00000001800158a8     libucrt:osfinfo.obj
 0001:000148a8       $unwind$__vcrt_InitializeCriticalSectionEx 00000001800158a8     libvcruntime:winapi_downlevel.obj
 0001:000148a8       $unwind$__acrt_free_locale 00000001800158a8     libucrt:locale_refcounting.obj
 0001:000148a8       $unwind$?dllmain_raw@@YAHQEAUHINSTANCE__@@KQEAX@Z 00000001800158a8     LIBCMT:dll_dllmain.obj
 0001:000148a8       $unwind$?setSBCS@@YAXPEAU__crt_multibyte_data@@@Z 00000001800158a8     libucrt:mbctype.obj
 0001:000148a8       $unwind$__acrt_InitializeCriticalSectionEx 00000001800158a8     libucrt:winapi_thunks.obj
 0001:000148a8       $unwind$_seh_filter_exe    00000001800158a8     libucrt:exception_filter.obj
 0001:000148bc       $unwind$__acrt_lowio_destroy_handle_array 00000001800158bc     libucrt:osfinfo.obj
 0001:000148cc       $unwind$__acrt_lowio_ensure_fh_exists 00000001800158cc     libucrt:osfinfo.obj
 0001:000148f8       $unwind$common_flush_all   00000001800158f8     libucrt:fflush.obj
 0001:00014934       $unwind$_isleadbyte_l      0000000180015934     libucrt:_wctype.obj
 0001:00014934       $unwind$?getSystemCP@@YAHH@Z 0000000180015934     libucrt:mbctype.obj
 0001:00014934       $unwind$?_TlgWrite@__vcrt_trace_logging_provider@@YAJPEBU_TlgProvider_t@1@PEFBXPEBU_GUID@@2IPEAU_EVENT_DATA_DESCRIPTOR@@@Z 0000000180015934     libvcruntime:telemetry.obj
 0001:0001493c       $unwind$_fcloseall         000000018001593c     libucrt:closeall.obj
 0001:00014960       $unwind$??_GPluginEditFieldBinding@@UEAAPEAXI@Z 0000000180015960     Brackets.obj
 0001:00014960       $unwind$__acrt_uninitialize_stdio 0000000180015960     libucrt:_file.obj
 0001:00014960       $unwind$?SaveValue@PluginIntEditFieldBinding@@UEAAXPEAUFarDialogItem@@H@Z 0000000180015960     Brackets.obj
 0001:00014960       $unwind$__std_type_info_destroy_list 0000000180015960     libvcruntime:std_type_info.obj
 0001:00014960       $unwind$__acrt_stdio_free_buffer_nolock 0000000180015960     libucrt:_freebuf.obj
 0001:00014960       $unwind$__vcrt_uninitialize_locks 0000000180015960     libvcruntime:locks.obj
 0001:00014960       $unwind$strcpy_s           0000000180015960     libucrt:strcpy_s.obj
 0001:00014960       $unwind$_onexit            0000000180015960     LIBCMT:utility.obj
 0001:00014960       $unwind$__vcrt_freeptd     0000000180015960     libvcruntime:per_thread_data.obj
 0001:00014960       $unwind$__vcrt_initialize_locks 0000000180015960     libvcruntime:locks.obj
 0001:00014960       $unwind$??_GPluginIntEditFieldBinding@@UEAAPEAXI@Z 0000000180015960     Brackets.obj
 0001:00014960       $unwind$__acrt_update_multibyte_info 0000000180015960     libucrt:locale_update.obj
 0001:00014960       $unwind$_set_statfp        0000000180015960     libucrt:fpctrl.obj
 0001:00014960       $unwind$?exit_or_terminate_process@@YAXI@Z 0000000180015960     libucrt:exit.obj
 0001:00014960       $unwind$??0bad_array_new_length@std@@QEAA@AEBV01@@Z 0000000180015960     LIBCMT:throw_bad_alloc.obj
 0001:00014960       $unwind$?SaveValue@PluginUIntEditFieldBinding@@UEAAXPEAUFarDialogItem@@H@Z 0000000180015960     Brackets.obj
 0001:00014960       $unwind$__acrt_initialize_locks 0000000180015960     libucrt:locks.obj
 0001:00014960       $unwind$??_GPluginUIntEditFieldBinding@@UEAAPEAXI@Z 0000000180015960     Brackets.obj
 0001:00014960       $unwind$initialize_pointers 0000000180015960     libucrt:initialization.obj
 0001:00014960       $unwind$?SaveValue@PluginEditFieldBinding@@UEAAXPEAUFarDialogItem@@H@Z 0000000180015960     Brackets.obj
 0001:00014960       $unwind$__acrt_uninitialize_winapi_thunks 0000000180015960     libucrt:winapi_thunks.obj
 0001:00014960       $unwind$??_GPluginRadioButtonBinding@@UEAAPEAXI@Z 0000000180015960     Brackets.obj
 0001:00014960       $unwind$_calloc_base       0000000180015960     libucrt:calloc_base.obj
 0001:00014960       $unwind$__raise_securityfailure 0000000180015960     LIBCMT:gs_report.obj
 0001:00014960       $unwind$??0bad_alloc@std@@QEAA@AEBV01@@Z 0000000180015960     LIBCMT:throw_bad_alloc.obj
 0001:00014960       $unwind$__acrt_freeptd     0000000180015960     libucrt:per_thread_data.obj
 0001:00014960       $unwind$_clrfp             0000000180015960     libucrt:fpctrl.obj
 0001:00014960       $unwind$__std_exception_destroy 0000000180015960     libvcruntime:std_exception.obj
 0001:00014960       $unwind$??_GPluginCheckBoxBinding@@UEAAPEAXI@Z 0000000180015960     Brackets.obj
 0001:00014960       $unwind$__scrt_uninitialize_crt 0000000180015960     LIBCMT:utility.obj
 0001:00014960       $unwind$??0exception@std@@QEAA@AEBV01@@Z 0000000180015960     LIBCMT:throw_bad_alloc.obj
 0001:00014960       $unwind$?SaveValue@PluginCheckBoxBinding@@UEAAXPEAUFarDialogItem@@H@Z 0000000180015960     Brackets.obj
 0001:00014960       $unwind$__scrt_release_startup_lock 0000000180015960     LIBCMT:utility.obj
 0001:00014960       $unwind$??_G?$DialogItemBinding@UFarDialogItem@@@@UEAAPEAXI@Z 0000000180015960     Brackets.obj
 0001:00014960       $unwind$__acrt_update_locale_info 0000000180015960     libucrt:locale_update.obj
 0001:00014960       $unwind$__scrt_initialize_crt 0000000180015960     LIBCMT:utility.obj
 0001:00014960       $unwind$??2@YAPEAX_K@Z     0000000180015960     LIBCMT:new_scalar.obj
 0001:00014960       $unwind$__vcrt_uninitialize 0000000180015960     libvcruntime:initialization.obj
 0001:00014960       $unwind$??_Gtype_info@@UEAAPEAXI@Z 0000000180015960     LIBCMT:std_type_info_static.obj
 0001:00014960       $unwind$__acrt_uninitialize_locks 0000000180015960     libucrt:locks.obj
 0001:00014960       $unwind$GetPluginInfoW     0000000180015960     Brackets.obj
 0001:00014960       $unwind$_malloc_base       0000000180015960     libucrt:malloc_base.obj
 0001:00014960       $unwind$uninitialize_allocated_memory 0000000180015960     libucrt:initialization.obj
 0001:00014960       $unwind$_fflush_nolock     0000000180015960     libucrt:fflush.obj
 0001:00014968       $unwind$__acrt_locale_free_monetary 0000000180015968     libucrt:initmon.obj
 0001:00014970       $unwind$__acrt_locale_free_time 0000000180015970     libucrt:inittime.obj
 0001:00014980       $unwind$_commit            0000000180015980     libucrt:commit.obj
 0001:00014980       $unwind$_close             0000000180015980     libucrt:close.obj
 0001:00014988       $unwind$??$?RV<lambda_b521505b218e5242e90febf6bfebc422>@@AEAV<lambda_6978c1fb23f02e42e1d9e99668cc68aa>@@V<lambda_314360699dd331753a4119843814e9a7>@@@?$__crt_seh_guarded_call@H@@QEAAH$$QEAV<lambda_b521505b218e5242e90febf6bfebc422>@@AEAV<lambda_6978c1fb23f02e42e1d9e99668cc68aa>@@$$QEAV<lambda_314360699dd331753a4119843814e9a7>@@@Z 0000000180015988     libucrt:commit.obj
 0001:000149ac       $unwind$_write             00000001800159ac     libucrt:write.obj
 0001:000149dc       $unwind$_write_nolock      00000001800159dc     libucrt:write.obj
 0001:000149f4       $unwind$?write_double_translated_ansi_nolock@@YA?AUwrite_result@?A0x9c548279@@HQEBDI@Z 00000001800159f4     libucrt:write.obj
 0001:00014a14       $unwind$?write_text_utf16le_nolock@@YA?AUwrite_result@?A0x9c548279@@HQEBDI@Z 0000000180015a14     libucrt:write.obj
 0001:00014a14       $unwind$?write_text_ansi_nolock@@YA?AUwrite_result@?A0x9c548279@@HQEBDI@Z 0000000180015a14     libucrt:write.obj
 0001:00014a34       $unwind$?write_text_utf8_nolock@@YA?AUwrite_result@?A0x9c548279@@HQEBDI@Z 0000000180015a34     libucrt:write.obj
 0001:00014a58       $xdatasym                  0000000180015a58     libucrt:log10.obj
 0001:00014a64       $unwind$fclose             0000000180015a64     libucrt:fclose.obj
 0001:00014a88       $unwind$__acrt_update_thread_locale_data$fin$0 0000000180015a88     libucrt:locale_refcounting.obj
 0001:00014a88       $unwind$?fin$0@?0??dllmain_crt_process_attach@@YAHQEAUHINSTANCE__@@QEAX@Z@4HA 0000000180015a88     LIBCMT:dll_dllmain.obj
 0001:00014a88       $unwind$__acrt_uninitialize_locale$fin$0 0000000180015a88     libucrt:wsetlocale.obj
 0001:00014a88       $unwind$common_flush_all$fin$1 0000000180015a88     libucrt:fflush.obj
 0001:00014a88       $unwind$_fcloseall$fin$0   0000000180015a88     libucrt:closeall.obj
 0001:00014a88       $unwind$?fin$0@?0???$?RV<lambda_b521505b218e5242e90febf6bfebc422>@@AEAV<lambda_6978c1fb23f02e42e1d9e99668cc68aa>@@V<lambda_314360699dd331753a4119843814e9a7>@@@?$__crt_seh_guarded_call@H@@QEAAH$$QEAV<lambda_b521505b218e5242e90febf6bfebc422>@@AEAV<lambda_6978c1fb23f02e42e1d9e99668cc68aa>@@$$QEAV<lambda_314360699dd331753a4119843814e9a7>@@@Z@4HA 0000000180015a88     libucrt:commit.obj
 0001:00014a88       $unwind$?fin$0@?0???$?RV<lambda_e24bbb7b643b32fcea6fa61b31d4c984>@@AEAV<lambda_275893d493268fdec8709772e3fcec0e>@@V<lambda_9d71df4d7cf3f480f8d633942495c3b0>@@@?$__crt_seh_guarded_call@H@@QEAAH$$QEAV<lambda_e24bbb7b643b32fcea6fa61b31d4c984>@@AEAV<lambda_275893d493268fdec8709772e3fcec0e>@@$$QEAV<lambda_9d71df4d7cf3f480f8d633942495c3b0>@@@Z@4HA 0000000180015a88     libucrt:onexit.obj
 0001:00014a88       $unwind$common_flush_all$fin$0 0000000180015a88     libucrt:fflush.obj
 0001:00014a88       $unwind$_ctrlfp$filt$0     0000000180015a88     libucrt:fpctrl.obj
 0001:00014a88       $unwind$?filt$0@?0??common_exit@@YAXHW4_crt_exit_cleanup_mode@@W4_crt_exit_return_mode@@@Z@4HA 0000000180015a88     libucrt:exit.obj
 0001:00014a88       $unwind$?fin$0@?0???$?RV<lambda_72d1df2b273a38828b1ce30cbf4cdab5>@@AEAV<lambda_876a65b173b8412d3a47c70a915b0cf4>@@V<lambda_41932305e351933ebe8f8be3ed8bb5dc>@@@?$__crt_seh_guarded_call@X@@QEAAX$$QEAV<lambda_72d1df2b273a38828b1ce30cbf4cdab5>@@AEAV<lambda_876a65b173b8412d3a47c70a915b0cf4>@@$$QEAV<lambda_41932305e351933ebe8f8be3ed8bb5dc>@@@Z@4HA 0000000180015a88     libucrt:per_thread_data.obj
 0001:00014a88       $unwind$fclose$fin$0       0000000180015a88     libucrt:fclose.obj
 0001:00014a88       $unwind$_query_new_handler$fin$0 0000000180015a88     libucrt:new_handler.obj
 0001:00014a88       $unwind$?fin$0@?0???$?RV<lambda_46352004c1216016012b18bd6f87e700>@@AEAV<lambda_3bd07e1a1191394380780325891bf33f>@@V<lambda_334532d3f185bcaa59b5be82d7d22bff>@@@?$__crt_seh_guarded_call@X@@QEAAX$$QEAV<lambda_46352004c1216016012b18bd6f87e700>@@AEAV<lambda_3bd07e1a1191394380780325891bf33f>@@$$QEAV<lambda_334532d3f185bcaa59b5be82d7d22bff>@@@Z@4HA 0000000180015a88     libucrt:per_thread_data.obj
 0001:00014a88       $unwind$?fin$0@?0???$?RV<lambda_bfedae4ebbf01fab1bb6dcc6a9e276e0>@@AEAV<lambda_2fe9b910cf3cbf4a0ab98a02ba45b3ec>@@V<lambda_237c231691f317818eb88cc1d5d642d6>@@@?$__crt_seh_guarded_call@H@@QEAAH$$QEAV<lambda_bfedae4ebbf01fab1bb6dcc6a9e276e0>@@AEAV<lambda_2fe9b910cf3cbf4a0ab98a02ba45b3ec>@@$$QEAV<lambda_237c231691f317818eb88cc1d5d642d6>@@@Z@4HA 0000000180015a88     libucrt:close.obj
 0001:00014a88       $unwind$__acrt_lowio_ensure_fh_exists$fin$0 0000000180015a88     libucrt:osfinfo.obj
 0001:00014a88       $unwind$?fin$0@?0???$?RV<lambda_99476a1ad63dd22509b5d3e65b0ffc95>@@AEAV<lambda_ad1ced32f4ac17aa236e5ef05d6b3b7c>@@V<lambda_f7424dd8d45958661754dc4f2697e9c3>@@@?$__crt_seh_guarded_call@X@@QEAAX$$QEAV<lambda_99476a1ad63dd22509b5d3e65b0ffc95>@@AEAV<lambda_ad1ced32f4ac17aa236e5ef05d6b3b7c>@@$$QEAV<lambda_f7424dd8d45958661754dc4f2697e9c3>@@@Z@4HA 0000000180015a88     libucrt:mbctype.obj
 0001:00014a88       $unwind$?fin$0@?0???$?RV<lambda_c36588078e9f5dfd39652860aa6b3aaf>@@AEAV<lambda_ec61778202f4f5fc7e7711acc23c3bca>@@V<lambda_dc9d2797ccde5d239b4a0efae8ebd7db>@@@?$__crt_seh_guarded_call@P6AXH@Z@@QEAAP6AXH@Z$$QEAV<lambda_c36588078e9f5dfd39652860aa6b3aaf>@@AEAV<lambda_ec61778202f4f5fc7e7711acc23c3bca>@@$$QEAV<lambda_dc9d2797ccde5d239b4a0efae8ebd7db>@@@Z@4HA 0000000180015a88     libucrt:signal.obj
 0001:00014a88       $unwind$?fin$1@?0??common_exit@@YAXHW4_crt_exit_cleanup_mode@@W4_crt_exit_return_mode@@@Z@4HA 0000000180015a88     libucrt:exit.obj
 0001:00014a88       $unwind$__acrt_update_thread_multibyte_data$fin$0 0000000180015a88     libucrt:mbctype.obj
 0001:00014a88       $unwind$?fin$0@?0??dllmain_crt_process_detach@@YAH_N@Z@4HA 0000000180015a88     LIBCMT:dll_dllmain.obj
 0001:00014a88       $unwind$_write$fin$0       0000000180015a88     libucrt:write.obj
 0001:00014a88       $unwind$?fin$0@?0???$?RV<lambda_5e887d1dcbef67a5eb4283622ba103bf>@@AEAV<lambda_4466841279450cc726390878d4a41900>@@V<lambda_341c25c0346d94847f1f3c463c57e077>@@@?$__crt_seh_guarded_call@X@@QEAAX$$QEAV<lambda_5e887d1dcbef67a5eb4283622ba103bf>@@AEAV<lambda_4466841279450cc726390878d4a41900>@@$$QEAV<lambda_341c25c0346d94847f1f3c463c57e077>@@@Z@4HA 0000000180015a88     libucrt:per_thread_data.obj
 0001:00014a88       $unwind$__acrt_initialize_lowio$fin$0 0000000180015a88     libucrt:ioinit.obj
 0001:00014a88       $unwind$raise$fin$0        0000000180015a88     libucrt:signal.obj
 0001:00014a88       $unwind$?fin$0@?0???$?RV<lambda_b8c45f8f788dd370798f47cfe8ac3a86>@@AEAV<lambda_4e60a939b0d047cfe11ddc22648dfba9>@@V<lambda_332c3edc96d0294ec56c57d38c1cdfd5>@@@?$__crt_seh_guarded_call@H@@QEAAH$$QEAV<lambda_b8c45f8f788dd370798f47cfe8ac3a86>@@AEAV<lambda_4e60a939b0d047cfe11ddc22648dfba9>@@$$QEAV<lambda_332c3edc96d0294ec56c57d38c1cdfd5>@@@Z@4HA 0000000180015a88     libucrt:onexit.obj
 0001:00014a88       $unwind$_IsNonwritableInCurrentImage$filt$0 0000000180015a88     LIBCMT:pesect.obj
 0001:00014a88       $unwind$?fin$0@?0???$?RV<lambda_fb3a7dec4e47f37f22dae91bb15c9095>@@AEAV<lambda_698284760c8add0bfb0756c19673e34b>@@V<lambda_dfb8eca1e75fef3034a8fb18dd509707>@@@?$__crt_seh_guarded_call@X@@QEAAX$$QEAV<lambda_fb3a7dec4e47f37f22dae91bb15c9095>@@AEAV<lambda_698284760c8add0bfb0756c19673e34b>@@$$QEAV<lambda_dfb8eca1e75fef3034a8fb18dd509707>@@@Z@4HA 0000000180015a88     libucrt:per_thread_data.obj
 0001:00014a90       $unwind$_putwch_nolock     0000000180015a90     libucrt:putwch.obj
 0001:00014a90       $unwind$__report_gsfailure 0000000180015a90     LIBCMT:gs_report.obj
 0001:00014a98       $unwind$_call_matherr      0000000180015a98     libucrt:libm_error.obj
 0001:00014aa0       $unwind$_handle_error      0000000180015aa0     libucrt:libm_error.obj
 0001:00014ac0       $unwind$__acrt_initialize_fma3 0000000180015ac0     libucrt:fma3_available.obj
 0001:00014ac8       $unwind$_log_special_common 0000000180015ac8     libucrt:log_special.obj
 0001:00014ad4       $unwind$_log10_special     0000000180015ad4     libucrt:log_special.obj
 0001:00014ad4       $unwind$_invalid_parameter_noinfo 0000000180015ad4     libucrt:invalid_parameter.obj
 0001:00014adc       $unwind$??$?RV<lambda_bfedae4ebbf01fab1bb6dcc6a9e276e0>@@AEAV<lambda_2fe9b910cf3cbf4a0ab98a02ba45b3ec>@@V<lambda_237c231691f317818eb88cc1d5d642d6>@@@?$__crt_seh_guarded_call@H@@QEAAH$$QEAV<lambda_bfedae4ebbf01fab1bb6dcc6a9e276e0>@@AEAV<lambda_2fe9b910cf3cbf4a0ab98a02ba45b3ec>@@$$QEAV<lambda_237c231691f317818eb88cc1d5d642d6>@@@Z 0000000180015adc     libucrt:close.obj
 0001:00014b00       $xdatasym                  0000000180015b00     libucrt:fpsr.obj
 0001:00014b08       $unwind$_raise_exc_ex      0000000180015b08     libucrt:fpexcept.obj
 0001:00014b1c       $unwind$_ctrlfp            0000000180015b1c     libucrt:fpctrl.obj
 0001:00014b44       $unwind$__GSHandlerCheckCommon 0000000180015b44     LIBCMT:_gshandler_.obj
 0001:00014b50       $xdatasym                  0000000180015b50     LIBCMT:_amdsecgs_.obj
 0001:00014b54       $unwind$_IsNonwritableInCurrentImage 0000000180015b54     LIBCMT:pesect.obj
 0001:00014b78       $unwind$capture_previous_context 0000000180015b78     LIBCMT:gs_report.obj
 0001:00014b88       $xdatasym                  0000000180015b88     libvcruntime:memcpy.obj
 0001:00014b90       $xdatasym                  0000000180015b90     libvcruntime:memcmp.obj
 0001:00014c90       .edata                     0000000180015c90     Brackets.exp
 0001:00014cb8       rgpv                       0000000180015cb8     Brackets.exp
 0001:00014ccc       rgszName                   0000000180015ccc     Brackets.exp
 0001:00014ce0       rgwOrd                     0000000180015ce0     Brackets.exp
 0001:00014cea       szName                     0000000180015cea     Brackets.exp
 0001:00014cf7       $N00001                    0000000180015cf7     Brackets.exp
 0001:00014d02       $N00002                    0000000180015d02     Brackets.exp
 0001:00014d11       $N00003                    0000000180015d11     Brackets.exp
 0001:00014d20       $N00004                    0000000180015d20     Brackets.exp
 0001:00014d26       $N00005                    0000000180015d26     Brackets.exp
 0002:00000000       ?HelpTopic@?1??ShowMenu@@YAHH@Z@4PAPEB_WA 0000000180016000     Brackets.obj
 0002:00000010       ?CmdName@?BB@??OpenW@@9@4PAU<unnamed-type-CmdName>@?BB@??1@YAPEAXPEBUOpenInfo@@@Z@A 0000000180016010     Brackets.obj
 0002:000000a0       ?_Tlg_Microsoft_CRTProviderProv@@3U_TlgProvider_t@__vcrt_trace_logging_provider@@A 00000001800160a0     libvcruntime:telemetry.obj
 0002:000000f0       ?__vcrt_flsindex@@3KA      00000001800160f0     libvcruntime:per_thread_data.obj
 0002:000000f8       __acrt_flsindex            00000001800160f8     libucrt:per_thread_data.obj
 0002:00000330       __rgctypeflag              0000000180016330     libucrt:mbctype.obj
 0002:00000340       __rgcode_page_info         0000000180016340     libucrt:mbctype.obj
 0002:000007ac       errno_no_memory            00000001800167ac     libucrt:errno.obj
 0002:000007b0       doserrno_no_memory         00000001800167b0     libucrt:errno.obj
 0002:00000980       ?dazSupported@?1??_ctrlfp@@9@9 0000000180016980     libucrt:fpctrl.obj
 0002:00000a40       ?Opt@@3UOptions@@A         0000000180016a40     Brackets.obj
 0002:00000b00       ?Info@@3UPluginStartupInfo@@A 0000000180016b00     Brackets.obj
 0002:00000c10       ?PluginMenuStrings@?1??GetPluginInfoW@@9@4PAPEB_WA 0000000180016c10     Brackets.obj
 0002:00000c18       ?__proc_attached@@3HA      0000000180016c18     LIBCMT:dll_dllmain.obj
 0002:00000c30       ?module_local_atexit_table@@3U_onexit_table_t@@A 0000000180016c30     LIBCMT:utility.obj
 0002:00000c48       ?module_local_at_quick_exit_table@@3U_onexit_table_t@@A 0000000180016c48     LIBCMT:utility.obj
 0002:00000c60       ?is_initialized_as_dll@@3_NA 0000000180016c60     LIBCMT:utility.obj
 0002:00000ca0       ?module_handles@@3PAPEAUHINSTANCE__@@A 0000000180016ca0     libvcruntime:winapi_downlevel.obj
 0002:00000cc0       ?encoded_function_pointers@@3PAPEAXA 0000000180016cc0     libvcruntime:winapi_downlevel.obj
 0002:00000d10       ?__vcrt_startup_thread_ptd@@3U__vcrt_ptd@@A 0000000180016d10     libvcruntime:per_thread_data.obj
 0002:00000d88       __vcrt_lock_table          0000000180016d88     libvcruntime:locks.obj
 0002:00000db0       __vcrt_locks_initialized   0000000180016db0     libvcruntime:locks.obj
 0002:00000e08       ?heap@@3V_HeapManager@@A   0000000180016e08     libvcruntime:undname.obj
 0002:00000e30       __acrt_new_handler         0000000180016e30     libucrt:new_handler.obj
 0002:00000e38       c_termination_complete     0000000180016e38     libucrt:exit.obj
 0002:00000e40       thread_local_exit_callback_func 0000000180016e40     libucrt:exit.obj
 0002:00000e48       ?c_exit_complete@?5??common_exit@@YAXHW4_crt_exit_cleanup_mode@@W4_crt_exit_return_mode@@@Z@4_NA 0000000180016e48     libucrt:exit.obj
 0002:00000ea0       __acrt_lock_table          0000000180016ea0     libucrt:locks.obj
 0002:000010a8       __acrt_locks_initialized   00000001800170a8     libucrt:locks.obj
 0002:000010b0       module_handles             00000001800170b0     libucrt:winapi_thunks.obj
 0002:00001150       encoded_function_pointers  0000000180017150     libucrt:winapi_thunks.obj
 0002:00001250       ?state_cache@?1??__acrt_is_packaged_app@@9@4JA 0000000180017250     libucrt:winapi_thunks.obj
 0002:00001258       __acrt_invalid_parameter_handler 0000000180017258     libucrt:invalid_parameter.obj
 0002:00001274       fSystemSet                 0000000180017274     libucrt:mbctype.obj
 0002:00001280       ?initialized@?1??__acrt_initialize_multibyte@@9@4_NA 0000000180017280     libucrt:mbctype.obj
 0002:000016b8       ctrlc_action               00000001800176b8     libucrt:signal.obj
 0002:000016c0       ctrlbreak_action           00000001800176c0     libucrt:signal.obj
 0002:000016c8       abort_action               00000001800176c8     libucrt:signal.obj
 0002:000016d0       term_action                00000001800176d0     libucrt:signal.obj
 0002:000016d8       user_matherr               00000001800176d8     libucrt:matherr.obj
 0002:000016f8       __acrt_global_new_mode     00000001800176f8     libucrt:new_mode.obj
 0002:0000171c       __acrt_app_type            000000018001771c     libucrt:report_runtime_error.obj
 0002:00001730       GS_ExceptionRecord         0000000180017730     LIBCMT:gs_report.obj
 0002:000017d0       GS_ContextRecord           00000001800177d0     LIBCMT:gs_report.obj
 0003:00000000       $pdata$?TraceLoggingRegister@__vcrt_trace_logging_provider@@YAJPEBU_TlgProvider_t@1@PEBU_GUID@@P6AX1KE_K2PEAU_EVENT_FILTER_DESCRIPTOR@@PEAX@Z4@Z 0000000180018000     libvcruntime:telemetry.obj
 0003:0000000c       $pdata$?_TlgEnableCallback@__vcrt_trace_logging_provider@@YAXPEBU_GUID@@KE_K1PEAU_EVENT_FILTER_DESCRIPTOR@@PEAX@Z 000000018001800c     libvcruntime:telemetry.obj
 0003:00000018       $pdata$?_TlgWrite@__vcrt_trace_logging_provider@@YAJPEBU_TlgProvider_t@1@PEFBXPEBU_GUID@@2IPEAU_EVENT_DATA_DESCRIPTOR@@@Z 0000000180018018     libvcruntime:telemetry.obj
 0003:00000030       $pdata$??0PluginIntEditFieldBinding@@QEAA@AEBUPluginStartupInfo@@PEAPEAXHPEAHH@Z 0000000180018030     Brackets.obj
 0003:0000003c       $pdata$??0PluginUIntEditFieldBinding@@QEAA@AEBUPluginStartupInfo@@PEAPEAXHPEAIH@Z 000000018001803c     Brackets.obj
 0003:00000048       $pdata$??1?$DialogBuilderBase@UFarDialogItem@@@@MEAA@XZ 0000000180018048     Brackets.obj
 0003:00000054       $pdata$0$??1?$DialogBuilderBase@UFarDialogItem@@@@MEAA@XZ 0000000180018054     Brackets.obj
 0003:00000060       $pdata$1$??1?$DialogBuilderBase@UFarDialogItem@@@@MEAA@XZ 0000000180018060     Brackets.obj
 0003:0000006c       $pdata$??_G?$DialogBuilderBase@UFarDialogItem@@@@MEAAPEAXI@Z 000000018001806c     Brackets.obj
 0003:00000078       $pdata$??_G?$DialogItemBinding@UFarDialogItem@@@@UEAAPEAXI@Z 0000000180018078     Brackets.obj
 0003:00000084       $pdata$??_GPluginDialogBuilder@@UEAAPEAXI@Z 0000000180018084     Brackets.obj
 0003:00000090       $pdata$??_GPluginCheckBoxBinding@@UEAAPEAXI@Z 0000000180018090     Brackets.obj
 0003:00000090       $pdata$??_GPluginEditFieldBinding@@UEAAPEAXI@Z 0000000180018090     Brackets.obj
 0003:0000009c       $pdata$??_GPluginRadioButtonBinding@@UEAAPEAXI@Z 000000018001809c     Brackets.obj
 0003:000000a8       $pdata$??_GPluginUIntEditFieldBinding@@UEAAPEAXI@Z 00000001800180a8     Brackets.obj
 0003:000000a8       $pdata$??_GPluginIntEditFieldBinding@@UEAAPEAXI@Z 00000001800180a8     Brackets.obj
 0003:000000b4       $pdata$?AddButtons@?$DialogBuilderBase@UFarDialogItem@@@@QEAAXHPEBHHH@Z 00000001800180b4     Brackets.obj
 0003:000000c0       $pdata$3$?AddButtons@?$DialogBuilderBase@UFarDialogItem@@@@QEAAXHPEBHHH@Z 00000001800180c0     Brackets.obj
 0003:000000cc       $pdata$4$?AddButtons@?$DialogBuilderBase@UFarDialogItem@@@@QEAAXHPEBHHH@Z 00000001800180cc     Brackets.obj
 0003:000000d8       $pdata$?AddIntEditField@PluginDialogBuilder@@UEAAPEAUFarDialogItem@@PEAHH@Z 00000001800180d8     Brackets.obj
 0003:000000e4       $pdata$?AddUIntEditField@PluginDialogBuilder@@UEAAPEAUFarDialogItem@@PEAIH@Z 00000001800180e4     Brackets.obj
 0003:000000f0       $pdata$?Config@@YAHXZ      00000001800180f0     Brackets.obj
 0003:000000fc       $pdata$?CreateCheckBoxBinding@PluginDialogBuilder@@MEAAPEAU?$DialogItemBinding@UFarDialogItem@@@@PEAHH@Z 00000001800180fc     Brackets.obj
 0003:00000108       $pdata$?CreateRadioButtonBinding@PluginDialogBuilder@@MEAAPEAU?$DialogItemBinding@UFarDialogItem@@@@PEAH@Z 0000000180018108     Brackets.obj
 0003:00000114       $pdata$?DoShowDialog@PluginDialogBuilder@@MEAA_JXZ 0000000180018114     Brackets.obj
 0003:00000120       $pdata$?InitDialogItem@PluginDialogBuilder@@MEAAXPEAUFarDialogItem@@PEB_W@Z 0000000180018120     Brackets.obj
 0003:0000012c       $pdata$?ItemWidth@?$DialogBuilderBase@UFarDialogItem@@@@IEAA_JAEBUFarDialogItem@@@Z 000000018001812c     Brackets.obj
 0003:00000138       $pdata$?MaxTextWidth@?$DialogBuilderBase@UFarDialogItem@@@@IEAA_JXZ 0000000180018138     Brackets.obj
 0003:00000144       $pdata$1$?MaxTextWidth@?$DialogBuilderBase@UFarDialogItem@@@@IEAA_JXZ 0000000180018144     Brackets.obj
 0003:00000150       $pdata$2$?MaxTextWidth@?$DialogBuilderBase@UFarDialogItem@@@@IEAA_JXZ 0000000180018150     Brackets.obj
 0003:0000015c       $pdata$?ReallocDialogItems@?$DialogBuilderBase@UFarDialogItem@@@@IEAAXXZ 000000018001815c     Brackets.obj
 0003:00000168       $pdata$?SaveValue@PluginCheckBoxBinding@@UEAAXPEAUFarDialogItem@@H@Z 0000000180018168     Brackets.obj
 0003:00000174       $pdata$?SaveValue@PluginEditFieldBinding@@UEAAXPEAUFarDialogItem@@H@Z 0000000180018174     Brackets.obj
 0003:00000180       $pdata$?SaveValue@PluginIntEditFieldBinding@@UEAAXPEAUFarDialogItem@@H@Z 0000000180018180     Brackets.obj
 0003:0000018c       $pdata$?SaveValue@PluginRadioButtonBinding@@UEAAXPEAUFarDialogItem@@H@Z 000000018001818c     Brackets.obj
 0003:00000198       $pdata$?SaveValue@PluginUIntEditFieldBinding@@UEAAXPEAUFarDialogItem@@H@Z 0000000180018198     Brackets.obj
 0003:000001a4       $pdata$?SaveValues@?$DialogBuilderBase@UFarDialogItem@@@@IEAAXXZ 00000001800181a4     Brackets.obj
 0003:000001b0       $pdata$1$?SaveValues@?$DialogBuilderBase@UFarDialogItem@@@@IEAAXXZ 00000001800181b0     Brackets.obj
 0003:000001bc       $pdata$2$?SaveValues@?$DialogBuilderBase@UFarDialogItem@@@@IEAAXXZ 00000001800181bc     Brackets.obj
 0003:000001c8       $pdata$?ShowMenu@@YAHH@Z   00000001800181c8     Brackets.obj
 0003:000001d4       $pdata$?UpdateBorderSize@?$DialogBuilderBase@UFarDialogItem@@@@IEAAXXZ 00000001800181d4     Brackets.obj
 0003:000001e0       $pdata$ConfigureW          00000001800181e0     Brackets.obj
 0003:000001ec       $pdata$GetGlobalInfoW      00000001800181ec     Brackets.obj
 0003:000001f8       $pdata$GetPluginInfoW      00000001800181f8     Brackets.obj
 0003:00000204       $pdata$OpenW               0000000180018204     Brackets.obj
 0003:00000210       $pdata$SetStartupInfoW     0000000180018210     Brackets.obj
 0003:0000021c       $pdata$??2@YAPEAX_K@Z      000000018001821c     LIBCMT:new_scalar.obj
 0003:00000228       $pdata$?dllmain_crt_dispatch@@YAHQEAUHINSTANCE__@@KQEAX@Z 0000000180018228     LIBCMT:dll_dllmain.obj
 0003:00000234       $pdata$?dllmain_crt_process_attach@@YAHQEAUHINSTANCE__@@QEAX@Z 0000000180018234     LIBCMT:dll_dllmain.obj
 0003:00000240       $pdata$?dllmain_crt_process_detach@@YAH_N@Z 0000000180018240     LIBCMT:dll_dllmain.obj
 0003:0000024c       $pdata$?dllmain_dispatch@@YAHQEAUHINSTANCE__@@KQEAX@Z 000000018001824c     LIBCMT:dll_dllmain.obj
 0003:00000258       $pdata$?dllmain_raw@@YAHQEAUHINSTANCE__@@KQEAX@Z 0000000180018258     LIBCMT:dll_dllmain.obj
 0003:00000264       $pdata$_DllMainCRTStartup  0000000180018264     LIBCMT:dll_dllmain.obj
 0003:00000270       $pdata$??0bad_alloc@std@@QEAA@AEBV01@@Z 0000000180018270     LIBCMT:throw_bad_alloc.obj
 0003:0000027c       $pdata$??0bad_array_new_length@std@@QEAA@AEBV01@@Z 000000018001827c     LIBCMT:throw_bad_alloc.obj
 0003:00000288       $pdata$??0exception@std@@QEAA@AEBV01@@Z 0000000180018288     LIBCMT:throw_bad_alloc.obj
 0003:00000294       $pdata$??_Gbad_alloc@std@@UEAAPEAXI@Z 0000000180018294     LIBCMT:throw_bad_alloc.obj
 0003:00000294       $pdata$??_Gexception@std@@UEAAPEAXI@Z 0000000180018294     LIBCMT:throw_bad_alloc.obj
 0003:00000294       $pdata$??_Gbad_array_new_length@std@@UEAAPEAXI@Z 0000000180018294     LIBCMT:throw_bad_alloc.obj
 0003:000002a0       $pdata$?__scrt_throw_std_bad_alloc@@YAXXZ 00000001800182a0     LIBCMT:throw_bad_alloc.obj
 0003:000002ac       $pdata$?__scrt_throw_std_bad_array_new_length@@YAXXZ 00000001800182ac     LIBCMT:throw_bad_alloc.obj
 0003:000002b8       $pdata$__scrt_acquire_startup_lock 00000001800182b8     LIBCMT:utility.obj
 0003:000002c4       $pdata$__scrt_dllmain_after_initialize_c 00000001800182c4     LIBCMT:utility.obj
 0003:000002d0       $pdata$__scrt_dllmain_before_initialize_c 00000001800182d0     LIBCMT:utility.obj
 0003:000002dc       $pdata$__scrt_dllmain_crt_thread_attach 00000001800182dc     LIBCMT:utility.obj
 0003:000002e8       $pdata$__scrt_dllmain_crt_thread_detach 00000001800182e8     LIBCMT:utility.obj
 0003:000002f4       $pdata$__scrt_dllmain_exception_filter 00000001800182f4     LIBCMT:utility.obj
 0003:00000300       $pdata$__scrt_dllmain_uninitialize_c 0000000180018300     LIBCMT:utility.obj
 0003:0000030c       $pdata$__scrt_dllmain_uninitialize_critical 000000018001830c     LIBCMT:utility.obj
 0003:00000318       $pdata$__scrt_initialize_crt 0000000180018318     LIBCMT:utility.obj
 0003:00000324       $pdata$__scrt_initialize_onexit_tables 0000000180018324     LIBCMT:utility.obj
 0003:00000330       $pdata$__scrt_is_nonwritable_in_current_image 0000000180018330     LIBCMT:utility.obj
 0003:0000033c       $pdata$__scrt_release_startup_lock 000000018001833c     LIBCMT:utility.obj
 0003:00000348       $pdata$__scrt_uninitialize_crt 0000000180018348     LIBCMT:utility.obj
 0003:00000354       $pdata$_onexit             0000000180018354     LIBCMT:utility.obj
 0003:00000360       $pdata$atexit              0000000180018360     LIBCMT:utility.obj
 0003:0000036c       $pdata$__security_init_cookie 000000018001836c     LIBCMT:gs_support.obj
 0003:00000378       $pdata$__scrt_initialize_default_local_stdio_options 0000000180018378     LIBCMT:default_local_stdio_options.obj
 0003:00000384       $pdata$__scrt_fastfail     0000000180018384     LIBCMT:utility_desktop.obj
 0003:00000390       $pdata$_RTC_Initialize     0000000180018390     LIBCMT:_initsect_.obj
 0003:0000039c       $pdata$_RTC_Terminate      000000018001839c     LIBCMT:_initsect_.obj
 0003:000003a8       $pdata$??_Gtype_info@@UEAAPEAXI@Z 00000001800183a8     LIBCMT:std_type_info_static.obj
 0003:000003b4       $pdata$__isa_available_init 00000001800183b4     LIBCMT:_cpu_disp_.obj
 0003:000003cc       $pdata$__telemetry_main_invoke_trigger 00000001800183cc     libvcruntime:telemetry.obj
 0003:000003d8       $pdata$__telemetry_main_return_trigger 00000001800183d8     libvcruntime:telemetry.obj
 0003:000003e4       $pdata$__vcrt_uninitialize_telemetry_provider 00000001800183e4     libvcruntime:telemetry.obj
 0003:000003f0       $pdata$__C_specific_handler 00000001800183f0     libvcruntime:_chandler_.obj
 0003:000003fc       $pdata$__std_exception_copy 00000001800183fc     libvcruntime:std_exception.obj
 0003:00000408       $pdata$__std_exception_destroy 0000000180018408     libvcruntime:std_exception.obj
 0003:00000414       $pdata$_CxxThrowException  0000000180018414     libvcruntime:throw.obj
 0003:00000420       $pdata$__vcrt_initialize   0000000180018420     libvcruntime:initialization.obj
 0003:0000042c       $pdata$__vcrt_thread_attach 000000018001842c     libvcruntime:initialization.obj
 0003:00000438       $pdata$__vcrt_thread_detach 0000000180018438     libvcruntime:initialization.obj
 0003:00000444       $pdata$__vcrt_uninitialize 0000000180018444     libvcruntime:initialization.obj
 0003:00000450       $pdata$__vcrt_uninitialize_critical 0000000180018450     libvcruntime:initialization.obj
 0003:0000045c       $pdata$__std_type_info_destroy_list 000000018001845c     libvcruntime:std_type_info.obj
 0003:00000468       $pdata$?try_get_function@@YAPEAXW4function_id@?A0x61ce2399@@QEBDQEBW4module_id@2@2@Z 0000000180018468     libvcruntime:winapi_downlevel.obj
 0003:00000474       $pdata$__vcrt_EventRegister 0000000180018474     libvcruntime:winapi_downlevel.obj
 0003:00000480       $pdata$__vcrt_EventSetInformation 0000000180018480     libvcruntime:winapi_downlevel.obj
 0003:0000048c       $pdata$__vcrt_EventUnregister 000000018001848c     libvcruntime:winapi_downlevel.obj
 0003:00000498       $pdata$__vcrt_EventWriteTransfer 0000000180018498     libvcruntime:winapi_downlevel.obj
 0003:000004a4       $pdata$__vcrt_FlsAlloc     00000001800184a4     libvcruntime:winapi_downlevel.obj
 0003:000004b0       $pdata$__vcrt_FlsFree      00000001800184b0     libvcruntime:winapi_downlevel.obj
 0003:000004bc       $pdata$__vcrt_FlsGetValue  00000001800184bc     libvcruntime:winapi_downlevel.obj
 0003:000004c8       $pdata$__vcrt_FlsSetValue  00000001800184c8     libvcruntime:winapi_downlevel.obj
 0003:000004d4       $pdata$__vcrt_InitializeCriticalSectionEx 00000001800184d4     libvcruntime:winapi_downlevel.obj
 0003:000004e0       $pdata$__vcrt_initialize_winapi_thunks 00000001800184e0     libvcruntime:winapi_downlevel.obj
 0003:000004ec       $pdata$__vcrt_uninitialize_winapi_thunks 00000001800184ec     libvcruntime:winapi_downlevel.obj
 0003:00000528       $pdata$__vcrt_freefls      0000000180018528     libvcruntime:per_thread_data.obj
 0003:00000534       $pdata$__vcrt_freeptd      0000000180018534     libvcruntime:per_thread_data.obj
 0003:00000540       $pdata$__vcrt_getptd_noexit 0000000180018540     libvcruntime:per_thread_data.obj
 0003:0000054c       $pdata$__vcrt_initialize_ptd 000000018001854c     libvcruntime:per_thread_data.obj
 0003:00000558       $pdata$__vcrt_uninitialize_ptd 0000000180018558     libvcruntime:per_thread_data.obj
 0003:00000564       $pdata$__vcrt_initialize_locks 0000000180018564     libvcruntime:locks.obj
 0003:00000570       $pdata$__vcrt_uninitialize_locks 0000000180018570     libvcruntime:locks.obj
 0003:0000057c       $pdata$_callnewh           000000018001857c     libucrt:new_handler.obj
 0003:00000588       $pdata$_query_new_handler  0000000180018588     libucrt:new_handler.obj
 0003:00000594       $pdata$_initterm           0000000180018594     libucrt:initterm.obj
 0003:000005a0       $pdata$_initterm_e         00000001800185a0     libucrt:initterm.obj
 0003:000005ac       $pdata$_seh_filter_exe     00000001800185ac     libucrt:exception_filter.obj
 0003:000005b8       $pdata$?common_exit@@YAXHW4_crt_exit_cleanup_mode@@W4_crt_exit_return_mode@@@Z 00000001800185b8     libucrt:exit.obj
 0003:000005c4       $pdata$?exit_or_terminate_process@@YAXI@Z 00000001800185c4     libucrt:exit.obj
 0003:000005d0       $pdata$?try_cor_exit_process@@YAXI@Z 00000001800185d0     libucrt:exit.obj
 0003:000005dc       $pdata$??$common_initialize_environment_nolock@D@@YAHXZ 00000001800185dc     libucrt:environment_initialization.obj
 0003:000005e8       $pdata$??$create_environment@D@@YAQEAPEADQEAD@Z 00000001800185e8     libucrt:environment_initialization.obj
 0003:000005f4       $pdata$??$free_environment@_W@@YAXQEAPEA_W@Z 00000001800185f4     libucrt:environment_initialization.obj
 0003:000005f4       $pdata$??$free_environment@D@@YAXQEAPEAD@Z 00000001800185f4     libucrt:environment_initialization.obj
 0003:00000600       $pdata$??$uninitialize_environment_internal@D@@YAXAEAPEAPEAD@Z 0000000180018600     libucrt:environment_initialization.obj
 0003:0000060c       $pdata$??$uninitialize_environment_internal@_W@@YAXAEAPEAPEA_W@Z 000000018001860c     libucrt:environment_initialization.obj
 0003:00000618       $pdata$__dcrt_uninitialize_environments_nolock 0000000180018618     libucrt:environment_initialization.obj
 0003:00000624       $pdata$??$?RV<lambda_b8c45f8f788dd370798f47cfe8ac3a86>@@AEAV<lambda_4e60a939b0d047cfe11ddc22648dfba9>@@V<lambda_332c3edc96d0294ec56c57d38c1cdfd5>@@@?$__crt_seh_guarded_call@H@@QEAAH$$QEAV<lambda_b8c45f8f788dd370798f47cfe8ac3a86>@@AEAV<lambda_4e60a939b0d047cfe11ddc22648dfba9>@@$$QEAV<lambda_332c3edc96d0294ec56c57d38c1cdfd5>@@@Z 0000000180018624     libucrt:onexit.obj
 0003:00000630       $pdata$??$?RV<lambda_e24bbb7b643b32fcea6fa61b31d4c984>@@AEAV<lambda_275893d493268fdec8709772e3fcec0e>@@V<lambda_9d71df4d7cf3f480f8d633942495c3b0>@@@?$__crt_seh_guarded_call@H@@QEAAH$$QEAV<lambda_e24bbb7b643b32fcea6fa61b31d4c984>@@AEAV<lambda_275893d493268fdec8709772e3fcec0e>@@$$QEAV<lambda_9d71df4d7cf3f480f8d633942495c3b0>@@@Z 0000000180018630     libucrt:onexit.obj
 0003:0000063c       $pdata$??R<lambda_4e60a939b0d047cfe11ddc22648dfba9>@@QEBAHXZ 000000018001863c     libucrt:onexit.obj
 0003:00000648       $pdata$_execute_onexit_table 0000000180018648     libucrt:onexit.obj
 0003:00000654       $pdata$_register_onexit_function 0000000180018654     libucrt:onexit.obj
 0003:00000660       $pdata$initialize_c        0000000180018660     libucrt:initialization.obj
 0003:0000066c       $pdata$uninitialize_environment 000000018001866c     libucrt:initialization.obj
 0003:00000678       $pdata$initialize_pointers 0000000180018678     libucrt:initialization.obj
 0003:00000684       $pdata$uninitialize_allocated_memory 0000000180018684     libucrt:initialization.obj
 0003:00000690       $pdata$__acrt_thread_attach 0000000180018690     libucrt:initialization.obj
 0003:0000069c       $pdata$__acrt_thread_detach 000000018001869c     libucrt:initialization.obj
 0003:000006a8       $pdata$__acrt_uninitialize_critical 00000001800186a8     libucrt:initialization.obj
 0003:000006b4       $pdata$terminate           00000001800186b4     libucrt:terminate.obj
 0003:000006c0       $pdata$strcpy_s            00000001800186c0     libucrt:strcpy_s.obj
 0003:000006cc       $pdata$_free_base          00000001800186cc     libucrt:free_base.obj
 0003:000006d8       $pdata$_malloc_base        00000001800186d8     libucrt:malloc_base.obj
 0003:000006e4       $pdata$abort               00000001800186e4     libucrt:abort.obj
 0003:000006f0       $pdata$_calloc_base        00000001800186f0     libucrt:calloc_base.obj
 0003:000006fc       $pdata$??0_LocaleUpdate@@QEAA@QEAU__crt_locale_pointers@@@Z 00000001800186fc     libucrt:output.obj
 0003:00000708       $pdata$__acrt_initialize_locks 0000000180018708     libucrt:locks.obj
 0003:00000714       $pdata$__acrt_uninitialize_locks 0000000180018714     libucrt:locks.obj
 0003:00000720       $pdata$??$?RV<lambda_46352004c1216016012b18bd6f87e700>@@AEAV<lambda_3bd07e1a1191394380780325891bf33f>@@V<lambda_334532d3f185bcaa59b5be82d7d22bff>@@@?$__crt_seh_guarded_call@X@@QEAAX$$QEAV<lambda_46352004c1216016012b18bd6f87e700>@@AEAV<lambda_3bd07e1a1191394380780325891bf33f>@@$$QEAV<lambda_334532d3f185bcaa59b5be82d7d22bff>@@@Z 0000000180018720     libucrt:per_thread_data.obj
 0003:0000072c       $pdata$??$?RV<lambda_5e887d1dcbef67a5eb4283622ba103bf>@@AEAV<lambda_4466841279450cc726390878d4a41900>@@V<lambda_341c25c0346d94847f1f3c463c57e077>@@@?$__crt_seh_guarded_call@X@@QEAAX$$QEAV<lambda_5e887d1dcbef67a5eb4283622ba103bf>@@AEAV<lambda_4466841279450cc726390878d4a41900>@@$$QEAV<lambda_341c25c0346d94847f1f3c463c57e077>@@@Z 000000018001872c     libucrt:per_thread_data.obj
 0003:00000738       $pdata$??$?RV<lambda_72d1df2b273a38828b1ce30cbf4cdab5>@@AEAV<lambda_876a65b173b8412d3a47c70a915b0cf4>@@V<lambda_41932305e351933ebe8f8be3ed8bb5dc>@@@?$__crt_seh_guarded_call@X@@QEAAX$$QEAV<lambda_72d1df2b273a38828b1ce30cbf4cdab5>@@AEAV<lambda_876a65b173b8412d3a47c70a915b0cf4>@@$$QEAV<lambda_41932305e351933ebe8f8be3ed8bb5dc>@@@Z 0000000180018738     libucrt:per_thread_data.obj
 0003:00000744       $pdata$??$?RV<lambda_fb3a7dec4e47f37f22dae91bb15c9095>@@AEAV<lambda_698284760c8add0bfb0756c19673e34b>@@V<lambda_dfb8eca1e75fef3034a8fb18dd509707>@@@?$__crt_seh_guarded_call@X@@QEAAX$$QEAV<lambda_fb3a7dec4e47f37f22dae91bb15c9095>@@AEAV<lambda_698284760c8add0bfb0756c19673e34b>@@$$QEAV<lambda_dfb8eca1e75fef3034a8fb18dd509707>@@@Z 0000000180018744     libucrt:per_thread_data.obj
 0003:00000750       $pdata$?construct_ptd_array@@YAXQEAU__acrt_ptd@@@Z 0000000180018750     libucrt:per_thread_data.obj
 0003:0000075c       $pdata$?destroy_fls@@YAXPEAX@Z 000000018001875c     libucrt:per_thread_data.obj
 0003:00000768       $pdata$?destroy_ptd_array@@YAXQEAU__acrt_ptd@@@Z 0000000180018768     libucrt:per_thread_data.obj
 0003:00000774       $pdata$?replace_current_thread_locale_nolock@@YAXQEAU__acrt_ptd@@QEAU__crt_locale_data@@@Z 0000000180018774     libucrt:per_thread_data.obj
 0003:00000780       $pdata$__acrt_freeptd      0000000180018780     libucrt:per_thread_data.obj
 0003:0000078c       $pdata$__acrt_getptd       000000018001878c     libucrt:per_thread_data.obj
 0003:00000798       $pdata$__acrt_getptd_noexit 0000000180018798     libucrt:per_thread_data.obj
 0003:000007a4       $pdata$__acrt_initialize_ptd 00000001800187a4     libucrt:per_thread_data.obj
 0003:000007b0       $pdata$__acrt_uninitialize_ptd 00000001800187b0     libucrt:per_thread_data.obj
 0003:000007bc       $pdata$?try_get_function@@YAPEAXW4function_id@?A0x63058377@@QEBDQEBW4module_id@2@2@Z 00000001800187bc     libucrt:winapi_thunks.obj
 0003:000007c8       $pdata$__acrt_FlsAlloc     00000001800187c8     libucrt:winapi_thunks.obj
 0003:000007d4       $pdata$__acrt_FlsFree      00000001800187d4     libucrt:winapi_thunks.obj
 0003:000007e0       $pdata$__acrt_FlsGetValue  00000001800187e0     libucrt:winapi_thunks.obj
 0003:000007ec       $pdata$__acrt_FlsSetValue  00000001800187ec     libucrt:winapi_thunks.obj
 0003:000007f8       $pdata$__acrt_InitializeCriticalSectionEx 00000001800187f8     libucrt:winapi_thunks.obj
 0003:00000804       $pdata$__acrt_LCMapStringEx 0000000180018804     libucrt:winapi_thunks.obj
 0003:00000810       $pdata$__acrt_LocaleNameToLCID 0000000180018810     libucrt:winapi_thunks.obj
 0003:0000081c       $pdata$__acrt_initialize_winapi_thunks 000000018001881c     libucrt:winapi_thunks.obj
 0003:00000828       $pdata$__acrt_is_packaged_app 0000000180018828     libucrt:winapi_thunks.obj
 0003:00000834       $pdata$__acrt_uninitialize_winapi_thunks 0000000180018834     libucrt:winapi_thunks.obj
 0003:00000840       $pdata$__acrt_call_reportfault 0000000180018840     libucrt:invalid_parameter.obj
 0003:0000084c       $pdata$_invalid_parameter  000000018001884c     libucrt:invalid_parameter.obj
 0003:00000858       $pdata$_invalid_parameter_noinfo 0000000180018858     libucrt:invalid_parameter.obj
 0003:00000864       $pdata$_invoke_watson      0000000180018864     libucrt:invalid_parameter.obj
 0003:00000870       $pdata$??$?RV<lambda_99476a1ad63dd22509b5d3e65b0ffc95>@@AEAV<lambda_ad1ced32f4ac17aa236e5ef05d6b3b7c>@@V<lambda_f7424dd8d45958661754dc4f2697e9c3>@@@?$__crt_seh_guarded_call@X@@QEAAX$$QEAV<lambda_99476a1ad63dd22509b5d3e65b0ffc95>@@AEAV<lambda_ad1ced32f4ac17aa236e5ef05d6b3b7c>@@$$QEAV<lambda_f7424dd8d45958661754dc4f2697e9c3>@@@Z 0000000180018870     libucrt:mbctype.obj
 0003:0000087c       $pdata$??R<lambda_ad1ced32f4ac17aa236e5ef05d6b3b7c>@@QEBAXXZ 000000018001887c     libucrt:mbctype.obj
 0003:00000888       $pdata$?getSystemCP@@YAHH@Z 0000000180018888     libucrt:mbctype.obj
 0003:00000894       $pdata$?setSBCS@@YAXPEAU__crt_multibyte_data@@@Z 0000000180018894     libucrt:mbctype.obj
 0003:000008a0       $pdata$?setSBUpLow@@YAXPEAU__crt_multibyte_data@@@Z 00000001800188a0     libucrt:mbctype.obj
 0003:000008ac       $pdata$?setmbcp_internal@@YAHH_N@Z 00000001800188ac     libucrt:mbctype.obj
 0003:000008b8       $pdata$__acrt_initialize_multibyte 00000001800188b8     libucrt:mbctype.obj
 0003:000008c4       $pdata$__acrt_update_thread_multibyte_data 00000001800188c4     libucrt:mbctype.obj
 0003:000008d0       $pdata$_setmbcp_nolock     00000001800188d0     libucrt:mbctype.obj
 0003:000008dc       $pdata$__dcrt_get_narrow_environment_from_os 00000001800188dc     libucrt:get_environment_from_os.obj
 0003:000008e8       $pdata$_recalloc_base      00000001800188e8     libucrt:recalloc.obj
 0003:000008f4       $pdata$__acrt_initialize_heap 00000001800188f4     libucrt:heap_handle.obj
 0003:00000900       $pdata$?initialize_inherited_file_handles_nolock@@YAXXZ 0000000180018900     libucrt:ioinit.obj
 0003:0000090c       $pdata$?initialize_stdio_handles_nolock@@YAXXZ 000000018001890c     libucrt:ioinit.obj
 0003:00000918       $pdata$__acrt_initialize_lowio 0000000180018918     libucrt:ioinit.obj
 0003:00000924       $pdata$__acrt_uninitialize_lowio 0000000180018924     libucrt:ioinit.obj
 0003:00000930       $pdata$__acrt_initialize_command_line 0000000180018930     libucrt:argv_data.obj
 0003:0000093c       $pdata$__acrt_execute_initializers 000000018001893c     libucrt:shared_initialization.obj
 0003:00000948       $pdata$__acrt_execute_uninitializers 0000000180018948     libucrt:shared_initialization.obj
 0003:00000954       $pdata$??$?RV<lambda_c36588078e9f5dfd39652860aa6b3aaf>@@AEAV<lambda_ec61778202f4f5fc7e7711acc23c3bca>@@V<lambda_dc9d2797ccde5d239b4a0efae8ebd7db>@@@?$__crt_seh_guarded_call@P6AXH@Z@@QEAAP6AXH@Z$$QEAV<lambda_c36588078e9f5dfd39652860aa6b3aaf>@@AEAV<lambda_ec61778202f4f5fc7e7711acc23c3bca>@@$$QEAV<lambda_dc9d2797ccde5d239b4a0efae8ebd7db>@@@Z 0000000180018954     libucrt:signal.obj
 0003:00000960       $pdata$__acrt_get_sigabrt_handler 0000000180018960     libucrt:signal.obj
 0003:0000096c       $pdata$raise               000000018001896c     libucrt:signal.obj
 0003:00000978       $pdata$__acrt_invoke_user_matherr 0000000180018978     libucrt:matherr.obj
 0003:00000984       $pdata$__acrt_errno_map_os_error 0000000180018984     libucrt:errno.obj
 0003:00000990       $pdata$__doserrno          0000000180018990     libucrt:errno.obj
 0003:0000099c       $pdata$_errno              000000018001899c     libucrt:errno.obj
 0003:000009a8       $pdata$_mbtowc_l           00000001800189a8     libucrt:mbtowc.obj
 0003:000009b4       $pdata$__acrt_update_locale_info 00000001800189b4     libucrt:locale_update.obj
 0003:000009c0       $pdata$__acrt_update_multibyte_info 00000001800189c0     libucrt:locale_update.obj
 0003:000009cc       $pdata$_fileno             00000001800189cc     libucrt:fileno.obj
 0003:000009d8       $pdata$__acrt_initialize_stdio 00000001800189d8     libucrt:_file.obj
 0003:000009e4       $pdata$__acrt_uninitialize_stdio 00000001800189e4     libucrt:_file.obj
 0003:000009f0       $pdata$__acrt_uninitialize_locale 00000001800189f0     libucrt:wsetlocale.obj
 0003:000009fc       $pdata$__pctype_func       00000001800189fc     libucrt:ctype.obj
 0003:00000a08       $pdata$__acrt_free_locale  0000000180018a08     libucrt:locale_refcounting.obj
 0003:00000a14       $pdata$__acrt_locale_free_lc_time_if_unreferenced 0000000180018a14     libucrt:locale_refcounting.obj
 0003:00000a20       $pdata$__acrt_release_locale_ref 0000000180018a20     libucrt:locale_refcounting.obj
 0003:00000a2c       $pdata$__acrt_update_thread_locale_data 0000000180018a2c     libucrt:locale_refcounting.obj
 0003:00000a38       $pdata$_updatetlocinfoEx_nolock 0000000180018a38     libucrt:locale_refcounting.obj
 0003:00000a44       $pdata$?GetTableIndexFromLocaleName@@YAHPEB_W@Z 0000000180018a44     libucrt:lcidtoname_downlevel.obj
 0003:00000a50       $pdata$__acrt_DownlevelLocaleNameToLCID 0000000180018a50     libucrt:lcidtoname_downlevel.obj
 0003:00000a5c       $pdata$?initialize_multibyte@@YAHXZ 0000000180018a5c     libucrt:multibyte_initializer.obj
 0003:00000a68       $pdata$__acrt_GetStringTypeA 0000000180018a68     libucrt:getstringtypea.obj
 0003:00000a74       $pdata$?__acrt_LCMapStringA_stat@@YAHPEAU__crt_locale_pointers@@PEB_WKPEBDHPEADHHH@Z 0000000180018a74     libucrt:lcmapstringa.obj
 0003:00000a80       $pdata$__acrt_LCMapStringA 0000000180018a80     libucrt:lcmapstringa.obj
 0003:00000a8c       $pdata$_msize              0000000180018a8c     libucrt:msize.obj
 0003:00000a98       $pdata$_realloc_base       0000000180018a98     libucrt:realloc_base.obj
 0003:00000aa4       $pdata$__acrt_lowio_create_handle_array 0000000180018aa4     libucrt:osfinfo.obj
 0003:00000ab0       $pdata$__acrt_lowio_destroy_handle_array 0000000180018ab0     libucrt:osfinfo.obj
 0003:00000abc       $pdata$__acrt_lowio_ensure_fh_exists 0000000180018abc     libucrt:osfinfo.obj
 0003:00000ac8       $pdata$_free_osfhnd        0000000180018ac8     libucrt:osfinfo.obj
 0003:00000ad4       $pdata$_get_osfhandle      0000000180018ad4     libucrt:osfinfo.obj
 0003:00000ae0       $pdata$_isatty             0000000180018ae0     libucrt:isatty.obj
 0003:00000aec       $pdata$__acrt_stdio_flush_nolock 0000000180018aec     libucrt:fflush.obj
 0003:00000af8       $pdata$_fflush_nolock      0000000180018af8     libucrt:fflush.obj
 0003:00000b04       $pdata$common_flush_all    0000000180018b04     libucrt:fflush.obj
 0003:00000b10       $pdata$_isleadbyte_l       0000000180018b10     libucrt:_wctype.obj
 0003:00000b1c       $pdata$_fcloseall          0000000180018b1c     libucrt:closeall.obj
 0003:00000b28       $pdata$__acrt_stdio_free_buffer_nolock 0000000180018b28     libucrt:_freebuf.obj
 0003:00000b34       $pdata$__acrt_locale_free_monetary 0000000180018b34     libucrt:initmon.obj
 0003:00000b40       $pdata$__acrt_locale_free_numeric 0000000180018b40     libucrt:initnum.obj
 0003:00000b4c       $pdata$?free_crt_array_internal@@YAXQEAPEBX_K@Z 0000000180018b4c     libucrt:inittime.obj
 0003:00000b58       $pdata$__acrt_locale_free_time 0000000180018b58     libucrt:inittime.obj
 0003:00000b64       $pdata$??$?RV<lambda_b521505b218e5242e90febf6bfebc422>@@AEAV<lambda_6978c1fb23f02e42e1d9e99668cc68aa>@@V<lambda_314360699dd331753a4119843814e9a7>@@@?$__crt_seh_guarded_call@H@@QEAAH$$QEAV<lambda_b521505b218e5242e90febf6bfebc422>@@AEAV<lambda_6978c1fb23f02e42e1d9e99668cc68aa>@@$$QEAV<lambda_314360699dd331753a4119843814e9a7>@@@Z 0000000180018b64     libucrt:commit.obj
 0003:00000b70       $pdata$_commit             0000000180018b70     libucrt:commit.obj
 0003:00000b7c       $pdata$?write_double_translated_ansi_nolock@@YA?AUwrite_result@?A0x9c548279@@HQEBDI@Z 0000000180018b7c     libucrt:write.obj
 0003:00000b88       $pdata$?write_text_ansi_nolock@@YA?AUwrite_result@?A0x9c548279@@HQEBDI@Z 0000000180018b88     libucrt:write.obj
 0003:00000b94       $pdata$?write_text_utf16le_nolock@@YA?AUwrite_result@?A0x9c548279@@HQEBDI@Z 0000000180018b94     libucrt:write.obj
 0003:00000ba0       $pdata$?write_text_utf8_nolock@@YA?AUwrite_result@?A0x9c548279@@HQEBDI@Z 0000000180018ba0     libucrt:write.obj
 0003:00000bac       $pdata$_write              0000000180018bac     libucrt:write.obj
 0003:00000bb8       $pdata$_write_nolock       0000000180018bb8     libucrt:write.obj
 0003:00000bd0       $pdata$??$common_lseek_nolock@_J@@YA_JH_JH@Z 0000000180018bd0     libucrt:lseek.obj
 0003:00000bdc       $pdata$_fclose_nolock      0000000180018bdc     libucrt:fclose.obj
 0003:00000be8       $pdata$fclose              0000000180018be8     libucrt:fclose.obj
 0003:00000bf4       $pdata$_putwch_nolock      0000000180018bf4     libucrt:putwch.obj
 0003:00000c00       $pdata$_call_matherr       0000000180018c00     libucrt:libm_error.obj
 0003:00000c0c       $pdata$_exception_enabled  0000000180018c0c     libucrt:libm_error.obj
 0003:00000c18       $pdata$_handle_error       0000000180018c18     libucrt:libm_error.obj
 0003:00000c24       $pdata$__acrt_initialize_fma3 0000000180018c24     libucrt:fma3_available.obj
 0003:00000c30       $pdata$_log10_special      0000000180018c30     libucrt:log_special.obj
 0003:00000c3c       $pdata$_log_special_common 0000000180018c3c     libucrt:log_special.obj
 0003:00000c48       $pdata$??$?RV<lambda_bfedae4ebbf01fab1bb6dcc6a9e276e0>@@AEAV<lambda_2fe9b910cf3cbf4a0ab98a02ba45b3ec>@@V<lambda_237c231691f317818eb88cc1d5d642d6>@@@?$__crt_seh_guarded_call@H@@QEAAH$$QEAV<lambda_bfedae4ebbf01fab1bb6dcc6a9e276e0>@@AEAV<lambda_2fe9b910cf3cbf4a0ab98a02ba45b3ec>@@$$QEAV<lambda_237c231691f317818eb88cc1d5d642d6>@@@Z 0000000180018c48     libucrt:close.obj
 0003:00000c54       $pdata$_close              0000000180018c54     libucrt:close.obj
 0003:00000c60       $pdata$_close_nolock       0000000180018c60     libucrt:close.obj
 0003:00000c6c       $pdata$__dcrt_lowio_initialize_console_output 0000000180018c6c     libucrt:initcon.obj
 0003:00000c78       $pdata$__dcrt_terminate_console_output 0000000180018c78     libucrt:initcon.obj
 0003:00000c90       $pdata$_raise_exc          0000000180018c90     libucrt:fpexcept.obj
 0003:00000c9c       $pdata$_raise_exc_ex       0000000180018c9c     libucrt:fpexcept.obj
 0003:00000ca8       $pdata$_set_errno_from_matherr 0000000180018ca8     libucrt:fpexcept.obj
 0003:00000cb4       $pdata$_clrfp              0000000180018cb4     libucrt:fpctrl.obj
 0003:00000cc0       $pdata$_ctrlfp             0000000180018cc0     libucrt:fpctrl.obj
 0003:00000ccc       $pdata$_set_statfp         0000000180018ccc     libucrt:fpctrl.obj
 0003:00000cd8       $pdata$_statfp             0000000180018cd8     libucrt:fpctrl.obj
 0003:00000ce4       $pdata$__GSHandlerCheck    0000000180018ce4     LIBCMT:_gshandler_.obj
 0003:00000cf0       $pdata$__GSHandlerCheckCommon 0000000180018cf0     LIBCMT:_gshandler_.obj
 0003:00000d08       $pdata$_IsNonwritableInCurrentImage 0000000180018d08     LIBCMT:pesect.obj
 0003:00000d14       $pdata$__raise_securityfailure 0000000180018d14     LIBCMT:gs_report.obj
 0003:00000d20       $pdata$__report_gsfailure  0000000180018d20     LIBCMT:gs_report.obj
 0003:00000d2c       $pdata$capture_previous_context 0000000180018d2c     LIBCMT:gs_report.obj
 0003:00000d5c       $pdata$?fin$0@?0??dllmain_crt_process_attach@@YAHQEAUHINSTANCE__@@QEAX@Z@4HA 0000000180018d5c     LIBCMT:dll_dllmain.obj
 0003:00000d68       $pdata$?fin$0@?0??dllmain_crt_process_detach@@YAH_N@Z@4HA 0000000180018d68     LIBCMT:dll_dllmain.obj
 0003:00000d74       $pdata$?filt$0@?0??dllmain_dispatch@@YAHQEAUHINSTANCE__@@KQEAX@Z@4HA 0000000180018d74     LIBCMT:dll_dllmain.obj
 0003:00000d80       $pdata$__scrt_is_nonwritable_in_current_image$filt$0 0000000180018d80     LIBCMT:utility.obj
 0003:00000d8c       $pdata$_query_new_handler$fin$0 0000000180018d8c     libucrt:new_handler.obj
 0003:00000d98       $pdata$?filt$0@?0??common_exit@@YAXHW4_crt_exit_cleanup_mode@@W4_crt_exit_return_mode@@@Z@4HA 0000000180018d98     libucrt:exit.obj
 0003:00000da4       $pdata$?fin$1@?0??common_exit@@YAXHW4_crt_exit_cleanup_mode@@W4_crt_exit_return_mode@@@Z@4HA 0000000180018da4     libucrt:exit.obj
 0003:00000db0       $pdata$?fin$0@?0???$?RV<lambda_e24bbb7b643b32fcea6fa61b31d4c984>@@AEAV<lambda_275893d493268fdec8709772e3fcec0e>@@V<lambda_9d71df4d7cf3f480f8d633942495c3b0>@@@?$__crt_seh_guarded_call@H@@QEAAH$$QEAV<lambda_e24bbb7b643b32fcea6fa61b31d4c984>@@AEAV<lambda_275893d493268fdec8709772e3fcec0e>@@$$QEAV<lambda_9d71df4d7cf3f480f8d633942495c3b0>@@@Z@4HA 0000000180018db0     libucrt:onexit.obj
 0003:00000dbc       $pdata$?fin$0@?0???$?RV<lambda_46352004c1216016012b18bd6f87e700>@@AEAV<lambda_3bd07e1a1191394380780325891bf33f>@@V<lambda_334532d3f185bcaa59b5be82d7d22bff>@@@?$__crt_seh_guarded_call@X@@QEAAX$$QEAV<lambda_46352004c1216016012b18bd6f87e700>@@AEAV<lambda_3bd07e1a1191394380780325891bf33f>@@$$QEAV<lambda_334532d3f185bcaa59b5be82d7d22bff>@@@Z@4HA 0000000180018dbc     libucrt:per_thread_data.obj
 0003:00000dbc       $pdata$?fin$0@?0???$?RV<lambda_c36588078e9f5dfd39652860aa6b3aaf>@@AEAV<lambda_ec61778202f4f5fc7e7711acc23c3bca>@@V<lambda_dc9d2797ccde5d239b4a0efae8ebd7db>@@@?$__crt_seh_guarded_call@P6AXH@Z@@QEAAP6AXH@Z$$QEAV<lambda_c36588078e9f5dfd39652860aa6b3aaf>@@AEAV<lambda_ec61778202f4f5fc7e7711acc23c3bca>@@$$QEAV<lambda_dc9d2797ccde5d239b4a0efae8ebd7db>@@@Z@4HA 0000000180018dbc     libucrt:signal.obj
 0003:00000dbc       $pdata$?fin$0@?0???$?RV<lambda_5e887d1dcbef67a5eb4283622ba103bf>@@AEAV<lambda_4466841279450cc726390878d4a41900>@@V<lambda_341c25c0346d94847f1f3c463c57e077>@@@?$__crt_seh_guarded_call@X@@QEAAX$$QEAV<lambda_5e887d1dcbef67a5eb4283622ba103bf>@@AEAV<lambda_4466841279450cc726390878d4a41900>@@$$QEAV<lambda_341c25c0346d94847f1f3c463c57e077>@@@Z@4HA 0000000180018dbc     libucrt:per_thread_data.obj
 0003:00000dbc       $pdata$?fin$0@?0???$?RV<lambda_fb3a7dec4e47f37f22dae91bb15c9095>@@AEAV<lambda_698284760c8add0bfb0756c19673e34b>@@V<lambda_dfb8eca1e75fef3034a8fb18dd509707>@@@?$__crt_seh_guarded_call@X@@QEAAX$$QEAV<lambda_fb3a7dec4e47f37f22dae91bb15c9095>@@AEAV<lambda_698284760c8add0bfb0756c19673e34b>@@$$QEAV<lambda_dfb8eca1e75fef3034a8fb18dd509707>@@@Z@4HA 0000000180018dbc     libucrt:per_thread_data.obj
 0003:00000dbc       $pdata$?fin$0@?0???$?RV<lambda_72d1df2b273a38828b1ce30cbf4cdab5>@@AEAV<lambda_876a65b173b8412d3a47c70a915b0cf4>@@V<lambda_41932305e351933ebe8f8be3ed8bb5dc>@@@?$__crt_seh_guarded_call@X@@QEAAX$$QEAV<lambda_72d1df2b273a38828b1ce30cbf4cdab5>@@AEAV<lambda_876a65b173b8412d3a47c70a915b0cf4>@@$$QEAV<lambda_41932305e351933ebe8f8be3ed8bb5dc>@@@Z@4HA 0000000180018dbc     libucrt:per_thread_data.obj
 0003:00000dbc       $pdata$?fin$0@?0???$?RV<lambda_99476a1ad63dd22509b5d3e65b0ffc95>@@AEAV<lambda_ad1ced32f4ac17aa236e5ef05d6b3b7c>@@V<lambda_f7424dd8d45958661754dc4f2697e9c3>@@@?$__crt_seh_guarded_call@X@@QEAAX$$QEAV<lambda_99476a1ad63dd22509b5d3e65b0ffc95>@@AEAV<lambda_ad1ced32f4ac17aa236e5ef05d6b3b7c>@@$$QEAV<lambda_f7424dd8d45958661754dc4f2697e9c3>@@@Z@4HA 0000000180018dbc     libucrt:mbctype.obj
 0003:00000dbc       $pdata$?fin$0@?0???$?RV<lambda_b8c45f8f788dd370798f47cfe8ac3a86>@@AEAV<lambda_4e60a939b0d047cfe11ddc22648dfba9>@@V<lambda_332c3edc96d0294ec56c57d38c1cdfd5>@@@?$__crt_seh_guarded_call@H@@QEAAH$$QEAV<lambda_b8c45f8f788dd370798f47cfe8ac3a86>@@AEAV<lambda_4e60a939b0d047cfe11ddc22648dfba9>@@$$QEAV<lambda_332c3edc96d0294ec56c57d38c1cdfd5>@@@Z@4HA 0000000180018dbc     libucrt:onexit.obj
 0003:00000dc8       $pdata$__acrt_update_thread_multibyte_data$fin$0 0000000180018dc8     libucrt:mbctype.obj
 0003:00000dd4       $pdata$__acrt_lowio_ensure_fh_exists$fin$0 0000000180018dd4     libucrt:osfinfo.obj
 0003:00000dd4       $pdata$__acrt_initialize_lowio$fin$0 0000000180018dd4     libucrt:ioinit.obj
 0003:00000de0       $pdata$raise$fin$0         0000000180018de0     libucrt:signal.obj
 0003:00000dec       $pdata$__acrt_uninitialize_locale$fin$0 0000000180018dec     libucrt:wsetlocale.obj
 0003:00000dec       $pdata$__acrt_update_thread_locale_data$fin$0 0000000180018dec     libucrt:locale_refcounting.obj
 0003:00000df8       $pdata$common_flush_all$fin$0 0000000180018df8     libucrt:fflush.obj
 0003:00000e04       $pdata$common_flush_all$fin$1 0000000180018e04     libucrt:fflush.obj
 0003:00000e10       $pdata$_fcloseall$fin$0    0000000180018e10     libucrt:closeall.obj
 0003:00000e1c       $pdata$?fin$0@?0???$?RV<lambda_bfedae4ebbf01fab1bb6dcc6a9e276e0>@@AEAV<lambda_2fe9b910cf3cbf4a0ab98a02ba45b3ec>@@V<lambda_237c231691f317818eb88cc1d5d642d6>@@@?$__crt_seh_guarded_call@H@@QEAAH$$QEAV<lambda_bfedae4ebbf01fab1bb6dcc6a9e276e0>@@AEAV<lambda_2fe9b910cf3cbf4a0ab98a02ba45b3ec>@@$$QEAV<lambda_237c231691f317818eb88cc1d5d642d6>@@@Z@4HA 0000000180018e1c     libucrt:close.obj
 0003:00000e1c       $pdata$?fin$0@?0???$?RV<lambda_b521505b218e5242e90febf6bfebc422>@@AEAV<lambda_6978c1fb23f02e42e1d9e99668cc68aa>@@V<lambda_314360699dd331753a4119843814e9a7>@@@?$__crt_seh_guarded_call@H@@QEAAH$$QEAV<lambda_b521505b218e5242e90febf6bfebc422>@@AEAV<lambda_6978c1fb23f02e42e1d9e99668cc68aa>@@$$QEAV<lambda_314360699dd331753a4119843814e9a7>@@@Z@4HA 0000000180018e1c     libucrt:commit.obj
 0003:00000e28       $pdata$_write$fin$0        0000000180018e28     libucrt:write.obj
 0003:00000e34       $pdata$fclose$fin$0        0000000180018e34     libucrt:fclose.obj
 0003:00000e40       $pdata$_ctrlfp$filt$0      0000000180018e40     libucrt:fpctrl.obj
 0003:00000e4c       $pdata$_IsNonwritableInCurrentImage$filt$0 0000000180018e4c     LIBCMT:pesect.obj
 0004:000004f4       .idata$6                   00000001800194f4     kernel32:KERNEL32.dll
 0004:00000510       .idata$6                   0000000180019510     user32:USER32.dll
 0004:000009e8       .idata$6                   00000001800199e8     advapi32:ADVAPI32.dll
 0005:00000000       __guard_fids__             000000018001a000     libucrt:initialization.obj
 0005:00000060       __guard_fids___acrt_initialize_ptd 000000018001a060     libucrt:per_thread_data.obj
 0005:00000064       __guard_fids__             000000018001a064     libucrt:multibyte_initializer.obj
 0005:00000068       __guard_fids__             000000018001a068     libucrt:stdio_initializer.obj
 0005:0000006c       __guard_fids__             000000018001a06c     libucrt:stdio_initializer.obj
 0005:00000070       __guard_fids__             000000018001a070     libucrt:locale_initializer.obj
 0005:00000074       __guard_fids__             000000018001a074     libucrt:fma3_initializer.obj
 0005:00000078       __guard_fids__             000000018001a078     libucrt:console_output_initializer.obj
 0005:0000007c       __guard_fids_?dllmain_crt_process_attach@@YAHQEAUHINSTANCE__@@QEAX@Z 000000018001a07c     LIBCMT:dll_dllmain.obj
 0005:00000084       __guard_fids_?dllmain_dispatch@@YAHQEAUHINSTANCE__@@KQEAX@Z 000000018001a084     LIBCMT:dll_dllmain.obj
 0005:00000088       __guard_fids__             000000018001a088     LIBCMT:throw_bad_alloc.obj
 0005:00000090       __guard_fids__             000000018001a090     LIBCMT:throw_bad_alloc.obj
 0005:00000098       __guard_fids__             000000018001a098     LIBCMT:throw_bad_alloc.obj
 0005:000000a0       __guard_fids__             000000018001a0a0     LIBCMT:std_type_info_static.obj
 0005:000000a4       __guard_fids__             000000018001a0a4     LIBCMT:guard_support.obj
 0005:000000a8       __guard_fids__             000000018001a0a8     libvcruntime:telemetry.obj
 0005:000000ac       __guard_fids_?TraceLoggingRegister@__vcrt_trace_logging_provider@@YAJPEBU_TlgProvider_t@1@PEBU_GUID@@P6AX1KE_K2PEAU_EVENT_FILTER_DESCRIPTOR@@PEAX@Z4@Z 000000018001a0ac     libvcruntime:telemetry.obj
 0005:000000b0       __guard_fids___vcrt_initialize_ptd 000000018001a0b0     libvcruntime:per_thread_data.obj
 0006:00000060       $R000000                   000000018001b060     Brackets.res
